:020000040800F2
:10000000005000204D240008FD2400080936000897
:10001000FD240008FD240008FD2400080000000065
:10002000000000000000000000000000FD240008A7
:10003000FD24000800000000FD2400087954000899
:10004000FD240008FD240008FD240008FD2400080C
:10005000FD240008FD240008FD240008FD240008FC
:10006000FD240008FD240008FD240008FD240008EC
:10007000FD240008FD2400088D530008FD2400081D
:10008000FD240008FD240008FD240008FD240008CC
:10009000FD240008FD240008FD240008FD240008BC
:1000A000FD240008FD240008FD2400082124000888
:1000B0002D2400083524000841240008754B000851
:1000C000F54E0008794B0008F14E0008FD240008A9
:1000D000FD240008C1530008FD530008FD2400085A
:1000E000FD240008FD240008FD2400080000000095
:1000F0000000000000000000000000000000000000
:0C01000000000000000000005FF808F1A3
:1001100010B5054C237833B9044810B10448AFF347
:1001200000800121217010BD9C050020000000000E
:10013000440F010808B5064B1BB106480649AFF34A
:1001400000800648016811B1054A02B1904708BD18
:1001500000000000440F0108A00500209C050020BD
:100160000000000081F0004102E000BF83F0004386
:1001700030B54FEA41044FEA430594EA050F08BF42
:1001800090EA020F1FBF54EA000C55EA020C7FEA06
:10019000645C7FEA655C00F0E2804FEA5454D4EB83
:1001A0005555B8BF6D420CDD2C4480EA020281EA4D
:1001B000030382EA000083EA010180EA020281EA85
:1001C0000303362D88BF30BD11F0004F4FEA0131D7
:1001D0004FF4801C4CEA113102D0404261EB4101E6
:1001E00013F0004F4FEA03334CEA133302D052426C
:1001F00063EB430394EA050F00F0A780A4F1010428
:10020000D5F1200E0DDB02FA0EFC22FA05F2801861
:1002100041F1000103FA0EF2801843FA05F3594147
:100220000EE0A5F120050EF1200E012A03FA0EFCC6
:1002300028BF4CF0020C43FA05F3C01851EBE371F0
:1002400001F0004507D54FF0000EDCF1000C7EEB0D
:1002500000006EEB0101B1F5801F1BD3B1F5001F4B
:100260000CD349085FEA30004FEA3C0C04F101046A
:100270004FEA445212F5800F80F09A80BCF1004F93
:1002800008BF5FEA500C50F1000041EB045141EA15
:10029000050130BD5FEA4C0C404141EB010111F416
:1002A000801FA4F10104E9D191F0000F04BF0146C1
:1002B0000020B1FA81F308BF2033A3F10B03B3F19F
:1002C00020020CDA0C3208DD02F1140CC2F10C022F
:1002D00001FA0CF021FA02F10CE002F11402D8BF8D
:1002E000C2F1200C01FA02F120FA0CFCDCBF41EA59
:1002F0000C019040E41AA2BF01EB0451294330BD28
:100300006FEA04041F3C1CDA0C340EDC04F1140404
:10031000C4F1200220FA04F001FA02F340EA0300DB
:1003200021FA04F345EA030130BDC4F10C04C4F121
:10033000200220FA02F001FA04F340EA0300294601
:1003400030BD21FA04F0294630BD94F0000F83F44B
:10035000801306BF81F480110134013D4EE77FEA2E
:10036000645C18BF7FEA655C29D094EA050F08BF7A
:1003700090EA020F05D054EA000C04BF194610465B
:1003800030BD91EA030F1EBF0021002030BD5FEA9F
:10039000545C05D14000494128BF41F0004130BDC7
:1003A00014F580043CBF01F5801130BD01F000451B
:1003B00045F0FE4141F470014FF0000030BD7FEA8E
:1003C000645C1ABF194610467FEA655C1CBF0B4689
:1003D000024650EA013406BF52EA033591EA030FA0
:1003E00041F4002130BD00BF90F0000F04BF002198
:1003F000704730B54FF4806404F132044FF00005CB
:100400004FF0000150E700BF90F0000F04BF002143
:10041000704730B54FF4806404F1320410F00045A9
:1004200048BF40424FF000013EE700BF42004FEAA4
:10043000E2014FEA31014FEA02701FBF12F07F4321
:1004400093F07F4F81F06051704792F0000F14BF1E
:1004500093F07F4F704730B54FF4607401F0004562
:1004600021F0004120E700BF50EA010208BF7047B9
:1004700030B54FF000050AE050EA010208BF7047AE
:1004800030B511F0004502D5404261EB41014FF417
:10049000806404F132045FEA915C3FF4DCAE4FF01B
:1004A00003025FEADC0C18BF03325FEADC0C18BF02
:1004B000033202EBDC02C2F1200300FA03FC20FA53
:1004C00002F001FA03FE40EA0E0021FA02F11444A0
:1004D000C1E600BF70B54FF0FF0C4CF4E06C1CEAB5
:1004E00011541DBF1CEA135594EA0C0F95EA0C0F2A
:1004F00000F0DEF82C4481EA030621EA4C5123EA9D
:100500004C5350EA013518BF52EA033541F48011CB
:1005100043F4801338D0A0FB02CE4FF00005E1FB7E
:1005200002E506F00042E0FB03E54FF00006E1FBC8
:1005300003569CF0000F18BF4EF0010EA4F1FF040B
:10054000B6F5007F64F5407404D25FEA4E0E6D414B
:1005500046EB060642EAC62141EA55514FEAC5205C
:1005600040EA5E504FEACE2EB4F1FD0C88BFBCF5D8
:10057000E06F1ED8BEF1004F08BF5FEA500E50F189
:10058000000041EB045170BD06F0004646EA01014F
:1005900040EA020081EA0301B4EB5C04C2BFD4EB81
:1005A0000C0541EA045170BD41F480114FF0000E7A
:1005B000013C00F3AB8014F1360FDEBF002001F0E8
:1005C000004170BDC4F10004203C35DA0C341BDC62
:1005D00004F11404C4F1200500FA05F320FA04F034
:1005E00001FA05F240EA020001F0004221F0004168
:1005F00010EBD37021FA04F642EB06015EEA430EDB
:1006000008BF20EAD37070BDC4F10C04C4F120050A
:1006100000FA04F320FA05F001FA04F240EA0200BD
:1006200001F0004110EBD37041F100015EEA430E8E
:1006300008BF20EAD37070BDC4F1200500FA05F2AE
:100640004EEA020E20FA04F301FA05F243EA02032D
:1006500021FA04F001F0004121FA04F220EA02003C
:1006600000EBD3705EEA430E08BF20EAD37070BD82
:1006700094F0000F0FD101F00046400041EB010162
:1006800011F4801F08BF013CF7D041EA060195F044
:10069000000F18BF704703F00046520043EB0303FE
:1006A00013F4801F08BF013DF7D043EA06037047EB
:1006B00094EA0C0F0CEA135518BF95EA0C0F0CD0F6
:1006C00050EA410618BF52EA4306D1D181EA03013C
:1006D00001F000414FF0000070BD50EA410606BF36
:1006E0001046194652EA430619D094EA0C0F02D17B
:1006F00050EA013613D195EA0C0F05D152EA0336C0
:100700001CBF104619460AD181EA030101F00041DD
:1007100041F0FE4141F470014FF0000070BD41F026
:10072000FE4141F4780170BD70B54FF0FF0C4CF400
:10073000E06C1CEA11541DBF1CEA135594EA0C0F1F
:1007400095EA0C0F00F0A7F8A4EB050481EA030E6C
:1007500052EA03354FEA013100F088804FEA033353
:100760004FF0805545EA131343EA12634FEA022221
:1007700045EA111545EA10654FEA00260EF00041E2
:100780009D4208BF964244F1FD0404F5407402D234
:100790005B084FEA3202B61A65EB03055B084FEAC5
:1007A00032024FF480104FF4002CB6EB020E75EBC2
:1007B000030E22BFB61A754640EA0C005B084FEAEA
:1007C0003202B6EB020E75EB030E22BFB61A754667
:1007D00040EA5C005B084FEA3202B6EB020E75EBB2
:1007E000030E22BFB61A754640EA9C005B084FEA2A
:1007F0003202B6EB020E75EB030E22BFB61A754637
:1008000040EADC0055EA060E18D04FEA051545EA25
:1008100016754FEA06164FEAC30343EA52734FEACE
:10082000C2025FEA1C1CC0D111F4801F0BD141EA47
:1008300000014FF000004FF0004CB6E711F4801FAC
:1008400004BF01430020B4F1FD0C88BFBCF5E06F8C
:100850003FF6AFAEB5EB030C04BFB6EB020C5FEA9C
:10086000500C50F1000041EB045170BD0EF0004EF1
:100870004EEA113114EB5C04C2BFD4EB0C0541EA23
:10088000045170BD41F480114FF0000E013C90E620
:1008900045EA060E8DE60CEA135594EA0C0F08BFE4
:1008A00095EA0C0F3FF43BAF94EA0C0F0AD150EAE3
:1008B00001347FF434AF95EA0C0F7FF425AF104676
:1008C00019462CE795EA0C0F06D152EA03353FF49E
:1008D000FDAE1046194622E750EA410618BF52EA1B
:1008E00043067FF4C5AE50EA41047FF40DAF52EAEF
:1008F00043057FF4EBAE12E74FEA4102B2F1E04369
:1009000024BFB3F5001CDCF1FE5C0DD901F0004CF6
:100910004FEAC0024CEA5070B2F1004F40EB830046
:1009200008BF20F00100704711F0804F21D113F172
:100930003872BCBF01F00040704741F480114FEAAB
:100940005252C2F11802C2F1200C10FA0CF320FA34
:1009500002F018BF40F001004FEAC1234FEAD32351
:1009600003FA0CFC40EA0C0023FA02F34FEA4303BB
:10097000CCE77FEA625307D150EA01331EBF4FF044
:10098000FE4040F44000704701F0004040F0FE405F
:1009900040F40000704700BF80F0004002E000BF5C
:1009A00081F0004142001FBF5FEA410392EA030F5A
:1009B0007FEA226C7FEA236C6AD04FEA1262D2EBA4
:1009C0001363C1BFD218414048404140B8BF5B42A9
:1009D000192B88BF704710F0004F40F4000020F042
:1009E0007F4018BF404211F0004F41F4000121F058
:1009F0007F4118BF494292EA030F3FD0A2F10102A2
:100A000041FA03FC10EB0C00C3F1200301FA03F1DF
:100A100000F0004302D5494260EB4000B0F5000F02
:100A200013D3B0F1807F06D340084FEA310102F1C1
:100A30000102FE2A51D2B1F1004F40EBC25008BF73
:100A400020F0010040EA03007047490040EB00003D
:100A500010F4000FA2F10102EDD1B0FA80FCACF16C
:100A6000080CB2EB0C0200FA0CF0AABF00EBC2506B
:100A700052421843BCBFD0401843704792F0000F59
:100A800081F4000106BF80F400000132013BB5E7AC
:100A90004FEA41037FEA226C18BF7FEA236C21D022
:100AA00092EA030F04D092F0000F08BF0846704787
:100AB00090EA010F1CBF0020704712F07F4F04D155
:100AC000400028BF40F00040704712F100723CBF68
:100AD00000F50000704700F0004343F0FE4040F492
:100AE000000070477FEA226216BF08467FEA236350
:100AF0000146420206BF5FEA412390EA010F40F43B
:100B0000800070474FF0000304E000BF10F0004386
:100B100048BF40425FEA000C08BF704743F096436D
:100B200001464FF000001CE050EA010208BF704788
:100B30004FF000030AE000BF50EA010208BF70470F
:100B400011F0004302D5404261EB41015FEA010C24
:100B500002BF84460146002043F0B64308BFA3F11C
:100B60008053A3F50003BCFA8CF2083AA3EBC253FE
:100B700010DB01FA02FC634400FA02FCC2F120021D
:100B8000BCF1004F20FA02F243EB020008BF20F054
:100B90000100704702F1200201FA02FCC2F12002BA
:100BA00050EA4C0021FA02F243EB020008BF20EAAF
:100BB000DC7070474FF0FF0C1CEAD0521EBF1CEADD
:100BC000D15392EA0C0F93EA0C0F6FD01A4480EACB
:100BD000010C400218BF5FEA41211ED04FF00063B4
:100BE00043EA501043EA5111A0FB01310CF00040E0
:100BF000B1F5000F3EBF490041EAD3715B0040EA06
:100C0000010062F17F02FD2A1DD8B3F1004F40EBD5
:100C1000C25008BF20F00100704790F0000F0CF0A8
:100C2000004C08BF49024CEA502040EA51207F3A6C
:100C3000C2BFD2F1FF0340EAC250704740F4000047
:100C40004FF00003013A5DDC12F1190FDCBF00F038
:100C500000407047C2F10002410021FA02F1C2F1E6
:100C6000200200FA02FC5FEA310040F1000053EA82
:100C70004C0308BF20EADC70704792F0000F00F0D0
:100C8000004C02BF400010F4000F013AF9D040EAD6
:100C90000C0093F0000F01F0004C02BF490011F46A
:100CA000000F013BF9D041EA0C018FE70CEAD15368
:100CB00092EA0C0F18BF93EA0C0F0AD030F0004CE8
:100CC00018BF31F0004CD8D180EA010000F000409C
:100CD000704790F0000F17BF90F0004F084691F05A
:100CE000000F91F0004F14D092EA0C0F01D1420294
:100CF0000FD193EA0C0F03D14B0218BF084608D15D
:100D000080EA010000F0004040F0FE4040F40000A6
:100D1000704740F0FE4040F4400070474FF0FF0C39
:100D20001CEAD0521EBF1CEAD15392EA0C0F93EA80
:100D30000C0F69D0A2EB030280EA010C49024FEAD2
:100D4000402037D04FF0805343EA111143EA10138B
:100D50000CF000408B4238BF5B0042F17D024FF443
:100D6000000C8B4224BF5B1A40EA0C00B3EB510F1E
:100D700024BFA3EB510340EA5C00B3EB910F24BF07
:100D8000A3EB910340EA9C00B3EBD10F24BFA3EB8C
:100D9000D10340EADC001B0118BF5FEA1C1CE0D154
:100DA000FD2A3FF650AF8B4240EBC25008BF20F007
:100DB000010070470CF0004C4CEA50207F32C2BF5B
:100DC000D2F1FF0340EAC250704740F400004FF0F8
:100DD0000003013A37E792F0000F00F0004C02BF29
:100DE000400010F4000F013AF9D040EA0C0093F0F3
:100DF000000F01F0004C02BF490011F4000F013B4D
:100E0000F9D041EA0C0195E70CEAD15392EA0C0FB4
:100E100008D142027FF47DAF93EA0C0F7FF470AFEC
:100E2000084676E793EA0C0F04D14B023FF44CAF2F
:100E300008466EE730F0004C18BF31F0004CCAD1C4
:100E400030F000427FF45CAF31F000437FF43CAF00
:100E50005FE700BF4FF0FF3C06E000BF4FF0010C22
:100E600002E000BF4FF0010C4DF804CD4FEA400204
:100E70004FEA41037FEA226C18BF7FEA236C11D04E
:100E800001B052EA530C18BF90EA010F58BFB2EB01
:100E9000030088BFC81738BF6FEAE17018BF40F081
:100EA000010070477FEA226C02D15FEA402C05D135
:100EB0007FEA236CE4D15FEA412CE1D05DF8040BBA
:100EC000704700BF844608466146FFE70FB5FFF74D
:100ED000C9FF002848BF10F1000F0FBD4DF808ED05
:100EE000FFF7F4FF0CBF012000205DF808FB00BFF6
:100EF0004DF808EDFFF7EAFF34BF012000205DF850
:100F000008FB00BF4DF808EDFFF7E0FF94BF01209C
:100F100000205DF808FB00BF4DF808EDFFF7D2FF99
:100F200094BF012000205DF808FB00BF4DF808EDDC
:100F3000FFF7C8FF34BF012000205DF808FB00BFA9
:100F40004FEA4002B2F1FE4F0FD34FF09E03B3EBD6
:100F500012620DD94FEA002343F0004310F0004F16
:100F600023FA02F018BF404270474FF0000070476C
:100F700012F1610F01D1420205D110F0004008BF0B
:100F80006FF0004070474FF00000704742000ED2F3
:100F9000B2F1FE4F0BD34FF09E03B3EB126209D4B4
:100FA0004FEA002343F0004323FA02F070474FF06A
:100FB0000000704712F1610F01D1420202D14FF0DF
:100FC000FF3070474FF00000704700BF2DE9FF4130
:100FD000334B8046187800283BD00024254626460F
:100FE0002746082232210DEB0203532003F05EFE58
:100FF0009DF809109DF80800013400EB01239DF8CD
:101000000B109DF80A001AB200EB01239DF80D1099
:101010009DF80C00E4B2BF181AB200EB01239DF852
:101020000F10B618202C1AB2154401F07F0001D021
:101030000028D6D11B4B97FBF4F796FBF4F695FBF3
:10104000F4F5ADF80070ADF80260ADF804501C7016
:101050001DE03221062202AB532003F027FE9DF84B
:1010600009209DF808109DF80B0001EB02239DF864
:101070000A20ADF8003002EB00219DF80C309DF8FD
:101080000D00ADF8021003EB0022ADF80420064A73
:1010900068464146127801F057FBBDE8FF8100BF6A
:1010A000B8050020B905002000000020154B10B540
:1010B0001B7804462D21532008227BB103F0BAFE91
:1010C00031210A22532003F0B5FE2C210C2253209B
:1010D00003F0B0FE53203821902209E003F0AAFE6D
:1010E00031210A22532003F0A5FE53202C210A228D
:1010F00003F0A0FE044840F2091202800CB103493B
:101100000C7010BDB8050020120000200000002067
:1011100037B5104B05461A680F480C46002182422D
:101120008DF8071001D1002013E0532001220DF1AA
:10113000070303F0BBFD0028F5D09DF80710E52953
:10114000F1D12A780548064B064920601A70616083
:1011500001203EBD4C010020001BB700AD1000086F
:10116000B8050020CD0F000813B5022204461B214C
:1011700001AB682003F09AFD9DF804209DF805302E
:1011800043EA022000F54E5110314FF48C7291FB6E
:10119000F2F3233323801CBD1FB504461D21062214
:1011A0006B46682003F082FD9DF800209DF8013019
:1011B00043EA022001B2042391FBF3F29DF80200FE
:1011C0009DF80310ADF8082041EA002210B290FB10
:1011D000F3F19DF805209DF80400ADF80A1042EAED
:1011E0000021064A08B290FBF3F3214602A81278C8
:1011F000ADF80C3001F0A8FA1FBD00BF02000020BE
:1012000010B50446192004F06AF96820152100225F
:1012100003F010FE10B9032004F0D2F90D4B162193
:101220001A78682042F0180203F004FE1721002209
:10123000682003F0FFFD3D210122682003F0FAFD44
:1012400068203E21012203F0F5FD0CB10248047034
:1012500010BD00BF010000200200002038B5054687
:1012600019200C4604F03BF968201521002203F0F8
:10127000E1FD18B3124B13481349144A622C2B603A
:101280006860A960EA60124B0FD004D80A2C12D013
:10129000142C0CD10DE0BC2C04D0B4F5807F06D109
:1012A000002009E00120187038BD022004E003206E
:1012B00002E0042000E005201870012038BD00BFC6
:1012C00001120008991100086911000818449231B0
:1012D00001000020064B07491A7812B14FF4FF6352
:1012E00001E04FF480530B8008B1034A107070473F
:1012F000BA05002012000020030000201FB504469C
:10130000432106226B46682003F0D0FC9DF80020A4
:101310009DF8013043EA022001B2042391FBF3F26D
:101320009DF802009DF80310ADF8082041EA002264
:1013300010B290FBF3F19DF805209DF80400ADF884
:101340000A1042EA0021064A08B290FBF3F3214654
:1013500002A81278ADF80C3001F0F6F91FBD00BFFD
:10136000050000201FB504463B2106226B4668207D
:1013700003F09CFC9DF800209DF801309DF80210C0
:1013800043EA02209DF80320ADF8080042EA012359
:101390009DF804009DF80510ADF80A30054B41EAB0
:1013A0000022ADF80C2002A821461A7801F0CCF9F1
:1013B0001FBD00BF0300002013B5224A4FF40053A5
:1013C00004460220ADF804308DF8070013681E486B
:1013D000042183428DF8061001D11C4803E01C490A
:1013E0008B4203D11B4801A903F08CFD6B218022A5
:1013F000682003F01FFD052004F071F81921002278
:10140000682003F017FD6B210322682003F012FD12
:1014100037210222682003F00DFD0F4A1A211278AD
:10142000682003F007FD1B211822682003F002FD4D
:1014300068201C21102203F0FDFC0CB1074B1C702E
:101440001CBD00BF4C01002000127A00000C0140BE
:10145000001BB70000100140040000200500002020
:101460002DE9F043814685B023200E461446984668
:1014700004F035F86820752101220DF1070303F00F
:1014800015FC00286FD09DF80770682F6AD10621DF
:101490000A4602AB384603F009FC9DF80B309DF874
:1014A0000D5003F0010105F001004A0042EA8005F9
:1014B0009DF8090000F001031D4308D0012D01D162
:1014C0002A481AE0022D0ED10023284813E00C21EF
:1014D000012238460DF1070303F0E8FB9DF80710E1
:1014E00011F00F0203D1052004F06AF806E0042A87
:1014F0001E4802D10123037000E005701C491D4AFB
:10150000C9F800101C481D4B1D49C9F80420306063
:101510007360F160B8F1000F03D0144A107888F8B6
:101520000000142C174B15D004D8052C16D00A2C0B
:101530000ED111E0BC2C08D0B4F5807F03D0622C12
:1015400006D102210BE0002109E0012018700AE019
:10155000032104E0042102E0052100E006211970C6
:10156000012000E0002005B0BDE8F083BA050020AE
:10157000D512000865130008B9130008FD12000811
:1015800019449231040000201FB50446A821062208
:101590006B46682003F08AFB9DF800209DF801301F
:1015A00043EA022001B2042391FBF3F29DF802000A
:1015B0009DF80310ADF8082041EA002210B290FB1C
:1015C000F3F19DF805209DF80400ADF80A1042EAF9
:1015D0000021064A08B290FBF3F3214602A81278D4
:1015E000ADF80C3001F0B0F81FBD00BF06000020C0
:1015F00010B50446642003F072FF68202321F02216
:1016000003F018FC10B9032003F0DAFF052003F003
:1016100066FF064B68201A78202142F00F0203F083
:1016200009FC0CB10248047010BD00BFBB050020CE
:101630000600002037B5054619200C4603F04FFF81
:1016400068200F2101220DF1070303F02FFB9DF805
:101650000730D32B16D10C480C490D4A4E2C28606C
:101660006960EA600B4B07D05D2C09D0362C01D0A5
:10167000002002E0402000E080201870012002E0FD
:10168000C020FAE700203EBDF115000889150008CA
:10169000DDE9A731BB0500202DE9F041057890B0C8
:1016A00000350646334818BF012509F077FF0024AE
:1016B0003148A542314B0CBF2146802106904FF4A2
:1016C00000500CBF4FF001084FF002084FF4807239
:1016D00005930A9120234FF480670E9005A92548B1
:1016E0000B920D930C970794CDF8208009940F94DA
:1016F00009F0CCFF1F48012109F0F5FF4FF46021EC
:10170000012702911E48694600948DF804508DF817
:10171000057003948DF8108009F0E6F8184804214C
:101720003A46032309F031F92DB1154831780222E8
:10173000032309F02AF91248012109F002F910489F
:10174000012109F0F5F80E4809F004F90C4809F0F8
:1017500006F90028FAD10A4809F005F9084809F005
:1017600007F90028FAD10648012109F005F910B05F
:10177000BDE8F08108000240BC0500204C24014077
:1017800000240140024B33F8100080B2704700BFC4
:10179000BC050020F8B5134B05469B890E46144640
:1017A000ECB116B116F8017B00E0FF270D480221CD
:1017B00009F094F80028F9D00A48394609F089F868
:1017C0000848012109F08AF80028F9D0054809F0F5
:1017D00082F8C0B20DB105F8010B013CE0E7012031
:1017E000F8BD00BF003800402DE9F047012188B066
:1017F0004FF4804009F0CEFD374C01214FF480407A
:1018000009F0E0FD03214FF420401823ADF800005B
:101810008DF80310204669468DF802304FF0040819
:1018200003F070FB2D4E4FF4804220466946ADF820
:1018300000204FF480554FF0100A8DF8028003F01D
:1018400061FB69462046ADF800508DF802A003F018
:1018500059FB304608F0E0FF07214FF400700023E9
:101860000222ADF81600ADF81C104FF00109304609
:1018700003A94FF48277ADF80C30ADF81030ADF815
:101880001A30ADF81220ADF80E70ADF814901F4666
:10189000ADF818A008F0F2FF3046494609F00DF8FF
:1018A0009F238DF804308DF805708DF806708DF843
:1018B00007700DEB08014246656102A8FFF76AFF59
:1018C00025619DF80900B0F1EF014A4252EB010099
:1018D00008B0BDE8F08700BF000C014000380040B0
:1018E000074BA1F57A7153F82000838802684B43B7
:1018F0004FF47A7093FBF0F18BB21380704700BF06
:10190000C0060020024B53F8200002681180704787
:10191000C00600202DE9F04FDFF828814FEA0015BE
:1019200058F805408E468BB008EB050711468346F4
:10193000924620467246019300F0C0FCB96807F158
:1019400008024FF0020C18237868ADF8141005A9AE
:101950008DF816308DF817C00392CDF808C003F04B
:10196000D1FA0398364E077906A809F05AFA702280
:101970000198DDF808C0ADF81820012100234FF4CC
:10198000807206EB0509ADF81A10ADF81C30ADF801
:101990001E00ADF820C0ADF824200C2F2BD8DFE8B6
:1019A00007F0072A2A2A102A2A2A192A2A2A220074
:1019B000204606A909F02EF92046082109F066FA0A
:1019C00019E0204606A909F069F92046082109F026
:1019D00065FA10E0204606A909F0A4F9204608217E
:1019E00009F066FA07E0204606A909F0DDF920466D
:1019F000082109F065FA08EB0B118B7B1BB120461F
:101A0000012109F02CFA2046012109F01CFA0C2FC3
:101A100010D8DFE807F0070F0F0F090F0F0F0B0F9C
:101A20000F0F0D00343404E0383402E03C3400E0A1
:101A300040347451A9F804A048460BB0BDE8F08FBB
:101A4000D4050020CCE800081B4A1C4813881180EC
:101A5000C91A89B240F68C2291420380184B02D9F0
:101A600000221A707047A1F2EF2080B240F2DA52E1
:101A7000904218D81B78072B15D81248032B20F852
:101A80001310114A09D811480088884205D2012153
:101A900001FA03F310780343137012780F2A02D16E
:101AA000094B002119700648094B0278511C01703E
:101AB00000201880704700BFC0050020B606002037
:101AC000D2050020C2050020B80600200800002032
:101AD0006A0700207FB5044601A80D46164609F0A6
:101AE000AAF900200123ADF80A00ADF80C0001A905
:101AF0002046ADF80450ADF80660ADF8083009F0A6
:101B00001BFA7FBD2DE9F743DFF858800501144E1D
:101B100005EB0804A3688946761928210746B271A7
:101B2000606802228DF8061001A9ADF804308DF826
:101B3000072003F0E7F955F80800217B0022FFF7A2
:101B4000C9FF204601224FF6FF7100F0D9FB204665
:101B500039464A4600F094FB3046BDE8FE8300BF9C
:101B6000D4050020CCE8000810B5134B00011B1869
:101B7000DA795AB901221981DA71104B0222191847
:101B8000097B1858BDE81040FFF7A4BF1C89598194
:101B90000B4A091B9C7989B222F814100024998100
:101BA000DC71064B22461918097B1858FFF792FF83
:101BB0000448048010BD00BFD4050020CCE8000814
:101BC000C20500206A0700202DE9F0410446028A80
:101BD000484B807961781A80002814BF02250025BF
:101BE00001B10135444F57F8257000257A5DFF2A71
:101BF00002F00F0002F0F00309D122893F4840496A
:101C0000B2F5FA7F016071D93E4B03606EE0A178B6
:101C100011B1811E012965D9E17811B1011F032994
:101C200060D9E17909B181425CD012F0300F03D064
:101C30002278002A08BF0023217931B1A27922B984
:101C4000A0F10801012998BF802362792AB1A17906
:101C500019B9021F032A98BF802303F01001CAB2EA
:101C60003AB100222849FFF74DFF284B08221A708D
:101C700038E003F02001CAB242B1244E2449327840
:101C8000FFF740FF3078411C31702BE003F040013A
:101C9000CAB292B123891F4AB3F5FA7F94BF0121DA
:101CA00008214A431C4EB2FBF3F39AB2A38996F87B
:101CB0000080FFF72FFE194B0EE01B0612D563893B
:101CC0001449174E91FBF3F292B2E389012196F881
:101CD0000080FFF71FFE134B43F8280008F10108AE
:101CE00086F8008001350E2D80D186E70020BDE802
:101CF000F08100BF0800002094E80008BC06002026
:101D000005190008E1180008491A0008B406002067
:101D1000691B000840420F00B5060020C0060020E5
:101D2000B9060020F006002008B5044B1A7882425C
:101D300002D9034B1A68904708BD00BFB5060020C2
:101D4000BC060020044B1A78824204D9034B53F896
:101D50002000026811807047B9060020F0060020BC
:101D6000014B33F810007047C20500207047017125
:101D70007047426A806A131A594251EB0300704758
:101D8000037913F001010BD0026AC3699A4205D0AE
:101D90009CBFC0681218D01AC0B2704700207047AC
:101DA00008467047037910B513F0010104460ED0C0
:101DB000FFF7E6FF60B1E3696269E168D05C4A1E43
:101DC000934201D2013300E00023E36110BD0846D5
:101DD00010BD03799A070AD5436A8269D154416AD2
:101DE00003694A1CB2FBF3F103FB11224262704704
:101DF00090F842321BB1D1F1010138BF0021D0F877
:101E000034014268836809B11361704753617047B8
:101E100007B5034699684822ADF8041002234068CC
:101E200001A98DF806208DF8073003F06BF80EBD80
:101E300058B50E4B044618680E460346B3FBF2F144
:101E4000B1F5803F03D3012BF8D95B08F6E7084AC8
:101E500089B2B0FBF2F3DAB2204600F051FA054A3B
:101E600020463146BDE8584000F00ABA5001002033
:101E700040420F00E92100087FB5044601A80D4645
:101E8000164608F0D8FF00200123ADF80A00ADF88F
:101E90000C0001A92046ADF80450ADF80660ADF87D
:101EA000083009F049F87FBD38B504460D46002AD0
:101EB0000CBF02220022217B0068FFF7DDFF034AEE
:101EC00020462946BDE8384000F0DAB97D200008F8
:101ED00007B5034699681022ADF804100223406844
:101EE00001A98DF806208DF8073003F00BF80EBD20
:101EF00000F134034FF48072436100F59C710023BC
:101F0000C2600362C36181610261836243627047A0
:101F10002DE9F0411D46194B0E4603210360017166
:101F2000044690460127FFF7E3FF002084F83C02B7
:101F300084F83902A4F84402A4F8460284F83872FE
:101F4000D4F8340184F84252FFF7C2FF206BFFF748
:101F50005FFF39462046FFF74BFF322003F0BFFA00
:101F6000D4F8340131464246FFF762FF206B314618
:101F70002A46BDE8F041FFF797BF00BFB4E800086C
:101F800010B5084A044608480B4602631032C0F8F0
:101F9000342100212246FFF7BBFF044B01201C60C7
:101FA000187110BD0CE900086C110020100700200A
:101FB000034607490748084AC0F8781212681031EA
:101FC000C0F87C1300F512700121FFF7A1BF00BF1C
:101FD0002CE900086C11002010070020C268036A79
:101FE000511E8B4201D3002300E00133036270478E
:101FF00010B590F83C220446AAB9836A416A994216
:1020000025D080692169C05C01338B42A36228BF5F
:10201000A26242000A2342F4007084F83D32A4F820
:102020003E02012311E090F93D3273B1B0F83E1247
:102030004A08A0F83E2201F00101FFF7D9FE94F80A
:102040003D02431E84F83D3210BD84F83C3210BD81
:1020500090F83B3210B583B990F83A3290F83922B3
:1020600093420AD2012101FA03F1B0F84042013350
:102070002143A0F84012DBB2F2E710BD2D4B10B5A2
:102080004FF4127404FB00342079C10751D594F841
:10209000381221B3236B0021186808F01BFF94F855
:1020A0003C1221B1B4F84402421CA4F84422236B30
:1020B00094F842221868197B002A14BF02220022D9
:1020C000FFF7DAFE0020012184F83B1284F8390280
:1020D00084F83A02A4F8400284F8380210BD94F85B
:1020E0003B222046012A04BF94F8392284F83A2280
:1020F000FFF7AEFF94F83B02236B58B9012094F828
:10210000422284F83B021868197B002A14BF02227D
:1021100000220AE0002184F83B1294F84222186859
:10212000197B002A0CBF02220022BDE81040FFF7F5
:10213000A3BE10BD6C11002090F83B1200230122B9
:10214000012980F8393280F838220CD180F83B32EE
:10215000036B90F84222197B1868002A0CBF0222F8
:102160000022FFF789BE704702790346D20713D5D4
:10217000B0F8402202F4007189B209B9D10705D440
:10218000B3F84602421CA3F8462270474169036A2D
:102190005208CA54FFF722BF704710B590F8383282
:1021A0000446002B1ED190F839124A1CD3B2092BD9
:1021B00080F8393203D1BDE81040FFF749BF0A2B40
:1021C00010D190F83B0228B9B4F8401241F0010256
:1021D000A4F840222046FFF7C7FF2046BDE8104084
:1021E000FFF7AABF10BD0000064B10B54FF41274E4
:1021F00004FB00342046FFF7FBFE2046BDE81040FC
:10220000FFF7CBBF6C11002030B500240E4D55F800
:102210002450854202D00134E4B2F7E7A400E4B2CE
:1022200000200A4D2D5C8D4202D0451CE8B2F8E733
:102230000019C0B20F2805D8054C04EB00108360CC
:102240000171027330BD00BFACE90008BCE90008B1
:10225000FC1500200C2912D8DFE801F0071111113C
:10226000091111110B1111110D00022104E00421BB
:1022700002E0082100E01021012208F0FEBD7047B5
:1022800038B504460D461346217B00682A46FFF701
:10229000BBFF2068217BBDE83840FFF7DBBF07B5F7
:1022A0008DF80400012000238DF806008DF807004A
:1022B00001A88DF8053008F0BFFB0EBD7FB50446C0
:1022C00001A80D46164608F0A3FD0B4B0B485E43D4
:1022D00001680023B1FBF6F2013D561E204601A91C
:1022E000ADF80850ADF80460ADF80A30ADF806302E
:1022F00008F046FC7FBD00BF40420F0050010020A7
:1023000010B504460068FFF7D9FF2068012108F0E6
:102310009AFD607BBDE81040FFF7C1BF00230C4A67
:1023200052F82320824202D05A1CD3B2F7E79B0016
:10233000D8B20023074AD25C8A4202D05A1CD3B2D8
:10234000F8E71818044BC1B203EB0110704700BF47
:10235000ACE90008BCE90008FC15002070B5044693
:1023600000262E4BF55C95B90221204608F08DFE23
:1023700001284FD12046022108F092FE294620462E
:10238000FFF7CCFF0546204608F072FE3DE0042D25
:1023900012D12046294608F078FE01283AD120467D
:1023A000294608F07DFE29462046FFF7B7FF05467F
:1023B000204608F060FE28E0082D12D1204629466C
:1023C00008F063FE012825D12046294608F068FE62
:1023D00029462046FFF7A2FF0546204608F04EFE9C
:1023E00013E00C2D16D11021204608F04EFE0128D6
:1023F00010D12046102108F053FE29462046FFF751
:102400008DFF0546204608F03CFEAA6801460AB149
:10241000287B90470136042EA3D170BDBCE900088B
:102420000148FFF79BBF00BF002C01404FF08040E8
:10243000FFF794BF0148FFF791BF00BF00040040C1
:102440000148FFF78BBF00BF000800401D481E4930
:10245000026800608A4200F01F80002100F004B88A
:102460001A4B5B584350043119481A4B42189A4290
:10247000FFF4F6AF184A00F003B8002342F8043B1B
:10248000164B9A42FFF4F9AF08F0B8F80BF0F6F8E3
:1024900000F0BAFFFFF7FEBF114E1248306012483D
:1024A000016821F070610160410201600F4C182049
:1024B00020600F490F4808600F48D0F800D04068EE
:1024C00000470000F04F0020EFBEADDE680F0108AE
:1024D000000000209C0500209C050020741D0020A9
:1024E000181002400900000004000140140C0140D3
:1024F000000C01404434434400F0FF1FFFF7FEBFCF
:10250000014B186802F039BD6C1B00200149002006
:1025100000F046BE0125000810B5FEF7F7FA0A499B
:10252000FEF748FB0949FEF7F9FB094B044618681A
:102530000078FEF7EBFA01462046FEF73BFBFEF77C
:1025400025FD80B210BD00BF3333534000F07F45FE
:102550002C07002038B50D4C00202578FFF712F924
:102560000B4A05F0070322F81300013500232570FC
:102570001846D15A02334018102B80B2F9D1C00846
:10258000FFF7CAFF034A107038BD00BF18070020CC
:102590001A070020FC160020074B084A19781088FB
:1025A000884207D3064B1A68907888428CBF002077
:1025B0000120704700207047FC160020FE16002006
:1025C0002C070020124B70B5186020240025002035
:1025D000FFF7D8F82D180A2002F081FF013CF6D150
:1025E000C5F34F10FFF798FF094902230A68517895
:1025F0004D006619B04203D30133062B0C44F8D1C9
:10260000044892780370534303490B8070BD00BFA8
:102610002C0700200A000020FE1600202DE9F04FB4
:102620000446008885B048B9B4F9023043B9B4F91A
:102630000420D2F1010138BF002102E0002100E0B6
:10264000014611F0010377D13D4D00B22B7000F02F
:10265000D7FC0646B4F9020000F0D2FC0546B4F9F6
:10266000040000F0CDFC0446304609F05FF8074650
:10267000304609F0CFF88046284609F057F806465C
:10268000284609F0C7F80546204609F04FF882466B
:10269000204609F0BFF8394681465046FEF78AFACF
:1026A000394683464846FEF785FA51460190404632
:1026B000FEF780FA494602904046FEF77BFA314623
:1026C00003905046FEF776FA1E4C4946206006F10C
:1026D0000040FEF76FFA29466060A5600298FEF799
:1026E00069FA01460198FEF75DF92946E060039812
:1026F000FEF760FA01465846FEF752F9314620616E
:1027000008F10040FEF756FA294660615846FEF788
:1027100051FA01460398FEF743F92946A061019852
:10272000FEF748FA01460298FEF73CF93946E061A7
:102730003046FEF73FFA206205B0BDE8F08F00BFDB
:102740000B00002030070020013A2DE9F8430C4629
:10275000072A30D8DFE802F004080F14191E2226D9
:1027600001882180428803E043880B80028852421E
:10277000628082881EE00388594221804288F6E701
:102780004388594221800288F2E703885942218018
:1027900041880CE042880A80018808E003880B80A9
:1027A000428803E043885942218002885142618077
:1027B00080884242A28030480278002A5AD1B4F977
:1027C0000000FEF7A3F98046B4F90200FEF79EF977
:1027D0000746B4F90400FEF799F9284D0646296822
:1027E0004046FEF7E7F9E96881463846FEF7E2F928
:1027F00001464846FEF7D6F8A96981463046FEF7FD
:10280000D9F901464846FEF7CDF808F0C3FF6968DC
:1028100020804046FEF7CEF9296981463846FEF70A
:10282000C9F901464846FEF7BDF8E96981463046D8
:10283000FEF7C0F901464846FEF7B4F808F0AAFFD3
:10284000A96860804046FEF7B5F969698046384658
:10285000FEF7B0F901464046FEF7A4F8296A07469C
:102860003046FEF7A7F901463846FEF79BF808F018
:1028700091FFA080BDE8F8830B0000203007002006
:10288000F8B5154C06462378274663B902F016FEC4
:10289000124D2A683232904205D30123237002F090
:1028A0000DFE2860F8BD3878A0B102F007FE0B4C91
:1028B0002168731898420DD307480022027002F075
:1028C000FDFD074920600B780BB15A1E0A700549BF
:1028D00001200870F8BD00BF540700205C070020ED
:1028E000550700205607002037B58DF805101F4901
:1028F0008DF807300B788DF8040002A88DF80620BB
:10290000C21812F8044C0D46443CE0B20A2828D8FC
:102910001749022B31F8104003D814B12046FFF7B5
:10292000AFFF2B78022B0BD9124D2D6802F0C6FD9C
:10293000021B954204D20D490F4B002008701870FD
:102940000E4802780146012A00D074B9074B187866
:10295000022801D8421C1A7000230B7008490B7022
:1029600003E03224022BD9D9DBE73EBD5A07002011
:10297000C0E900085C07002055070020560700202A
:102980005407002070B5374B04465A7B364802B1D5
:10299000012202704FF4007000F032F9F0B13349B7
:1029A0004B78181C18BF012000F0CCFC38B1304D1A
:1029B0000120287000F0D2FC08B102222A7000F039
:1029C000AFFC28B129494B7813B9294A022010706D
:1029D00000F09CFC10B1264B00211970202005F05E
:1029E0009DF860B11F482349827A0AB9C37A23B19E
:1029F0001E48C27A0AB9012300E000230B701C496B
:102A00000878022802D14C204E211DE0012807D170
:102A10004D2153204C220B46BDE87040FFF764BFA8
:102A2000144A1378012B03D1532001464E2206E0AD
:102A30000D490878012804D15320014602464D2350
:102A4000EAE724B153204D210A464423E4E70A4A29
:102A5000137823B13220BDE87040FFF711BF07495A
:102A60000C7070BD001D002057070020EF1C0020D7
:102A70005807002059070020550700205407002060
:102A80000E4B1A783E2A16D15888B0F5667F12D1BF
:102A90001979BE290FD193F896230020EF2A0CD183
:102AA00013F8011B064A48409342F9D1D0F10100C6
:102AB00038BF0020704700207047704700F80108B9
:102AC00098FB010838B5FFF7DBFF10B90A2002F0C8
:102AD00077FD164C164920464FF466720AF018FE30
:102AE00094F89433022B02D9002084F8940394F8CC
:102AF0009413CC2202FB01430E4D03F59871284636
:102B00000AF006FE05F11F0005F0BEF805F11F00F2
:102B1000B4F8D010B4F8D22005F0D0F8287801F03D
:102B200019F9BDE8384003F0E7BF00BFD017002017
:102B300000F80108041700202C4B70B53E22064611
:102B40004FF466701A705880BE25EF2200201D7168
:102B500083F8962383F8970349B193F89413CC2212
:102B600002FB0133224903F598700AF0D1FD0021E0
:102B70000D461E4A885C0131B1F5667F85EA000585
:102B8000F7D182F89753002508F016FB342008F09F
:102B900027FB184808F07AFB042811D1154C164B76
:102BA0002046E15808F048FB042805D0013508F01C
:102BB0000FFB032DE8D103E0104A04349442EED118
:102BC00008F006FB032D02D0FFF75AFF10B90A20C8
:102BD00002F0F6FCFFF776FF36B10F201421012238
:102BE000BDE8704007F0F0BC70BD00BFD0170020FA
:102BF0000417002000F80108D01FFE1798FB0108F9
:102C0000034B996808420CBF00200120704700BFA9
:102C1000D0170020024B9A6810439860704700BF9D
:102C2000D01700202DE9F3470446FFF729FF10B124
:102C3000002C00F06D81B84AB84D10685168B84C4E
:102C40006B4603C34FF46672002128460AF00EFE5D
:102C5000CC22002120460AF009FE3E2003212870E4
:102C600002206971FFF7D6FFFA22A5F8F2202A2385
:102C70006E22A5F8EE304FF4FA7085F804212B236C
:102C800040F24C42A5F8F60085F80531212002F506
:102C90004873202185F80601A5F8163140F27E40E0
:102CA0004FF47A7300274FF001094FF4167685F838
:102CB000F410A5F8142140F2DC5100F52F72A5F8AC
:102CC000D00003F5CB70A5F8F060A5F81211A5F8B7
:102CD000D22085F89473A5F8F870A5F8FA70A5F8D5
:102CE000FC7085F8E27085F8E37085F8E470A5F86B
:102CF000E670A5F8E870A5F8EA7085F8ED7085F83B
:102D0000EC9085F8077185F82A7185F82B7185F8A4
:102D10002C7185F8107185F8187185F8197185F88E
:102D20001A91A5F8D430A5F8D6006C30A5F8D800D3
:102D30004FF4C870322340F2B452A5F8DE004FF4CD
:102D40001650A5F8DA20A5F8DC301A46A5F8E030D0
:102D5000C5F824014FF4E1331E20C5F82031E0729C
:102D600040F6AC5320735520AB81E07017230B2045
:102D70004FF028086375A37560712D2314204FF060
:102D8000080E4FF00E0A63732271A07184F810E0F0
:102D9000A37685F81C7185F81D7185F8287185F872
:102DA000297185F81B71277084F8018084F80280EE
:102DB000E775A7732776E773677684F807A06074D2
:102DC0005020E076E1845A20042120722375E077B8
:102DD000412384F82E105348534984F82030534B34
:102DE0004FF00A0A4FF0640C4FF0780E84F821205F
:102DF00060631522E1634E4805F5847184F8312043
:102E0000A36384F812A084F81CC084F8098084F8B5
:102E10000AE084F81E9084F8237084F8247084F803
:102E2000257084F822706785A785278584F82F8010
:102E300084F8308084F8409004F07EFF4FF44872AC
:102E4000C8204FF4966340F2D9313E4684F86C7046
:102E500084F86D7084F86E8084F86F9084F87270D6
:102E6000A4F8702084F8B4A084F8B500A4F8B630B3
:102E7000A4F8B8104FF4FA601DF807104FF47F72F1
:102E8000A0F5FA730137A4F87420A4F87600A4F82A
:102E9000783084F87A100834082FEBD1204C0122C6
:102EA000C820142384F8BA2084F8BB2084F8BC20FE
:102EB000A4F8BE0084F8C0301E2184F8C2204FF46C
:102EC00096706422282384F8C110A4F8C420A4F8C2
:102ED000C600A4F8C830114C522184F89513002282
:102EE000A31810320020C02A1861F9D1002411491A
:102EF000CC2260180A49CC340AF00AFCB4F5197FD8
:102F0000F5D10020014602B0BDE8F047FFF714BE3E
:102F100002B0BDE8F08700BF64E80008D0170020C9
:102F2000041700209A99193F3D0A773FF6287C3F05
:102F3000D6E9000800190020024B9A6822EA000036
:102F400098607047D0170020014B9868704700BF09
:102F5000D0170020884203DB8242B4BF11460146ED
:102F6000084670470023036170472DE9F041066968
:102F700004460136012E0D46066105D1002361602D
:102F800021608360BDE8F081D0F8008008464146AA
:102F9000FDF706FD07463046FDF7B8FD0146384609
:102FA000FDF7BCFE01464046FDF7FCFC06466060AE
:102FB00031462846FDF7F4FC01463846FDF7FAFD98
:102FC000A168FDF7EFFC2660E060A060BDE8F0813D
:102FD00010B504460069012807DD0138FDF796FDAC
:102FE0000146E068FDF79AFE10BD002010BD08B54F
:102FF000FFF7EEFFBDE8084008F09ABC00000000B3
:1030000008B5FDF701FA04A3D3E90023FDF762FA3E
:10301000FDF772FC08BD00BF399D52A246DF913F0B
:103020002DE9F041069C06460F46002B0CBF4FF0E1
:1030300020084FF03008204610F8013B0BB9154628
:1030400003E0002AFBDD013AF6E7002D04DD3046FF
:103050004146B847013DF8E714F8011B11B130466D
:10306000B847F9E7BDE8F0812DE9F04389B006469D
:103070000F4603921C46039A134613F8011B039351
:10308000002900F08A80252901D0304683E0002005
:1030900004905578911C302D039105D19578033219
:1030A00003924FF0010800E08046A5F13003D8B24A
:1030B000092806D8284603A90A2204AB00F00CF917
:1030C00005466C2D05D10399012211F8015B03918E
:1030D00000E00022642D2FD010D8582D3AD006D809
:1030E000002D5AD0252DC6D13046294653E0632DF8
:1030F000C1D130462178251DB8474AE0752D0DD045
:10310000782D27D0732DB6D1251D24683046009424
:103110003946049A0023FFF783FF3AE0251D206813
:103120000A2122B1002205AB00F060F802E005ABF5
:1031300000F08CF82C4623E005AD04F1040920686A
:10314000294612B100F077F801E000F0A4F84C46EF
:10315000009517E004F104092068102142B1B5F18F
:103160005804634253EB040205AB00F03FF806E05D
:10317000B5F158035A425A4105AB00F067F84C4686
:1031800005A8009030463946049A4346FFF748FFA9
:1031900071E72C466FE7B8476DE709B0BDE8F083EB
:1031A000024B196002490860704700BF60070020A9
:1031B000640700200FB407B5094904AB0868094942
:1031C00053F8042B09680193FFF74EFF064B18686C
:1031D00001F0F2FE0028F9D0BDE80E4004B07047BF
:1031E00064070020600700206C1B0020F0B501245C
:1031F000B0FBF4F58D4201D34C43F9E70026C4B18E
:10320000B0FBF4F504FB1500B4FBF1F41EB9002D7E
:1032100001DC002CF4D1092DEFB204DD002A0CBF33
:103220005725372500E03025ED1903F8015B0136FD
:10323000E5E71C70F0BD00280B4603DA2D22404262
:1032400003F8012B0A210022FFF7D0BFF0B50124BB
:10325000B0FBF4F58D4201D34C43F9E70026C4B12D
:10326000B0FBF4F504FB1500B4FBF1F41EB9002D1E
:1032700001DC002CF4D1092DEFB204DD002A0CBFD3
:103280005725372500E03025ED1903F8015B01369D
:10329000E5E71C70F0BD00280B4603DA2D22404202
:1032A00003F8012B0A210022FFF7D0BFA0F1300361
:1032B000DAB2092A01D818467047A0F16101052940
:1032C00001D857387047A0F14103052B01D8373892
:1032D00070474FF0FF3070472DE9F8430D68044602
:1032E0000F469046994600262046FFF7DFFF00284C
:1032F00006DB404504DC08FB060615F8014BF3E746
:103300003D602046C9F80060BDE8F883034BB3F97F
:103310000000D0F1010038BF002070476A0700208C
:10332000064B0749B3F9000091F8B4300522534326
:103330009842D4BF00200120704700BF6A070020D8
:103340000417002010B50446FFF7EAFF002814BF59
:103350002046002000F0010010BD00000749084B86
:1033600091F8B420B3F9000091F8B530D1180522D6
:1033700051438842D4BF0020012070470417002029
:103380006A07002008B504F0E9FB024B00221A701E
:1033900008BD00BFEF1C002010B54FF40070FFF710
:1033A0002FFC18B3FFF7BCFFE0B1114B5C78201C79
:1033B00018BF0120FFF7C6FF70B10E480E4BB0F8E2
:1033C00012210E49B3F8B6000A804A808A80C8806C
:1033D0000B490A88531C0B80FFF7C0FF00B90CB9DA
:1033E000FFF7D0FF074801884A1C028010BD00BFCC
:1033F000EF1C0020D017002004170020301D0020F3
:10340000680700206A07002010B586B002F072F845
:10341000FFF77CF80020FFF705FCFFF753FB6F4A2E
:1034200092F8073133B1012B01D0092B02D18DF86D
:10343000003004E000208DF8000082F807016846A3
:10344000FEF72AF96648FFF7E9F8022004F070FB5E
:1034500002F07AFD61494C790E2C01D0082C01D183
:10346000012200E000224FF480708DF80A20FFF75F
:10347000C7FB18B90820FFF7C3FB00E0012000F0EC
:10348000010340208DF80630FFF7BAFB8DF80700E6
:103490000120FFF7B5FB8DF805000820FFF7B0FB12
:1034A0005049514A4C7C92F8BC308DF808404B4C46
:1034B00080F001008DF80400B4F8DE10C3F3800042
:1034C000B4F8E0208DF809004FF47A734FF480408F
:1034D000ADF80C10ADF80E20ADF81030FFF790FBF2
:1034E00018B1B4F8DA00ADF81000BDF80C10B1F561
:1034F000FA7F02D90022ADF810203B48B4F812310F
:1035000094F80741B0F8B810012CADF81230ADF8BE
:10351000141004D0092C01D1072400E0002401A8D4
:103520008DF80B40FEF750FB304804F037FB4FF4AA
:103530008070FFF765FB40B10820FFF761FB20B901
:10354000264A92F81D0103F029FB0A24192001F0F4
:10355000C6FF192001F0C3FF631E13F0FF04F5D16D
:1035600001F0DAF802F0C4F80220FFF749FB10B1CD
:103570001F48FFF727F8194CD4F8200106F064FA29
:103580004020FFF73DFB48B1D4F8240194F82811FE
:10359000FEF7F6FC94F82901FEF70AFD4FF40060EF
:1035A000FFF72EFB08B104F06DFE01F06DFF11492D
:1035B00008600A484279052A03D10F4B4FF4C874BA
:1035C0001C800E484FF47A710D4C0E4B0180C822BE
:1035D00001212280597300F0CBFBFCE7D0170020BB
:1035E000B61800206C1B002004170020D8180020FB
:1035F000D4180020E80700200808002072080020E6
:1036000070080020EF1C002008B5034BB3F9D4006C
:1036100002F0BEFDFEE700BFD01700202DE9F04FFD
:10362000794B0024B3F902A0B3F9000087B0BAF1D6
:10363000000FB8BFCAF1000A0028B8BF4042824557
:10364000B8BF82462546A04627460594A146264691
:103650006E49CA7812B90B79002B40D0022E3ED0A9
:103660006B4B6C486849B0F8F620685EE95EDFF89D
:10367000B4B101EB40005142FFF76CFC664A05EB28
:103680000B0335F902C0B3F92A10CCEB00009BF80C
:10369000082000EB010902FB09F09BF81C306421B3
:1036A00090FBF1F005226FF0040159435A43CDF825
:1036B0001090FFF74FFC594BDDF810C0E258584905
:1036C00081460CEB020042F210720493FFF742FCB9
:1036D00004999BF8123060505843001305904B49F1
:1036E000CA781AB10B790BB9022E30D1464F4D482A
:1036F000EF5F5021794306EB000B9BF801204A4B0A
:10370000DFF83C8191FBF2F0E95E54F80820401AA2
:10371000801846494FF47A520493FFF71BFC049B30
:1037200048F80400E95E0029B8BF4942B1F5207F9E
:1037300002DD002048F8040058F804207D239BF89F
:103740000B1092FBF3FE01FB0EFC4FEAAC182F4866
:103750000279A2B1022E12D00AFB07F1CAF5FA7360
:1037600003FB09104FF4FA7190FBF1F20AFB08F029
:10377000DDF814B003FB0B0393FBF1F308E0C3780F
:103780000BB1022E02D143463A4601E0059B4A4660
:103790002549DFF8B0C0695A16F80CB008B20BFB27
:1037A00000FB6FF04F0C9BFBFCFB9344204ACDF8D1
:1037B00004B035F902C0A952CCEB00001D4ADFF875
:1037C00088C0029054F80C10A05840180299039039
:1037D0004018A15844F80C100299A150164A04341C
:1037E000B15C202201FB00F090FBF2F15B1A134A5E
:1037F0009B44013625F802B00235032E7FF428AF32
:1038000007B0BDE8F08F00BFB01B0020EF1C002008
:10381000E0070020D0170020180C0020F00700203F
:10382000F0D8FFFF04170020F40B002080C1FFFF39
:1038300078070020D4070020FE1B0020B81B0020C2
:103840006C070020011C0020980700202DE9F74F8D
:10385000002425462646A246474BDA780AB918794D
:10386000C8B1022E19D0454B45484649B0F8F6205C
:103870006F5EE85E514200EB4700FFF76BFB424A88
:10388000424F35F902A0EB19CAEB0001B3F92A0047
:1038900001EB000A0BE0022E09D13C49394B91F8AB
:1038A0002470B3F904201B3757437B1116E03249CB
:1038B000364ACF7877B9334892F823702B5E1B379E
:1038C0005F4309793B1149B1927C02FB0AF703EB94
:1038D000272303E0137A03FB0AF003112C48DFF8D7
:1038E000C8B0295EBBF800005F1A284B784306EB8E
:1038F000030898F80120DFF8B4907A4398F80B1089
:103900004FEAE21C54F80920C31201FB03202149AD
:1039100044F809004FF40012CDF804C0FFF71AFB79
:103920001D4B4FF6FF72E158E750791ABBF8007053
:1039300044F809003B09B2FBF3F74F43174A184B11
:1039400054F80290E158BF11A750494498F8152047
:10395000C9194A43DDF804C012490CEB603044F841
:103960000390013600EB22236B5204340235032E00
:103970007FF472AFBDE8FE8FEF1C0020E00700204F
:10398000D0170020B01B0020180C002004170020C6
:10399000F40B00200000E0FFB4070020C407002063
:1039A00084070020B81B0020E40700206C070020DB
:1039B0000B4B0C481A8852B9817841B142786AB9E8
:1039C000012141700848094B02881A8070474378EA
:1039D00023B90220FF21012206F0F6BD704700BF87
:1039E00072080020EF1C0020581C0020FC1B002047
:1039F0002DE9F04FA94BAA4AB3F90600D18C85B046
:103A000088420FDBB0F5FA6F92F8254007DA451AC5
:103A10006C43A1F5FA6694FBF6F4643403E0C4F158
:103A2000640400E064249F4A9D4BB2F8127192F93D
:103A3000EC2093F823100097574293F86C500191B3
:103A400093F86D60B9B293F824300291002103938A
:103A50000A46924FDDF8008031F907C040F2E637A0
:103A6000C8EB0C0303F2F31EBE4503D8002BB8BF0E
:103A70005B4201E04FF4FA73022ADFF834822CD063
:103A800025B1AB42CCBFC5EB030300236427DFF8AD
:103A90004CA293FBF7FE6FF0630B3AF81E900BFB02
:103AA0000E3B0EF1010E3AF91EA00FFA89FECEEB85
:103AB0000A0E0EFB0BFE9EFBF7FEF14428F8019068
:103AC000DDF8048003FB08FE774B9EFBF3F3DB1964
:103AD0009BB2634393FBF7F712E026B1B342CCBF2E
:103AE000C6EB03030023029F5F43A8F80470039F03
:103AF000002BB8BF5B427B436B4F93FBF7F76437F8
:103B0000674B02EB030E9EF80190642307FB09F854
:103B100098FBF3F9DFF8C88102F808909EF80B9043
:103B20009EF815E007FB09F807FB0EF798FBF3F981
:103B3000DFF8B08197FBF3F302F80890DDF800801E
:103B40005A4FC445D35503DA594BCF5A7F42CF520F
:103B500001320231032A7FF47CAF524C4FF4FA62F7
:103B6000B4F81411FFF7F6F9B4F814614FF47A754C
:103B7000801B4543C6F5FA63B5FBF3F564214D4858
:103B800095FBF1F36FF0630630F8132006FB035545
:103B9000013330F9130013B2C01A4543464B444C6D
:103BA00095FBF1F1587A8A18E280002838D0434F0B
:103BB000434D3E882988721A10B2FFF721FA074652
:103BC00007F0B4FD0646384607F024FE0546B4F972
:103BD0000200FCF79BFF0746B4F90000FCF796FFD4
:103BE00031468046FCF7E6FF294681463846FCF719
:103BF000E1FF01464846FCF7D3FEFDF7A1F9314647
:103C000020803846FCF7D6FF294606464046FCF79A
:103C1000D1FF01463046FCF7C5FEFDF791F9608003
:103C20000220FEF7EDFF90B1264806220378591CCA
:103C3000CBB20370B3FBF2F002FB103111F0FF0FB7
:103C400005D1FEF787FCFEF7A7FC1F4B18701E4A34
:103C50001078003018BF0120FEF794FE1B490B8836
:103C60002BB91B4A108838B904F0E8FA04E00220A6
:103C700003F054FF0028F4D01649174A0968136866
:103C8000C81A002832DB0C4B587B68BB987001F5D2
:103C9000F42303F59070106028E000BF301D002071
:103CA00004170020D01700200CFEFFFFFE1B002091
:103CB000B01B0020181D0020EF1C0020581C002005
:103CC000FC1B0020F8070020A607002008080020A1
:103CD00072080020FC070020A8070020541D0020C7
:103CE000011C0020F41B00200121997005F032FF17
:103CF000124A117831B94FF40060FEF781FF08B124
:103D000004F0E6FA202003F009FF78B10C4B1868A4
:103D10000C4B1A68811A002908DB0B4A1178042918
:103D200004D900F5123000F5F8721A60074B996853
:103D300009B10748884705B0BDE8F08FD4100020CE
:103D4000FC07002094070020FA1B0020301C0020F4
:103D5000901B00200128034B14BF034A034A1A603A
:103D6000704700BF0C0000201D3600084D380008C9
:103D700038B50820FEF744FF90B19F4B93F810012F
:103D800003280CD8DFE800F00202050804F004FA6A
:103D900006E004F05FF803E004F012F900E0002010
:103DA0009649974A0B681168591A002902DA0028C7
:103DB00000F0618203F59C449248203492491460DB
:103DC00003F00AFF4FF48040FEF71AFF20B18F4D39
:103DD0002B780BB903F0C2FE874A92F81B11B1B1E0
:103DE0008B4CC81C34F910504FF47A720021A5F5A1
:103DF0007A70FFF7AFF8FCF789FE8649FCF78EFF73
:103E00008549FCF7D7FEFDF7C1F8844B1880FFF712
:103E1000C3FA794AB2F81401B2F8164100221546E5
:103E20007B49AD08535E8342C4BF65F07F05EDB2A8
:103E3000A342B8BF45F040050232082AF0D17848C5
:103E4000784A04780346AC4204D11078F92803D8A4
:103E5000411C00E0002111704FF480401D70FEF7FE
:103E6000CFFE68B1644B6A4DB3F81211B3F8DC2091
:103E7000B5F90640881A844202DD8D18AC420CDB8D
:103E80004FF48040FEF7BCFEF8B9614C5A4BB4F9D0
:103E90000610B3F81421914217DA63496348644C61
:103EA000B1F8423000250560456085602560656099
:103EB0005BB1564A5F4D1078002800F06D822C7877
:103EC000002C00F06982FFF773FD564B1A78142A14
:103ED00040F0D58057484478ECB1534CB4F84220B8
:103EE0002AB94F4D29785F2901D103F037FE4248A6
:103EF00090F81831002B00F0C2804B4CB4F84220EF
:103F0000002A40F0BC80464D29787D2940F0B780DA
:103F100003F024FEB3E0424D2978572918D1464CCE
:103F20004FF47A724FF480702280FEF769FE08B178
:103F300002F090FD042003F0F1FD10B13F490A2585
:103F40000D80082003F0EAFDD8B93D4B188018E039
:103F50000420FEF755FEA0B12B785A2B11D1394819
:103F600002781AB10470384B012009E0374C384B05
:103F7000257885F00101217009B1022000E00320BD
:103F80001870274802785D2A00F00D825B2A00F045
:103F90000C825E2A00F00B822348B0F8422032B92E
:103FA0001F4C25786F2D02D1FFF702FD15E0124955
:103FB0001B4B91F8180118B112B91A787E2AF3D068
:103FC0001C78972C04D1234B4FF4C870188004E060
:103FD000A72C02D1174901258D73114A1478BB2CE7
:103FE00003D1114CA18D8D1C04E0B72C34D10E4CA3
:103FF000A28D951EA5853BE0D0170020FC07002070
:10400000AC070020D8180020161D0020001D00203D
:10401000301D002000007A4400C07F44F81B0020BF
:10402000A4070020C0070020041700206C07002010
:10403000F0070020EF1C002072080020700800200C
:10404000581C00207E07002090070020A5070020B4
:104050005507002008080020BE2C03D18A4D6B8D27
:10406000981C04E0BD2C0AD1874D698D881E688597
:1040700001200146FEF760FD844B002018700420EB
:10408000FEF7BEFD00282CD0814B187888B1814CFA
:10409000627872B1804D8148B5F90610B0F81441CC
:1040A000A14206DD7E4A15781DB97E49322008807E
:1040B0001D707B4B5C7C54B17B4B1D782DB97B4ACA
:1040C000107810B9774C32212180012408E0774D17
:1040D0002A7832B16F48417819B9754B297001249B
:1040E0001C700023734C1A4634F8020F40F213552B
:1040F00001B2A942CCBF0025012505FA03F5A0F2C3
:104100001550B0F5C77F8CBF002001202A435D1CED
:1041100000FA05F0024340F2A4608142D4BF0021BE
:104120000121981C01FA00F103330A430C2B92B2CF
:10413000DAD1002354485A4900EB4300B0F842005A
:1041400002420CBF0020012058540133152BF1D13D
:104150004A7822B1022003F0E1FC28B90DE0FFF714
:10416000DFF80028F6D108E04A4AD37843B952492B
:1041700001200B604B60D07002E046480021C17006
:10418000474A444B917839B118790021D97020B948
:10419000494A0121106050601971414B187810B9DB
:1041A0003C4901220A70202003F0B8FC002852D0BC
:1041B000384BD87A1A46002848D040490878042855
:1041C00044D93748817A79B1DA79002A43D13C4819
:1041D0000121D9711A723B4B011D1A7002F036FD94
:1041E000394A0220107036E0C27AD9711AB32648D3
:1041F0003649B0F8C820B1F900000028B8BF4042E5
:10420000904218DAB1F902100029B8BF4942914230
:1042100011DA187AF8B901241C722A4B2C4918704B
:104220002C480A684B68011D0260436002F00EFDD5
:10423000254804700FE02348164B017800221A72BB
:1042400049B90122027002F029FC04E00023D37175
:1042500013721D4A137012490E4B087B00B10120E6
:104260000E4A98725179082901D00E2951D1094B73
:10427000002058724DE018480368042B49D8DFE845
:1042800003F02D2F3235410004170020C007002015
:10429000A5070020EF1C0020301D0020D0170020B3
:1042A000001D0020B0070020EC0700207E07002042
:1042B00090070020361D0020F0070020FA1B002088
:1042C000C01B002010000020B2070020B01B0020FF
:1042D000DC1B0020A01B00208007002001220260C0
:1042E00001684B1C03600268511C01603848036878
:1042F0005A1C02604FF48070FEF782FC10B102F08D
:104300003FFD06E03248002101604FF40050FEF707
:1043100077FC01F0B9F82F4A2F4910608A892F4B9A
:104320001AB11968411A002951DB8018186001F090
:10433000F3FBFFF75DFB01F0A7F8294B254A19684D
:1043400010601860421A2748274990F872300A8096
:1043500053B12649CA780AB9087928B1244B2549AE
:10436000DA8808888118D980202003F0D7FB40B173
:104370001E4BD87908B91A7A1AB1197B09B103F022
:1043800047FB1D4B1868804701F014FF01F08CFEBD
:10439000BDE8384001F0E8BE697800293FF495ADEA
:1043A00003F0DCFB91E5012402E0022400E0032499
:1043B000E5B2094B0020691E83F894130146FEF70D
:1043C000BBFB022028212A4606F0FEF8E4E538BDB2
:1043D00080070020FC070020D0170020D007002015
:1043E000E807002004170020E4070020EF1C00204D
:1043F000B01B0020340C00200C000020F8B5614BED
:10440000188800283BD000231A46B0F5C87F5E49C3
:1044100001D100248C505D4C8E581F5F5A4DF61907
:104420008E50002119535A4C04321E190233062BA8
:10443000A6F8F810E9D101281DD12A684FF4C873F5
:1044400002F1C80292FBF3F2A4F8F8206A68C832BD
:1044500092FBF3F2A4F8FA20AA68C83292FBF3F3B5
:104460004C4A12889B1A4C4AA4F8FC30518591851D
:104470000146FEF761FB434801884B1E0380042080
:10448000FEF7BEFB00286BD0444A1288322A11D1B5
:104490003F4C434DB4F8F860B4F8FA00B4F8FC109F
:1044A0002E806880A9803C4D3E4B6C8DAE8D1C806B
:1044B0005E8001E0002A32D000231946322A3A48B1
:1044C00001D100254550314D44585E5FA619465034
:1044D0002F4800245C531D1802330431062B264656
:1044E000A5F8F840EAD1012A16D1304B30491A70AC
:1044F000304B0C7002211970294B1988A0F8F81064
:1045000059889B88A0F8FA102649A0F8FC30224B65
:104510000888498858859985204B013A1A80264891
:104520000178E9B1002303701F48194A0468322159
:1045300094FBF1F4A2F8F8404468806894FBF1F42D
:1045400090FBF1F11348A2F8FA400088091AA2F88A
:10455000FC100120104A014653859385FEF7ECFAC2
:104560000A4B0B4A1888B2F8F810401A1880B2F8B3
:10457000FA105888B2F8FC20401A99885880881A96
:104580009880F8BD080800201C080020781C002036
:10459000D01700201200002004170020B0070020D0
:1045A000020800200A080020100800207E070020D2
:1045B000EC070020550700209007002008B5044BA9
:1045C000044859688847BDE80840FFF717BF00BF97
:1045D0001C1C0020781C00202DE9F84F414B188846
:1045E00000286ED00024254626463E490A88B2F5AA
:1045F0007A7F08D13C4B3D4900271420EF5000FB47
:104600000610FEF7AFFCDFF8F0A0374F3AF90400D0
:10461000EA59DFF8D8901318EB51FCF777FA4FF00E
:10462000140B0BFB069B01464FF000085846FEF7A3
:104630009CFC24F80A80DFF8ACA02D48BAF80010E2
:1046400024F80080012933D15846FEF7D0FC294ACE
:10465000834692F8F400E0B1FCF758FA0146584658
:10466000FCF764FCA8B14FF47A714846AAF8001030
:10467000FEF778FC09F11400FEF774FC09F128003C
:10468000FEF770FCC7F80880C7F80480C7F8008000
:104690000EE0154B4FF47A72E858154B00F5FA719D
:1046A00091FBF2F0E0520F210A20012205F08CFF6D
:1046B000013604350234032E97D10A480288531E6E
:1046C00003800D4B0A4A18881188401A18805188B7
:1046D00058889288401A99885880881A9880BDE82E
:1046E000F88F00BF7208002064080020280800200E
:1046F0000C0C0020D0170020601C002008B5044BD3
:10470000044859688847BDE80840FFF765BF00BF07
:10471000301C0020601C00202DE9F341454C464828
:104720004649B4F8EE20464BFCF79AFE98B9434848
:10473000B4F8EE10FCF77EFF08B100270CE03F480C
:10474000B4F8EE10FCF78AFD07460028F5D10320E7
:1047500000F036FF00E00127364B93F8ED00052806
:1047600028D8DFE800F007071B272703022003F003
:10477000E7F91FE000218DF804104FF4487201A8FA
:104780002D49ADF80620FCF7C3FC10B12D4B0124D8
:104790001C70284890F8ED1001290BD057B1254A1C
:1047A000274B25482549B2F8EE20FCF759FE254B4A
:1047B00002241C70234802784AB91E4C94F8ED106C
:1047C00011B184F8ED20C7E7022003F0B9F9022007
:1047D00003F0A4F9174F20B1174B97F8E3001A68BC
:1047E00090471648046897F8E200A0471649082049
:1047F0000F8D03F093F9154CC0B13FB2642697FBBF
:10480000F6F52846FCF782F906FB1572804610B2D1
:10481000FCF77CF90E49FCF7CDF901464046FCF760
:10482000C1F80C49FCF7C6F9206001E000232360C1
:10483000BDE8FC81D01700201C1C0020301C00208B
:104840007C1B002074080020041700203C0C002072
:104850008988883C000020412DE9F84F9C4C206855
:10486000838A9BB213F0010239D0018821F40063DE
:104870001A04110C0180012106F06EFE954A964B38
:10488000117800201870D9B1944803781BB9944A64
:104890001178FF2914D10123037092480278022A6B
:1048A00006D18B490B68188882B242F400611980E6
:1048B0008D4B874819780068012206F067FE2FE1CA
:1048C0008948834B01780022186806F05FFE844A0D
:1048D0001178FF2900F02481FF207F4BDEE003F0F8
:1048E0000201C9B200293DD0BFF35F8F7D4D2E7804
:1048F000012E354616D177490B789BB177490B7855
:1049000083B1114606F028FEBFF35F8F2068314661
:10491000038B06F015FE754A206816704FF480610F
:104920003246FBE0038BBFF35F8F6E490A78022AA1
:1049300009D1684B1A7832B1684B1A781AB1002144
:1049400006F00AFEE5E00978032907D1614B1A78E1
:1049500022B162490B78002B40F0DD804FF480617A
:104960000122DBE003F00406F6B2002E71D0594BB1
:10497000DFF878811A78012688F80060574B002A02
:104980004DD01A78002A4AD0564D2F78524D022F1A
:10499000574F29D906F0E0FD206895F80090D7F828
:1049A00000A006F0F0FD4FFA89FB0AF80B0009EBB6
:1049B000060031462870206806F0C2FD206888F89D
:1049C00000603F6895F8008006F0DDFD4FFA88F939
:1049D00007F80900B04420684FF48061324685F83A
:1049E000008006F0C5FD2BE0314606F0A9FD2068E9
:1049F0002E78D7F8008006F0C6FD4FFA86F9731CB2
:104A000008F80900D9B220684FFA81F83F68297088
:104A100006F0B9FD033607F808002E7010E01B7889
:104A2000012113B9334A13782BB106F089FD2A48C6
:104A30000278511C03E006F077FD2848012101703F
:104A4000234A11680B8803F4807082B2002AF9D1DE
:104A500066E003F040010F461F4D09B3244B2F7849
:104A6000D3F8008006F08FFD4FFA87F908F80900A7
:104A7000781CC1B229701B4D4FB22A780337BA4255
:104A800005D120684FF48061324606F071FD124B6B
:104A900028781A7851B2884242D1501C18703FE0F1
:104AA0001B063DD52B785EB2721C27D0124901330C
:104AB0000A682B70915D06F064FD0A4895F90020A4
:104AC000017891422CD120684FF480613A4625E06C
:104AD0008C0800208A08002088080020890800200F
:104AE000790800207A08002091080020780800202A
:104AF0007C0800208008002084080020154A2970C6
:104B0000117806F03EFD1448017811B9134B1A785C
:104B100032B9134800684FF48061002206F028FD86
:104B20000E4A104B117893F900004A1C90420ED1A6
:104B30000D4B0E49187800220A7028B10849086800
:104B40004FF4407106F014FD094B00221A70BDE8C5
:104B5000F88F00BF790800208A0800207A0800201A
:104B60008C08002088080020780800208908002090
:104B700090080020FFF770BEFFF76EBEF0B5484CFE
:104B800089B04FF440651C2307460226204602A93F
:104B9000ADF808508DF80A308DF80B6000F0B2F9CE
:104BA0004048142107608DF80E10204603A9ADF887
:104BB0000C508DF80F6000F0A5F925610825384CE0
:104BC000A268520503D40A2000F07EFCF7E74FF4F8
:104BD00080660A20666100F077FC6F1E0A2026615D
:104BE00000F072FC17F0FF05E9D14FF40067676130
:104BF0000A2000F069FC66610A2000F065FC26616D
:104C00000A2000F061FC022027611C218DF80F00B2
:104C10002046244C4FF440638DF80E1003A9ADF8E4
:104C20000C3000F06FF9206806F0E0FB04A806F0F5
:104C300061FC20682A464FF4407106F099FC1A483E
:104C40004FF480434BF6FF72049001212068ADF8C9
:104C50001C30ADF81620ADF8145006F059FC04A92C
:104C6000206806F0DDFB4FF4A06005F0DBFE22219A
:104C7000012201A88DF804108DF805508DF806501A
:104C80008DF8072005F0D8FE212301A82E468DF8C7
:104C900004308DF8055005F0CFFE09B0F0BD00BF1F
:104CA000000C01408C080020801A060010B540005E
:104CB000244CC0B220702448244C01700021217083
:104CC000234C01202070234C2360234C2360234B72
:104CD0001A70234A1070234801702349086883889A
:104CE00003F4007291B2A1B9038803F4807291B207
:104CF00041B9038803F4007291B20029F9D101216E
:104D000006F012FC18484FF440710068012206F0CA
:104D10002FFC47F23053124A117811B1013BFAD1FE
:104D200000E053B911490A88501C83B20B800E4928
:104D30000868FFF723FF002010BD0A4B187880F0A9
:104D4000010010BD91080020790800208008002093
:104D50008A0800207C080020840800207A080020AF
:104D600090080020810800208C0800207608002090
:104D700010B54000244CC0B220702448244C01706F
:104D800024490120087000212170234C2360234C0A
:104D90002360234B1A70234A107023480170234963
:104DA0000868838803F4007291B2A1B9038803F400
:104DB000807291B241B9038803F4007291B2002964
:104DC000F9D1012106F0B0FB18484FF4407100689A
:104DD000012206F0CDFB47F23053124A117811B18F
:104DE000013BFAD100E053B911490A88501C83B243
:104DF0000B800E490868FFF7C1FE002010BD0A4B6A
:104E0000187880F0010010BD91080020790800207A
:104E10008A08002080080020840800207C080020E8
:104E20007A08002090080020810800208C080020CB
:104E30007608002007B502AB03F8012D0122FFF729
:104E400097FF0EBD274B37B51868818A8AB2019249
:104E5000019B13F4706F02D0234A01211170019B52
:104E600013F4E06F31D04FF480610022038B06F021
:104E70007FFB0198810528D41A4D2868018801F428
:104E8000007293B20BBB048804F480718CB29CB1A5
:104E9000028802F4807399B20029F9D1012106F049
:104EA0004FFB10480068028802F4007399B2002991
:104EB000F9D1FFF763FE08E0012106F041FB286805
:104EC0004FF44071224606F053FB06480268938A6D
:104ED00023F470610804030C0449938200220A70D1
:104EE0003EBD00BF8C0800208108002090080020F3
:104EF000FFF7A8BFFFF7A6BF014B188880B2704725
:104F0000760800202DE9F0410F88002347FA03F2CC
:104F1000D2072DD58A7803F00705DC08AD0012F022
:104F2000100F18BF91F803C002F00F0618BF46EA31
:104F30000C064FF00F0C0CFA05FC06FA05F550F8BC
:104F40002480282A28EA0C0C45EA0C0540F8245055
:104F500006D1012202FA03F2C46824EA020206E042
:104F6000482A05D1012202FA03F2C4682243C26032
:104F70000133102BCAD1BDE8F08108B503681A6867
:104F8000904708BD38B505460C4614F8011B19B109
:104F90002846FFF7F2FFF8E738BD08B503685968FF
:104FA000884708BD08B503689968884708BD08B5F3
:104FB0000368DA68904708BD08B50368196988472F
:104FC00008BD08B503685A69904708BD7047036B70
:104FD00013B15A68006C01E0026AC069101A18BF68
:104FE00001207047436B13B190F844007047826A08
:104FF000406A111A4B4253EB01007047836A816982
:10500000426BC918D160416A994203D9CB1A5360E7
:10501000816204E00169CB1A5360002282620021A0
:1050200080F84410406B012106F05DBB30B50446AA
:10503000007985B000230D460091C107ADF804301A
:10504000ADF80630ADF80830ADF80C30ADF80A30E8
:1050500002D50422ADF80A20820705D5BDF80A1052
:1050600041F00803ADF80A30A06C694606F01CF860
:10507000A56005B030BD026B034610B5406942B172
:105080001A6CD9688C1A013A18BF1146005D196470
:1050900010BD196ADA68405C0131B1FBF2F402FB21
:1050A0001411196210BD10B5426A8469A154416A95
:1050B00002690131B1FBF2F402FB1411426B41624F
:1050C00032B11368DB070BD4BDE81040FFF796BF81
:1050D000806C40F227710122BDE8104006F048B80C
:1050E00010BD0000214B13B5986021480C46586153
:1050F0002048214A2149186314381A6099614FF4F5
:105100008072586301214FF48040DA601A6106F022
:1051100035F94FF4007102231822ADF80010A107F1
:105120008DF803308DF8022003D515486946FFF746
:10513000E9FE48234FF48060E207ADF800008DF8E7
:10514000023003D50E486946FFF7DCFE01220E212E
:1051500001A88DF804108DF805208DF806208DF833
:10516000072005F069FC01481CBD00BF540B00205E
:10517000520A002058000240E0E90008D20800204E
:10518000000801401F4B13B51F4A98600C46802051
:105190004021D86019611D481D491A601D4A986157
:1051A00099644FF4003001215A6106F0F3F80223AC
:1051B000042218208DF80330A307ADF800208DF8E5
:1051C000020003D514486946FFF79CFE08214823D6
:1051D000E007ADF800108DF8023003D50E4869469F
:1051E000FFF790FE012026228DF8050002218DF8A0
:1051F000070001A88DF804208DF8061005F01CFCAE
:1052000000481CBDA00B0020E0E900089208002027
:1052100000440040D2090020000801402DE9F0417F
:105220001E46584B90B0984205468846174604D112
:1052300010463146FFF756FF07E0534800248542E9
:1052400004D110463146FFF79DFF0446002106F0C9
:1052500004022671A7600197A5642162E161A16241
:105260006162C4F82C80ADF8081002F0FF0732B17B
:105270004FF40053ADF80A304FF4806701E0ADF809
:105280000A700020ADF80C7016F00107ADF81000A0
:1052900002D1ADF80E7002E00421ADF80E1006F058
:1052A000020606F0FF082EB1BDF80E2042F00803FA
:1052B000ADF80E30284601A905F0F6FE012128467A
:1052C00005F04AFF05A806F001FA0023281D4FF457
:1052D0008051802205900E910F9309930B930A92AF
:1052E0000C9317B3206BD0B16269E1680793202358
:1052F0000D930692089106F051F9206B05A906F06E
:10530000C5F9206B012106F0EEF928464021012263
:1053100005F048FF206B06F0FBF9206405E0284605
:1053200040F22551012205F023FFB8F1000F24D0EF
:10533000606BE0B1266910210896002607910D9652
:1053400006F02CF9606B05A906F0A0F90122606B4C
:10535000022106F0D3F9606B314606F0D7F9606B95
:10536000802146600122284605F01CFF05E0284602
:1053700040F22771012205F0FBFE204610B0BDE887
:10538000F08100BF003801400044004010B50B4CD4
:105390004FF4005006F0C0F90021606B06F0A3F94D
:1053A000626AA36A9A4204D02046BDE81040FFF723
:1053B00025BE012084F8440010BD00BF540B00201E
:1053C0000D4B986C028802F080018AB29AB19A6AF9
:1053D000596A8A420AD09969895C013281801969C7
:1053E000B2FBF1F001FB10229A62704740F2277184
:1053F000002205F0BDBE7047540B00201C4B10B5B9
:105400009A6C1488A4B204F0200188B290B1D96AD1
:1054100019B1938898B288470CE09288D969586985
:10542000D2B24254D869DA68411CB1FBF2F002FBF7
:105430001011D96104F08004A4B2C4B10C4B9A6A73
:10544000586A82420BD09869996C805C01328880DE
:105450001969B2FBF1F001FB10229A6210BD986C41
:1054600040F227710022BDE8104005F081BE10BD5A
:10547000A00B002070470000024B1A68501C1860F7
:10548000704700BFEC0B002010B5094A09491368AA
:105490008C6810688342F8D1074A106811684FF48D
:1054A0007A725043001BB0FBF1F102FB031010BDF8
:1054B000EC0B002010E000E0F00B0020014B18681E
:1054C000704700BFEC0B002038B50446FFF7DCFF47
:1054D0000546FFF7D9FF401BA042FAD338BD10B5EF
:1054E00004462CB14FF47A70FFF7EEFF013CF8E769
:1054F00010BD000010B586B005F0E0F80121254888
:1055000005F048FF012144F61D2005F037FF01207A
:10551000014605F027FF002405F060FF4FF6FF73FA
:1055200069461D48ADF800308DF80240FFF7EAFCEF
:1055300069461A48FFF7E6FC69461948FFF7E2FC9E
:105540001848426842F000714160FFF793FF01A8DC
:1055500005F0BAFE019B1448144AB3FBF0F114485D
:10556000116001684FF47A73B1FBF3F2114B501ED6
:10557000114A5860F021072082F823109C601860BF
:105580000E48FFF7FBFAFCF72FF96420FFF7A7FF9F
:1055900006B010BD0700400000080140000C0140AB
:1055A000001001400000014040420F00F00B0020BD
:1055B0005001002010E000E000ED00E00058004045
:1055C00010B540F2DB146043841E2046FFF787FFCE
:1055D0001920FFF784FFF8E710B1034A034B1A6064
:1055E00003480449C8607047EFBEADDEF04F0020AD
:1055F0000400FA0500ED00E02DE9F84F384E0446AE
:105600003768384606F092F80546384606F002F943
:1056100076688046304606F089F88346304606F0C4
:10562000F9F8D4F80490064629464846FBF7C2FA32
:10563000A768824641463846FBF7BCFA0146504609
:10564000FBF7AEF9216882465846FBF7B3FA4146AC
:1056500004464846FBF7AEFA3146FBF7ABFA014683
:105660002046FBF79FF9314604463846FBF7A2FA7D
:105670002946FBF79FFA01462046FBF793F90146BE
:10568000504606F053F91749FBF794FAFAF7CEFEA5
:1056900011A3D3E90023FBF747F8134B044618681E
:1056A0000D46FAF7C3FE02460B4620462946FAF796
:1056B0005FFD00220D4BFBF737F8FBF71DF906F0F5
:1056C00069F881B20A0444BF00F5B47189B208B226
:1056D000BDE8F88FAFF30080182D4454FB2109403A
:1056E000FC0B00200000E1443C0C002000002440A2
:1056F000174B10B51888FBF709FA16490446FBF753
:1057000059FAFBF71DFC1449088021461348FBF7A2
:1057100005FB1349FBF702FB124A10601248B0F870
:105720007000FBF7F3F901461048FBF7F7FAFAF7B8
:105730007DFE05A3D3E90023FAF7CCFEFBF7DCF8E6
:105740000B4B186010BD00BF3B597E90A9E781400C
:1057500012000020C903683F280C00200AE81C4101
:1057600000401C46741C0020041700200000614407
:10577000901C0020AFF300802DE9F0410446006842
:105780000D460146FBF716FAD4F80480064641465A
:105790004046FBF70FFA01463046FBF703F9A768CE
:1057A000064639463846FBF705FA01463046FBF710
:1057B000F9F806F0BDF800210646FBF78FFB70B93B
:1057C00020683146FBF7AAFA314628606068FBF78B
:1057D000A5FA31466860A068FBF7A0FAA860BDE8AA
:1057E000F0812DE9F04F0C68836889B0D0F800A0F3
:1057F000D0F804800646204603938B4605F096FFBA
:105800000746204606F006F8DBF8044081462046AD
:1058100005F08CFF0546204605F0FCFFDBF808206C
:1058200004461046019205F081FF8346019805F079
:10583000F1FF394602905846FBF7BCF9394604900F
:105840000298FBF7B7F9594605904846FBF7B2F9BD
:10585000029906904846FBF7ADF92946079058464D
:10586000FBF7A8F901465046FBF7A4F92146834609
:105870000698FBF79FF901460598FBF793F8014658
:105880004046FBF797F901465846FBF78BF821464F
:1058900083460498FBF78EF901460798FBF780F8DA
:1058A00001460398FBF786F901465846FBF77AF85C
:1058B0003060029905F10040FBF77CF90146504643
:1058C000FBF778F9214683460798FBF773F9014601
:1058D0000498FBF765F801464046FBF76BF9014673
:1058E0005846FBF75FF8214683460598FBF762F9B7
:1058F00001460698FBF756F801460398FBF75AF95C
:1059000001465846FBF74EF8214670605046FBF7BB
:1059100051F92946044609F10040FBF74BF90146CD
:105920004046FBF747F901462046FBF73BF839466E
:1059300004462846FBF73EF901460398FBF73AF97F
:1059400001462046FBF72EF8B06009B0BDE8F08FA5
:105950001FB50B684A6889680193039101A90292F7
:10596000FFF73FFF05B000BD80EAE073A3EBE073F3
:105970008B4206DB002801DD401A704702D0401838
:105980007047002070470000F0B5574B87B01A6889
:105990005B6802F1004203F100430193534B05465B
:1059A000B3F900000092FBF7B1F800F10040FAF7FC
:1059B0003DFD4BA3D3E90023FAF78CFDFAF79CFFDA
:1059C0004B4C0290B4F90000FBF7A0F80390B4F937
:1059D0000200FBF79BF80490B4F90400FBF796F87B
:1059E0006946059003A8FFF7FCFE424B93F8403050
:1059F000012B16D14048417869B9404C40262268B5
:105A000092FBF6F7D01BFBF781F80599FAF7CAFF6E
:105A1000FBF796FA2060394B4021186890FBF1F0B3
:105A200001E0374B1888FBF771F801460598FAF743
:105A3000B7FF05902846FBF765F832490746FAF7A5
:105A4000B1FF01463846FBF769F92F4E0746346827
:105A500005982146FAF7A4FF01463846FBF7AAF855
:105A600001462046FAF79EFF224C306005F092FE78
:105A700094F82F10FFF778FFFBF748F8059003988C
:105A800005F088FE94F83010FFF76EFFFBF73EF844
:105A90000390049805F07EFE94F83010FFF764FF41
:105AA000FBF734F804901948194B01681A684C1C2C
:105AB0000460184CAD1803981D60256805F06AFE57
:105AC0002B1804986568236005F064FE2A18059871
:105AD000A568626005F05EFE2818A06007B0F0BD02
:105AE000399D52A246DF913FFC0B0020581C00203C
:105AF000881C002004170020EF1C0020380C002018
:105B0000120000203661823C040C0020300C002082
:105B1000140C0020681C00202DE9F04F87B0FEF720
:105B2000EDFD022001F0FAFF002800F0A781FEF74A
:105B300045FDFFF7A9FCAA4C05462768C71B384658
:105B4000FAF7E0FFA749C968FBF734F88346A6488F
:105B5000256090F82E8000252C462E46A34A105F23
:105B6000FAF7D4FF5946FBF725F803AB5851B8F1C3
:105B7000000F27D04046FAF7C9FF01464FF07E508C
:105B8000FBF7CCF8DFF8A492824651464FF07E50E6
:105B9000FAF706FF55F80910FBF70CF8944903468D
:105BA000085F0193FAF7B2FF5146FBF703F801468D
:105BB0000198FAF7F7FE49F80500FBF7C1F98D4A9D
:105BC000105303E08A498B4A605AA052894B04352E
:105BD000E15E0234062C01FB0166BFD1864A6420D7
:105BE000138846435B43854803A996FBF3F6FFF70A
:105BF000AFFE082001F092FF20B1814803A9FFF712
:105C0000A7FE07E07F4803A9FFF7A2FE7D480146F3
:105C1000FFF7B2FD493EB1B23B2904D9082001F09B
:105C20007DFF48BB50E0784CB4F8F000FAF76AFF0B
:105C30004FF07E518046FAF7B5FE01464FF07E5098
:105C4000FBF76CF8002406466C4D404655F81410DE
:105C5000FAF7B0FF81466748005FFAF757FF014641
:105C60004846FAF79FFE3146FAF7A4FF45F81400BC
:105C70000234062CE8D1D1E7634A0024B2F8F200DE
:105C8000FAF740FF4FF07E518046FAF78BFE01464F
:105C90004FF07E50FBF742F80646594D404655F806
:105CA0001410FAF787FF594B8146185FFAF72EFF59
:105CB00001464846FAF776FE3146FAF77BFF45F88B
:105CC00014000234062CE8D151494C4DB1F90000C2
:105CD000FAF71CFFAE6801463046FBF727F94D4B3B
:105CE00010B10120587300E058733146686805F020
:105CF0001DFE494C2A682060686802F10046014692
:105D0000FAF758FFD5F80880054641464046FAF7AD
:105D100051FF01462846FAF745FE05F009FE014607
:105D2000304605F003FE60602068FAF77FFB2AA387
:105D3000D3E90023FAF7CEFBFAF7DEFD05F02AFDE2
:105D4000364D28806068FAF771FB23A3D3E900235E
:105D5000FAF7C0FBFAF7D0FD05F01CFD68800820BB
:105D600001F0DCFE2E4C08B1254800E02548FFF785
:105D700043FC1D4D20803846FFF706FE95F8721053
:105D800000297FD01D4E306877680146FAF712FF70
:105D9000B468394606463846FAF70CFF01463046E5
:105DA000FAF700FE214606462046FAF703FF0146B1
:105DB0003046FAF7F7FD05F0BBFD01462046FAF73D
:105DC000ADFF18490446FBF79DF888B3164B002039
:105DD000188057E0AFF300803B597E90A9E78140DF
:105DE0002C0C0020301C002004170020601C002018
:105DF000781C0020881C002012000020941C002029
:105E00001C0C002014000020D0170020141C0020BF
:105E1000280C0020EF1C0020FC0B0020180C002098
:105E2000581C00208FC2753C340C0020440C00200C
:105E3000204605F02BFD264B1968FAF7BBFE05F04E
:105E4000A9FCB0F5617FA8BF4FF46170FAF7DCFAE6
:105E50001DA3D3E90023FAF767FCFAF74DFD05F01F
:105E6000D9FC044695F87200FAF750FE2146FAF77D
:105E7000A1FE05F08FFC174B188003E0164B18802D
:105E800058809880154A164B5179012907D015483A
:105E90001A8859889B8802804180838011E01249CA
:105EA000B3F90420B1F9000002EB4000032290FB9B
:105EB000F2F080B20B4A088019885B8890801180CC
:105EC000538007B0BDE8F08FA2EB0FE5DD169640DA
:105ED000901C0020340C0020781C0020D0170020DB
:105EE000601C0020F40B0020500C0020AFF3008059
:105EF000074B03EBC001B1F878301AB2112A04DC69
:105F00000728DCBF034B33F8123018B2704700BFCC
:105F100004170020301D002010B500244FF48040ED
:105F2000FCF76EFE064B10B1B3F8DA0001E0B3F8EF
:105F3000D400044AA0520234182CEFD110BD00BF87
:105F4000D0170020B81C0020F8B53D4D3D4E6B79B0
:105F50003D4C06EBC30041780A1C18BF01222020EB
:105F60006274FCF74DFE324608B1012666746B7907
:105F7000162B1CD10024324E0021A6193069FAF7E5
:105F8000ADFF28B14FF48040FCF73AFE50BB23E050
:105F90002E4B06F110001D190FC885E80F002C4983
:105FA00010340A78531CC02C0B70E4D1EAE7284F58
:105FB00012F8336002EBC3003E704768002FE1D057
:105FC0000024B442DEDA214D21016D187A180FCA7F
:105FD000013485E80F00F4E719481E4B4179082980
:105FE00023D124E01A4E3678012EF5D91A4C00251B
:105FF0001034B542F0DA54F8100C4FF07C51FAF737
:10600000D9FD4FF07C5144F8100C54F8140CFAF7F9
:10601000D1FD4FF07C5144F8140C54F80C0CFAF7F5
:10602000C9FD013544F80C0CE2E70E2901D101222B
:1060300000E000221A74BDE8F840FFF76DBF00BF12
:10604000D0170020C8EB00086C1B0020580C002063
:10605000520C0020EF1C0020600C0020F0B5002343
:10606000461C0E4A002198181033C02B0161F8D14C
:106070000B4F07EBC6035F6807B9F0BD0024084A61
:1060800012F83600844208DA064D21014D197B18BA
:106090000FCB013485E80F00F1E7F0BDD0170020E9
:1060A000C8EB0008E01700202A4B10B5587C0028E8
:1060B0004ED029494A79531E142B3AD8DFE803F011
:1060C0000B3939213D3939193939393939293939B2
:1060D000393939212900214890F8BB1019B1204BDA
:1060E0000020598930E01F4A50780028F7D1014636
:1060F0002AE01B4C0020E188FBF724FE01202189C7
:1061000022E0174C00202189FBF71CFE0120618949
:106110001AE0134C0020E188FBF714FE01202189CE
:10612000FBF710FE02206189FBF70CFE0320A1891A
:106130000AE02020FCF764FD50B1094C00202188C2
:10614000FBF700FE61880120BDE81040FBF7FABDB7
:1061500010BD00BF6C1B0020D017002004170020CA
:1061600020000020EF1C002010B50024064B1878FA
:10617000A04208D90549204631F814100134FBF734
:10618000D3FDE4B2F2E710BD520C0020A01C0020A9
:10619000064B1A780023D9B2914204D2044921F85F
:1061A00013000133F7E7FFF7DFBF00BF520C0020F9
:1061B000A01C00202DE9F84FB24B187803280FD906
:1061C000B149B24CB1F904206FF06305002AB8BFA1
:1061D0005242A91AB4F904006432FCF7BBFEA08055
:1061E000A84A1678012E1DD8A94EAA4C75796A1EA8
:1061F000142A00F2F981DFE812F0C200F701F7017A
:106200008400D500F701F7017101F701F701F701EB
:10621000F701F701F100F701F701F701F701F701C5
:106220005E00C7019B48994B90F9BA90964FB3F91D
:106230000440C9F10001B7F806A004FB01F95F882A
:10624000B3F80080944C00251034B542CCD20FFA3C
:106250008AF0FAF75BFC54F8101CFAF7ABFC8346A3
:1062600038B2FAF753FC54F8081CFAF7A3FC0146BD
:106270005846FAF797FB83460FFA88F0FAF746FC80
:1062800054F80C1CFAF796FC01465846FAF78AFBBC
:1062900083464846FAF73AFC54F8041CFAF78AFC9D
:1062A00001465846FAF77EFBFAF74AFE7B4B23F885
:1062B00015000135C8E794F89A20744D12F0010FCB
:1062C0006B880CBF01264FF0FF365E43744CB7B2AB
:1062D00004202781FFF70CFE29886E4D381895F8A9
:1062E000A230208113F0010F0CBF01224FF0FF32CA
:1062F0004A43052096B26681FFF7FAFD3718678199
:1063000072E194F89A50614805F002084FFA88F655
:10631000002E0CBF01214FF0FF3115F0010F458811
:106320000CBF01224FF0FF326A438688042001FB34
:1063300006F497B2FFF7DCFD1FFA84F808EB0003C0
:106340005448F91890F8A270554C07F0020253B265
:106350002181002B0CBF01214FF0FF314E4317F07C
:10636000010F0CBF01204FF0FF3045430520FFF720
:10637000BFFDB6B2ADB23718EA19628134E14349C4
:1063800094F8A2408E8814F0010F0CBF01234FF047
:10639000FF3305205E43FFF7ABFDB5B2404F281831
:1063A000788121E10020FFF7A3FD3E4F94F97A3078
:1063B000B7F902603A4D7343322693FBF6F1401869
:1063C00028800120FFF794FDB7F9002094F982405E
:1063D000544394FBF6F3C7186F8005E1324C6078A4
:1063E00020B9B6F8D4202E4BDA810AE02649B6F857
:1063F000D220B1F90600B6F8D010FCF7ABFD284D5D
:10640000E881274E254CF7892780214F97F81901FD
:1064100030B3204D0220FFF76BFDB5F98410B5F9BC
:106420008620FCF797FD214BB7F812111A880C1A39
:1064300016B220B2864203DA97F81961B41803E065
:1064400003DD97F81971D41B1C8095F98A50B3F9B4
:10645000003064226B43124F93FBF2F00918B980AD
:10646000114C0F4DA67A56B1074B1A880324EA80C7
:106470002A81988868815988A981094D18E0034BC1
:10648000F3E700BF520C0020B01B0020B81B002017
:10649000D017002004170020580C0020A01C00205A
:1064A00020000020180C0020EF1C0020540C0020BD
:1064B000AA4FB5F9062007EBC40696F97A30642096
:1064C0005A4392FBF0F7EF802046FFF711FD0134AD
:1064D0003918E9800235072CEAD185E0A04B5A78BB
:1064E00022B9B6F8D4709F49CF810AE09E48B6F829
:1064F000D010B6F8D220B0F90600FCF72BFD994E6B
:10650000F081964E974B964A96F89270974DDC899B
:10651000907A17F0010F2C800CBF01254FF0FF354A
:1065200008B1914900E09249488807F002044543C8
:1065300096F89A60098862B2002A0CBF01274FF0D2
:10654000FF3716F0010F0CBF01244FF0FF3407FB9B
:106550000155604306F0020257B2DD80002F0CBFE8
:1065600001254FF0FF3505FB010018810320FFF7DF
:10657000BFFC7C4EF388C1180420F180FFF7B8FC03
:106580003489021932812FE0794F0324BF88734B7D
:1065900003EBC40090F87A60C4F1060306F0020130
:1065A0004DB2002D0CBF01224FF0FF327A437049EB
:1065B000580831F8105016F0010F0CBF01264FF0AB
:1065C000FF3606FB0522674D96B225F8146020467B
:1065D000FFF78EFC331825F814300134072CD6D180
:1065E000614F6249F88808802020FCF709FB0028E9
:1065F00041D00020FFF77CFC5A4C0546208001204A
:10660000FFF776FC5B4A6080137AA3B3534F5A4A74
:1066100097F8BC1001F00206F3B2CBB1B2F900302A
:1066200097F9821097F97A70B2F9022059437B42A8
:106630005343322691FBF6F16FF0310789B293FB99
:10664000F7F28F187D1993FBF6F625808E1910E06E
:1066500097F97A10B2F9026097F982704E43B2F955
:1066600000203221574396FBF1F3ED18258097FB6C
:10667000F1F680196080414C384D04F11006B4F9F0
:106680000200B5F97410B5F97620FCF763FC24F824
:10669000020F0835B442F2D1304991F8BC3003F012
:1066A0000402D7B22FB93148354B07881C78012234
:1066B0001CE0344D68790E280AD0082808D0324CE6
:1066C00004EBC0014B78002B14BF0225002500E02D
:1066D000042500242D4F621907EB4401D0B209892B
:1066E0000134FBF72FFB042CF4D1DCE7A24209D2E2
:1066F0001E483FB230F912100132B942A8BF0F460E
:10670000BFB2F3E70024A0461D4A1178884567D23E
:106710001C4D3BB2B5F8D200834204DD134DC21BC1
:10672000615B501860534FF48040FCF769FA0F4DDD
:1067300070B3164B40F2DC51B3F90620114B8A427C
:10674000285FC7BFB3F8D810B3F8D220B3F8D4107D
:10675000B3F8D620FCF7FEFB285336E004170020E0
:10676000EF1C002020000020B01B0020A01C0020F7
:10677000B81B0020001D0020180C00201E00002067
:10678000520C0020D0170020C8EB0008301D00205C
:10679000144E285FB6F8D010B6F8D220FCF7DAFB1A
:1067A000114BB6F81411B3F9062005EB04098A421F
:1067B00028530ADA1020FCF723FA10B9B6F8D000F3
:1067C00001E0B6F8D400A9F80000084A507818B9DA
:1067D0000749084B625AE25208F10108023493E774
:1067E000BDE8F88FD0170020301D0020EF1C0020DE
:1067F000B81C0020A01C002044F25063984203DD26
:10680000A0F50C40A038704703498842BCBF00F592
:106810000C40A030704700BFB0B9FFFF10B5FAF7C9
:1068200075F900210446FAF781FB08B1204601E022
:1068300004F100400549FAF771FA0549FAF7BAF987
:1068400004F074FF034B186010BD00BF8096184B16
:1068500035FA8E3C3000002010B5044C0023207027
:106860002361FEF72BFE606110BD00BFD41C002029
:10687000F8B51D4614460E46FAF748F96968FAF766
:1068800099F93146FAF796F92168FAF78BF8206002
:10689000FAF756FBED68074605F10040FAF750FBA2
:1068A00006462846FAF74CFB314602463846FCF7C6
:1068B00051FBFAF72BF92060FAF742FBF8BD000014
:1068C000F8B5101A0C461F46FAF720F90546381B92
:1068D000FAF71CF9174B079E1968FAF76BF9294666
:1068E00004462846FAF766F9214607462046FAF795
:1068F00061F901463846FAF755F805F019F80E49DE
:10690000FAF758F9FAF742FB06990860214605F1B3
:10691000004005F00BF80949FAF74CF90849FAF775
:1069200041F8FAF70DFB0028BCBF00F50C40A03081
:106930003060F8BD300000202C7D8E3FA00CB345A8
:1069400000A00C4610B50446002003460D49CA5C61
:10695000A2B12E2A04D1013394B1C91800220A55DC
:10696000084A0A21D25C4843A2F13001092901D822
:10697000303880180E2B02D80133E7E710BD002015
:1069800010BD00BF780D0020F8B52D4B93F81C0109
:1069900010B1012850D10AE02A4B2B4A58782B4BD2
:1069A00002EB001149685868FEF701FB41E0274DF2
:1069B0006868FEF701FB00283ED0224C217826466D
:1069C00001291ED1FEF77AFD06466069321A632A54
:1069D00035D92169042912D81B4F686807EB0113C8
:1069E0005968FEF7E4FA607807EB0017B968686841
:1069F000FEF7C8FA22696661511C21611CE0022081
:106A000018E022693AB964780F4B686803EB041107
:106A10004968FEF7CCFA33690A4C8B2B09D80C4A2B
:106A20000A48D15C4068FEF7A8FA21694B1C236133
:106A300002E00320FFF710FF024A00205060F8BD7B
:106A4000D0170020D41C002088F000086C1B002008
:106A5000FAEF000810B50B4CE37A8BB10A480178C5
:106A600004290DD9094A0A4B106851681860596009
:106A7000FFF7D4FE0748084B028801211A802173D2
:106A800010BD00BFEF1C0020FA1B0020DC1B002003
:106A9000C01B0020581C0020DA0D0020002370B518
:106AA0001C460F4800211952142060430D4A0E4E17
:106AB0000E4D995200223250595335180C4E6960D0
:106AC000AA60325035180B4E01346960AA60023357
:106AD0003518022C32506960AA60E2D170BD00BF47
:106AE000941B0020E0070020980D0020981B002038
:106AF000440D0020140E002070B5204C204D60790C
:106B0000FAF700F81F49FAF709F92860E07BF9F76E
:106B1000F9FF1C49FAF702F91B4E6860EE60A07994
:106B2000F9F7F0FF1949FAF7F9F8194D2860207CB8
:106B3000F9F7E8FF1349FAF7F1F86860A07EF9F772
:106B4000E1FF1449FAF7EAF8EE60A860E079F9F796
:106B5000D9FF0E49FAF7E2F80F4D2860607CF9F78B
:106B6000D1FF0849FAF7DAF86860E07EF9F7CAFF62
:106B70000849FAF7D3F8EE60A86070BD041700204A
:106B8000C40D00200000C8420000FA44000020416B
:106B9000F00D002000007A44880D002070B5124CE2
:106BA00005460020FFF758FE6570FEF787FC0F4B87
:106BB000A06093F81C0100266660B0420CBF01245F
:106BC0000324FFF799FF0A49234601EB05156A687C
:106BD00031460848FEF722FB074A50600120BDE815
:106BE0007040FFF739BE00BFD41C0020D017002032
:106BF00088F00008004400406C1B002038B5114BA1
:106C0000187803281BD1104C6068FEF7C6F938B11C
:106C100060682568FEF7C6F901462846FEF7ADF91B
:106C20002068094DFEF7B9F90028ECD095E811006D
:106C3000FEF7B8F901462046FEF79FF9E3E74FF06B
:106C4000FF3038BDD41C00206C1B0020F7B5036852
:106C5000164C174D23600968164E61600068FFF7F7
:106C6000DDFD94E80C0014480196009095E80300BF
:106C7000FFF726FE6B68114A61683668C81A16600D
:106C8000F9F744FF0E4A0F4F1168F9F793FFFAF72F
:106C900057F92968786020680B4A431A0B483B6013
:106CA000B0F8C4100A4B16601980FEBDE00D00203C
:106CB000DC1B0020400E00204C0E0020DC0D0020CC
:106CC00030000020740E0020540E00200417002015
:106CD000700E0020264BF0B51D68024600F1100131
:106CE00016781446AB195B78013203F00403DBB26B
:106CF00063B18A42F4D10020F0BD13B10A2253439C
:106D0000DBB210F8011B30395B18DBB2211A022903
:106D1000F3DC0021844209D911B10A225143C9B2DE
:106D200010F8012B303A8918C9B2F3E72E2E11D191
:106D30000134042000220A2672432678AF197F7896
:106D400007F00407FFB217B1303A92190134013845
:106D5000F1D100E00022074C6420614300FB0211E6
:106D600006240548B1FBF4F200FB0320F0BD00BF90
:106D70006C01002040420F00809698000000000047
:106D80002DE9F04F9A4B91B05868C0B9994C2178D1
:106D90004A1E032A00F20286DFE812F0C605C60585
:106DA000DF05C9056068FEF7FDF89349044691F8D0
:106DB0001C31012B00F0DF8008D3022B06D08C4C55
:106DC0006068FEF7EAF80028ECD1DFE7242C07D151
:106DD0008A4B8B4A8B4C0021197011702170C5E0D1
:106DE0002C2C02D02A2C40F08280854D834A2978B1
:106DF000854B157800205854844AB5B91878157019
:106E0000472868D15978502965D19878472840F0AB
:106E1000B385D978472940F0AF851B79412B40F0E5
:106E2000AB850120107000F0A7BD117801293AD17F
:106E3000022D05D11846FFF74DFF754908604AE05D
:106E4000032D07D11978532945D17148026853425F
:106E5000036040E0042D05D11846FFF73BFF6C4B63
:106E6000586038E0052D07D11B78572B33D168497E
:106E70004A68504248602EE0062D07D119786548CF
:106E8000302994BF00210121C17224E0072D04D1D3
:106E9000FFF758FD604A10701DE0092D1BD1FFF768
:106EA00051FD5E4B16E0022915D1072D0CD10120B2
:106EB000FFF748FD41F2184250434FF47A71584BA6
:106EC000B0FBF1F0188006E0082D04D10120FFF797
:106ED00039FD544B1880494B4949013500202A2C73
:106EE0001D70087039D15048012404703EE00D2C0B
:106EF0004D4A01D00A2C26D11478FCB1424C21789D
:106F00006478A1F13000C3B2092B84BFA1F137032B
:106F1000DBB2A4F1300003F00F02C3B21101092B60
:106F200084BFA4F13703DBB2364C03F00F0289189B
:106F30002078CBB2C21A514251EB02043A4B0020E6
:106F400018707CB912E02E490B780E2B03D82E480E
:106F5000C45401330B70127842B92A4B1A7854404A
:106F60001C7003E0294A1078012800D00020C007D7
:106F700000F1338123E72D4B0022197808293FF6D1
:106F80001EAFDFE801F00A051119275F7C96A0000B
:106F9000622801D1022105E01A70B52C7FF40FAFF1
:106FA0001C78611C19700AE72149224A03261E70C9
:106FB00008701070204B0BE01E4E042119703278BF
:106FC0001D4BA1181878CAB2101818701B4B3270DC
:106FD0001C70F4E605211970164B174E1A7830789C
:106FE000A118CAB210183070154E1A703480E6E637
:106FF0006C1B0020D41C0020D0170020590E00204C
:10700000EE0D00206D0E0020780D0020480F0020AE
:10701000DC1B0020EF1C0020FA1B0020921B00202C
:107020009C1B002000080020500E0020100E0020A5
:10703000580E0020D40D0020D50D0020400D00205A
:10704000D80D00206C4906261E700A786B4BA618D6
:107050001878F2B210181870694B0A70198801EB91
:107060000424A6B2B6F5007F01D81E8003E00022FA
:107070001A80644B1A700024634B00F052BC5E49C6
:107080005E4E0A783078A318DAB2101830705E4E6F
:107090000A7033885A4AC72B98BF5C49108898BF3A
:1070A000CC545C1CA1B2884231807FF488AE0721A9
:1070B00007E0514A08261E70137883423FF47FAEE2
:1070C0000021504B6EE74D4E1A70337883427FF4A7
:1070D00076AE4F4C207806283BD005D8022813D036
:1070E00003287FF46CAE23E0122847D030287FF4C9
:1070F00066AE464A474C1679444A102E88BF102681
:1071000026702178002347E0404C434E6368A06816
:1071100021697360414B4FF47A723060404C91FBAF
:10712000F2F618783F492680C87201223E4923E0D2
:1071300036494A7912F0010004D00E79F41E6342F8
:1071400053EB040035490870002839D1354AD07214
:1071500036E02E4EF47A14F0010104D0B07AC21E4B
:10716000534253EB02012D4E317009B92D4CE1729F
:1071700026482E4990F82F200A7021E023482C49F8
:107180008669426942F210742A4B96FBF4F00A8039
:10719000188001222849EFE70C328B4210DA12F8EE
:1071A000046C264812F8034C1E54254E25489C5565
:1071B00012F8014C16781C54234C1E550133EBE792
:1071C00019490A78002A3FF4FAAD1B4B1E78002EAD
:1071D0003FF4F5AD00240C701C701C4CA068E060FE
:1071E000FEF76CF9A060202000F0A2FC18490A7894
:1071F000012A2FD100232EE0D40D0020D50D002030
:10720000D80D0020100E0020C00D0020800E0020A0
:10721000400D0020FB1B0020DC1B00206C0E00201A
:10722000921B0020EF1C0020D60D0020FA1B00202E
:107230009C1B0020000800205A0E0020801B00200C
:10724000CA1B0020E41B0020041C0020D41C0020CA
:10725000A707002001237E4C0B70E07A00283FF442
:10726000AEAD7C490A78042A7FF6A9AD677807B9E4
:107270002773257B15B90FB1FFF7ECFB764E05217F
:107280003378764F5C1C94FBF1F001FB10423270B6
:10729000734E97F800C0734D06EB82020023724CC8
:1072A00072491F59DFF810E27148724E5F5097FB28
:1072B000FEF1195006FB0170DFF8009203EB040A9F
:1072C00042F2107490FBF4F71668BCB253F80970E0
:1072D0001060C6EB07084044052643F8090090FB00
:1072E000F6F00EFB01016448BCF1010F25F8024FD6
:1072F000195005D1023CB4F5797F98BFCAF8001047
:1073000004331432082BCAD1FEF7D8F85B4D5C4C1D
:107310002A68801AF9F7F6FB5A49F9F7FFFC206052
:10732000FEF7CCF8286025684FF07E512846F9F723
:10733000DFFD08B94FF07E5525600CA90DAC4A4819
:10734000514B0194009103C80CCBFFF7B9FA0C9A8A
:1073500064234E49B2FBF3F008800D9A3C4892FB3F
:10736000F3F34B4C027B23800AB90A8022804949FF
:107370000C78002C36D0424F4FF07E503968F9F728
:10738000CDFC454D384E2B6804463068C01AF9F7DD
:10739000BDFB2146F9F70EFCF9F7D2FD726869686A
:1073A0003E4D0746501AF9F7B1FB2968F9F702FC80
:1073B0002146F9F7FFFBF9F7C3FD04B2384802256F
:1073C000B0F902303FB2E21892FBF5F1B0F90020BB
:1073D0008BB2B918334C91FBF5F291B263802180E6
:1073E000438001802B4B01201F4C1870184B6168A3
:1073F000294A20681C7A516010601CB9DA79002A89
:107400003FF4DDAC284E294D294C01960095164FCE
:1074100094E80C00FFF754FA61687868254E081A62
:10742000F9F774FB1D4B1968F9F7C4FBF9F788FDF0
:1074300070600A48226890F900303C68012BC4EB68
:10744000020131603CD0022B7FF4B9ACF2E000BF06
:10745000EF1C0020FA1B00207C0E0020B207002049
:10746000180D0020E80D0020DC1B0020640E002019
:10747000040E0020806967FF700D00204C0F002073
:10748000000E002000007A44C01B0020BE1B00201C
:10749000C81B0020E80D00205C0E002030000020FA
:1074A0003C0E00200C0E0020400E00204C0E002050
:1074B000E00D0020740E002080969800440E0020FD
:1074C000002634463546DFF874B28B4F5BF82580D2
:1074D000DFF864924046F9F719FB3968F9F76AFB5F
:1074E000F9F72EFD34F80910844B421A90B2E0529D
:1074F00007B2CDF80890DFF8489238460397F9F7BD
:1075000005FBD9F80010F9F755FBF9F719FD81B221
:107510007B48142202FB0507DFF800A2039B0891B9
:1075200003EB0800DAF800104B463A46FFF7A0F9E3
:107530000899DFF810820A185BF82500DAF800B025
:1075400024F8082008905846F8F770FFD7F808A0EC
:10755000CDE904015046F8F769FF6A4BCDE9060111
:1075600093F8C000F9F7CEFAF8F760FF60A3D3E90B
:107570000023F8F7AFFF02460B4600206249F9F7F7
:10758000D3F8DDE90423F8F7F3FD0B460246DDE905
:107590000401F9F7C9F8089ACDE9040179680135C1
:1075A000501AF9F7B3FA5946F9F7B8FB5146F9F70B
:1075B000F7F9F8F73BFF02460B46DDE90401F8F75F
:1075C00089FF0B460246DDE90601F8F7D1FDF9F720
:1075D00093F9089938617960B860D9F80810F9F71B
:1075E000E9FAF9F7ADFC49494FF4FA62FBF7B2FC4E
:1075F000DDF808C034F8081034F80C20313293B2AA
:10760000622B98BF0020401882B224F8082010B2E4
:107610003F4940F6B832FBF79DFC394B28F804008F
:1076200099593C48023431501436022D7FF44BAF47
:10763000FFF7C5BB2F68334D374CB5F9C6807E08C0
:10764000B04528BFB04625881FFA88F80FFA88F29F
:1076500029B28A420BDD314831490068F9F7AAFAAC
:10766000F9F76EFC43191FFA83F8A4F800802D4E39
:107670002D4D34682A68A61A3046FFF7BDF8002859
:10768000D8BF404241F293118842CCBF0020012074
:10769000002859D03046F9F739FA2449F9F78AFA1F
:1076A00004F0B8F805463846F9F72CFA01462846A2
:1076B000F9F780FAF9F744FC1D4B1549188040F69C
:1076C000B83200B2FBF746FC201848F6A044A042AE
:1076D00003DDA0F50C40A03804E00028BCBF00F595
:1076E0000C40A030134A106030E000BFAFF30080C0
:1076F000182D4454FB211940C40D00206C0D0020AE
:10770000440D0020041700200000F03F30F8FFFF78
:1077100048F4FFFF140E0020700E0020000E002021
:107720000000C842400E0020540E0020D30237391A
:107730006E0E0020DC0D00200C0E0020740E0020C8
:10774000F00D0020981B0020994F3C60984E0025BA
:1077500031682C46C1F50C502830F9F7D7F9954916
:10776000F9F728FA074603F0E1FF0F90384604F0D6
:1077700051F82F460E900FFA88F0F9F7C7F90EABC3
:1077800053F82710F9F716FA06468B48DFF86CA273
:10779000005FF9F7BBF901463046F9F701F9F9F74F
:1077A000CFFB864924F80A004FF47A7200B2FBF747
:1077B000D1FB82B211B2DFF8489224F80A200846C1
:1077C0000391F9F7A3F9D9F80010F9F7F3F9F9F7EC
:1077D000B7FB83B27A48142606FB0706DFF824B20B
:1077E000039ADBF80010069310464B463246FFF72B
:1077F0003FF8DBF800C034F90A1009906046D6F86B
:1078000008A00891CDF808C0F8F710FECDE90401F2
:107810005046F8F70BFEDFF8F0B1CDE90A019BF80E
:10782000C000F9F76FF9F8F701FE5FA3D3E9002371
:10783000F8F750FE02460B4600206249F8F774FF45
:10784000DDE90423F8F794FC02460B46DDE9040168
:10785000F8F76AFF089BCDE9040170680137181A30
:10786000F9F754F9DDF808C06146F9F757FA5146BF
:10787000F9F796F8F8F7DAFD02460B46DDE9040160
:10788000F8F728FE02460B46DDE90A01F8F770FC1E
:10789000F9F732F8089A099B72603061B060069E71
:1078A000D9F80810F618F9F785F9F9F749FB3018F7
:1078B000454E81B2A15308B240F6B8324349FBF7B6
:1078C00049FB3F4A3053424BA8580234E850143524
:1078D000022F58467FF44FAF90F8C21031B1344AAE
:1078E000642413683B4A93FBF4F111803A4BB0F8DF
:1078F000BE001C6884420ED9384939480A680368BA
:1079000042F21074D01AFEF777FF0028B8BF404249
:10791000A0427FF754AA3348334A012104882D4BF3
:1079200011701C80FFF74BBAFFF72EF836E0626843
:107930006078531C411CCAB263600523B2FBF3F0AC
:1079400003FB10216170FDF7B9FD284AA0602848AB
:107950000023C372137001200BE0FDF7AFFDA36895
:1079600040F6C411C01A884218D9202000F0E8F867
:107970000420FEF771FF11E01E498A78522A7FF435
:10798000AAAACB784D2B7FF4A6AA087943287FF4C6
:10799000A2AA194A02211170FFF79DBA11B0BDE8E1
:1079A000F08F00BFAFF30080182D4454FB21194025
:1079B000DC0D0020D30237390C0E002018FCFFFF2D
:1079C000140E00200000F03F981B002048F4FFFF39
:1079D000440D00202C1C00204C0E0020400E0020E6
:1079E000540E0020DA0D0020B2070020FA1B002000
:1079F000EF1C0020780D0020480F00206C0D0020A7
:107A0000880D0020000E002004170020AFF3008036
:107A10003B4B2DE9F047B3F90000F9F777F8394906
:107A2000F9F7C8F8044603F0F5FE0646204603F0D1
:107A30007DFEDFF8E490054699F8C180324FB8F139
:107A4000000F29D0314CB7F90200B4F802A00FFAA8
:107A50008AF1401AFEF7D0FEC8F100014246FBF75A
:107A600079FAB4F80080B7F900700FFA88F300EBE8
:107A70000A02F81A6280FEF7BFFE99F8C12051424F
:107A8000FBF768FA404487B22780B4F90200F9F79F
:107A90003DF8804638B206E0B7F90200F9F736F84B
:107AA0008046B7F90000F9F731F829460746404605
:107AB000F9F780F8314681463846F9F77BF80146F8
:107AC0004846F8F76DFF1249F9F728F9F9F738FA3F
:107AD000104C314620804046F9F76CF8294606469E
:107AE0003846F9F767F801463046F8F75BFF084972
:107AF000F9F714F9F9F724FA6080BDE8F08700BFC0
:107B0000581C002035FA8E3C981B0020941B002046
:107B100000002041E007002004170020034B1968F3
:107B200008420CBF00200120704700BF500F00200A
:107B3000024B1A6810431860704700BF500F0020B6
:107B4000024B1A6822EA000018607047500F0020AC
:107B5000014B1868704700BF500F0020024B5A7845
:107B60000AB1002058707047EF1C0020037A032BE5
:107B70000FD8DFE803F00202060A0649064A00F0C1
:107B8000D5BA0449044A00F03BB90249024A00F060
:107B9000FDB97047161D0020980F002010B5002376
:107BA00004466189094A99520233242BF9D10820ED
:107BB000FBF726F820B12046BDE81040FFF7D6BFFE
:107BC00003480449BDE8104000F0D8B8301D00203B
:107BD000161D0020980F00202DE9F84307460820C5
:107BE0008846FBF70DF870B10024224A414613681D
:107BF0003846E2B29847204921F814000134082C95
:107C0000F3D1BDE8F8831D4A1D4D1378591CCCB241
:107C100004F00306147005EB4609044606461548B1
:107C20004146036832463846984729F824002A8896
:107C30006988AB885018EA88C118881803B2991C63
:107C4000042291FBF2F00C4A0E4BA15EE052CB1ED7
:107C5000984201DA811CA152135FD91C884201DDD0
:107C6000023810530136F6B202340835082ED6D148
:107C7000BDE8F883980F0020301D0020540F00202D
:107C8000560F00209C0F002010B544780078002388
:107C900003FB03F11939614301F6C4115943414310
:107CA00040F6C41291FBF2F1034A22F8131001339B
:107CB000072BEDD110BD00BF541D00202DE9F04F62
:107CC00085784FF00A0C0CFB05FCC778C5F16408F9
:107CD0006E425FFA88F8C7F16409B6B2002330B289
:107CE000002804DCB8BF2C4602DB012400E0444637
:107CF00000FB00FB64430BFB07FB9BFBF4F44C44D1
:107D000044434FF00A0B94FBFBF00CEB000420B251
:107D1000C1EB020A00FB0AF44FF47A7094FBF0F412
:107D200004480C191C5202335E44182BB6B2D6D14B
:107D3000BDE8F08F181D0020F8B505460F46441E1B
:107D400014F8011F49B1054E304605F04BFE0028DE
:107D5000F6D0861B631BBB55F2E7F8BDD8F00008D0
:107D600010B50446805CF9F7FBFFA0F2EE2291B259
:107D700040F2DC53994288BF608910BD024B0B6012
:107D800008210170704700BF617D0008825C044BD0
:107D900053F82200410801F5777290B2704700BF96
:107DA000B40F002038B50446FDF76EFB104B40F6CB
:107DB000C4111A68821A8A421A460E4B01D9002150
:107DC00019701B7810600BB90F2C10D10A480021D4
:107DD0000170084A4BB1094D182B1D4405F8014CA0
:107DE00003D101230370117038BD0133137038BD06
:107DF000AC0F0020B00F0020B10F0020D40F0020E6
:107E0000408938B50D4B0D46A0F5777114464A00F0
:107E10001A605A609A60DA601A615A619A61DA618E
:107E200007490848084A0523FDF7F8F90749C860DB
:107E30000CB10748206008222A7038BDB40F00201A
:107E4000A57D000800440040A08601006C1B0020B6
:107E50008D7D0008274970B50878002849D0264B49
:107E6000987DC0F3C000002841D1244A10805D787D
:107E70001C78234A05F0070644EA062414609C781F
:107E800004F03F06760146EAD5055560DE78B50078
:107E900045EA94151C7904F0010645EA86259560AB
:107EA0005D7905F00F06F60146EA5404D4609C792A
:107EB00004F07F06360146EA15151561DE79750076
:107EC00045EAD4141D7A05F0030644EA46245461B9
:107ED0005C7A04F01F06B60146EA950595619B7A27
:107EE0000870DB0043EA5414D461012070BD002007
:107EF000087070BDB10F0020D40F00206A07002069
:107F0000B40F0020825C034B53F82200C0F3CF0073
:107F1000704700BF0810002010B50446FDF7B4FA02
:107F2000154B1A68811AB1F57A6F1A46134B01D9AD
:107F3000002119701060187820B9A82C1AD1104BA4
:107F4000187006E0022802D10E4A147001E01428CD
:107F500001D80D490C540B490130C3B20878074AC7
:107F60004100481D8342137004D10023044913705B
:107F700001220A7010BD00BF28100020041000204C
:107F80000210002003100020ED0F002038B5084833
:107F900001230D46144607494FF4E132FDF73EF93F
:107FA000054BD8600CB1054820600821297038BD08
:107FB00000440040197F00086C1B0020057F00086A
:107FC000134A10B513780BB9002010BD11490020D9
:107FD00010704A78012AF7D10F4B18800F480178AA
:107FE000082901D90822027001780D4A0023D8B26D
:107FF000023288420AD212F8010C12F8024C40EA0E
:108000000424084840F823400133F0E7012010BD64
:1080100002100020ED0F00206A070020031000204E
:10802000F00F002008100020124B012210B51A702A
:108030000446FDF729FA104A0146106811600B1A30
:108040000E4841F288318B4203600D4B01D900226A
:108050001A7018780B49E4B20F280C5406D10A495B
:108060000A4B0120002208701A8010BD044A431CEC
:10807000137010BD6C1000202C1000203410002054
:1080800039100020621D0020381000206A070020EF
:108090001F4B2DE9F0431B7823B31E4C1E4D277850
:1080A00091F800C095F8008002231C4C03F10109EF
:1080B000E65C46FA07F606F00F05EEB266450BD20F
:1080C0000B2E09D8E65C14F8094006EA080604EB12
:1080D0000626134C44F825600233102BE5D10C4BD7
:1080E00000241C700978914202D90E4B197811B9FD
:1080F0004089BDE8F0830C4B825C1978084B53F83B
:10810000220001B1400800F5777188B2BDE8F08324
:1081100038100020301000206E100020621D00205A
:108120003C1000206C1000206D10002010B5037A68
:1081300014465BB1012B13D1104A03201070104A72
:10814000072010700F4803700C2308E00B4A022030
:1081500010700B4A032010700A48037007230B703D
:1081600009490A484FF4E1320123FDF757F808495D
:10817000C8600CB1074A226010BD00BF301000205B
:108180006E1000206D10002029800008004400407F
:108190006C1B002091800008014B1878704700BFCD
:1081A0003810002008B54FF40060FAF729FD08B92F
:1081B000002008BD4020FAF723FD094B20B993F8B1
:1081C0002B21501E0128F3D993F82A01012805D14B
:1081D000034991F82B31002BEAD008BD012008BDDE
:1081E000D0170020084B93F82B215AB993F82C0193
:1081F00010B9064A537801E005490B7D181C18BFD9
:108200000120704701207047D0170020EF1C00208C
:10821000001D002010B5084B93F82A211C460AB90E
:1082200000F0AEF894F82A01012803D1BDE810400F
:1082300000F066BA10BD00BFD017002038B50E4B55
:108240001878C0B1FFF7CEFF0C4904460A78824285
:1082500011D060B10A4D95F82A310BB900F09CF8A5
:1082600095F82A01012804D100F042FA01E0FFF755
:10827000D1FF02490C7038BD701000206F10002033
:10828000D017002010B54020FAF7BAFC0B4C08B903
:1082900084F82B01FFF786FF94F82B21084B012A65
:1082A0001870084801D1084A03E0022A0CBF074AA7
:1082B00002688260BDE81040FFF7C0BFD017002001
:1082C000701000206C1B00206C110020B4130020E3
:1082D0000B4B10B5187888B1FFF784FF70B10949CE
:1082E00091F82A210C460AB900F06EF894F82A3168
:1082F000012B03D1BDE8104000F00ABA10BD00BF49
:1083000070100020D017002038B5064C05465E21BD
:10831000A068FCF732FEA0682946BDE83840FCF7AB
:108320002CBE00BF6C1B0020024B5E219868FCF73E
:1083300024BE00BF6C1B002010B50A4C5E2801460D
:10834000A06805D15D21FCF718FEA0683E2105E07C
:108350005D2903D1FCF711FEA0683D21BDE8104066
:10836000FCF70BBE6C1B002010B50446C0B2FFF733
:10837000E3FFC4F30720BDE81040FFF7DDBF0000B6
:10838000044B93F82B211AB9D3F8200101F05CBB00
:10839000704700BFD0170020044B93F82B0118B989
:1083A0004FF4165001F050BB704700BFD0170020AB
:1083B00008B5044B9868FCF7F0FDD0F1010038BF18
:1083C000002008BD6C1B00202DE9F041FFF7F0FFF5
:1083D000002800F04081FDF771F8A04B1A68811A5F
:1083E0007C2940F2388118609D480478651C05702E
:1083F000002404F12406F0B2FFF786FF994B33F90D
:108400001400F8F783FB984A05461088F8F77EFBBE
:1084100001462846F8F782FC9449F8F7CBFBF8F7B9
:108420008FFD013400B2FFF79FFF032CE1D1302014
:10843000FFF76AFF8E49B1F90000FFF795FFFFF7DC
:1084400073FF8748067816F0030629D1894D10205E
:10845000FFF75AFF2B68642493FBF4F210B2FFF786
:1084600083FF2120FFF750FF296891FBF4F004FB04
:10847000101484EAE473A3EBE47318B2FFF774FFFB
:108480001420FFF741FF7C4AB2F90000FFF76CFFB0
:108490001C20FFF739FF3046FFF766FFFFF744FF68
:1084A0006F490878430740F0B080744D0220FFF711
:1084B0002BFFB5F900300A2593FBF5F0FFF754FFC9
:1084C0000220FAF79DFB002847D06D4F6D4E38789B
:1084D000347840F63401B4FBF0F26B4C4A43218807
:1084E0002A2391FBF0F800FB1810B2FBF3F24FEADD
:1084F000001399B241EA022C1FFA8CFEC2F3032248
:108500004EEA02080620FFF7FFFE0FFA88F0FFF799
:108510002BFF20883F78431C9AB292FBF7F107FBB0
:108520001120367820806E247443152394FBF3F4D5
:108530003A206427FFF7E8FEB4FBF7F63046FFF772
:1085400013FF3B20FFF7E0FE07FB164291B24C1DE4
:1085500094FBF5F000B2FFF707FF2020FFF7DEFAEB
:10856000002850D0494C1320FFF7CEFE2568484F15
:10857000002DB8BF6D4295FBF7F630B2FFF7F4FE61
:108580001B20FFF7C1FE23680A26002BB8BF5B4201
:1085900093FBF6F142F2107591FBF5F205FB121018
:1085A00000B2FFF7E1FE2320FFF7AEFE2368002BA9
:1085B000ACBF4E205320FFF7D7FE1220FFF7A4FEDA
:1085C00061680029B8BF494291FBF7F210B2FFF78A
:1085D000CBFE1A20FFF798FE60680028B8BF404223
:1085E00090FBF6F696FBF5F305FB136108B2FFF777
:1085F000BBFE2220FFF788FE6268002AACBF452040
:108600005720FFF7B1FEFFF78FFE15480378282BA0
:1086100021D100240470FCF751FF4FF47A753C24FB
:10862000B0FBF5F61720FFF76FFEB6FBF4F5B5FBD0
:10863000F4F104FB1152100200B2FFF795FE18206E
:10864000FFF762FE04FB156318B2FFF78DFEBDE86D
:10865000F041FFF769BEBDE8F08100BF7410002053
:1086600071100020881C00201200002000007A44B5
:10867000400C0020080C0020581C0020901B0020FB
:108680000A000020FC16002078100020DC1B0020CF
:10869000A0860100154B2DE9F04180460F469868F1
:1086A0000221FCF78EFC00242646781E84420F4DE2
:1086B0000DDA18F80410A8688E190134FCF75DFC77
:1086C0004FF47A70B6B2FCF7FFFEE4B2EDE7F1B218
:1086D000A868FCF752FC4FF47A70FCF7F5FEA86826
:1086E0000121BDE8F041FCF76CBC00BF6C1B002011
:1086F000024B01219868FCF764BC00BF6C1B002092
:10870000024B03219868FCF75CBC00BF6C1B002087
:10871000F8B5544CA068FCF740FC002800F0A0809D
:10872000A068FCF73FFC05460520FCF7D8FE8A2D23
:1087300021D08E2DEDD14C4C00212E22204605F06B
:1087400095F84A4A7C2323701378E0207D21E0705D
:1087500084F82C1014204FF4FA71A3772375482263
:1087600078232076607661836570628484F8243093
:1087700020462E2171E02020FFF7D0F90028C8D034
:108780003B4C00212C22204605F070F8A021E1701E
:10879000384B39497C207D22207084F82B201878B2
:1087A000CA7A6570A076002A52D0344934480F68DE
:1087B0006625FE0F97FBF0FC6672324E5FFA8CFC6A
:1087C00006FB0C7284F8295006256A4342F21073A6
:1087D000B2FBF3FE03FB1E274968277391FBF0F001
:1087E0003F0AC0B26773CF0F06FB00116943B1FBAC
:1087F000F3F5642203FB1513E9B202FB0010010A32
:10880000E0732148217401885FFA8EFE63741B0AAD
:1088100002FB0CECA374B1FBF2F224235A4390B296
:108820001A4A010A1388E0712172180A1849207542
:1088300018480A8801884FEA1C2EE374130A84F84A
:108840000AC084F80BE0A7736275A375217702E074
:10885000202384F8293006482C21FFF71BFF58E716
:10886000F8BD00BF6C1B0020A6100020FC160020E5
:108870007A100020FA1B0020EF1C0020DC1B0020D7
:10888000A08601006079FEFF9C1B0020BE1B00201B
:10889000921B0020C81B002070B50646B6FBF2F400
:1088A0000846154614B12046FFF7F6FF05FB146491
:1088B000024B195D00F8011B70BD00BF5CF200089F
:1088C0002DE9F041027803460130202AFAD0092A26
:1088D000F8D02D2A02D10346414D04E02B2A08BFCF
:1088E00003464FF07E551E460024334616F8010B12
:1088F000A0F13007F9B209290DD83A492046F8F716
:1089000059F904463846F8F701F901462046F8F7C8
:1089100049F80446E9E72E2817D1324F334616F8B6
:10892000010B3038C2B2092A0FD8F8F7EFF83946F0
:10893000F8F7F4F901462046F8F734F829490446D7
:108940003846F8F737F90746E8E71878652801D080
:10895000452839D15E782D2E02D19F1C012605E0D5
:108960002B2E01D05F1C00E09F1C00267B1E0027E1
:1089700013F8012F303AD1B2092903D80A2000FB9D
:108980000727F5E7B7F59A7F28BF4FF49A77B846DF
:108990004FF07E51B8F1070F07D908461249F8F792
:1089A00009F9A8F108080146F4E707F0070737B10D
:1089B00008460C49F8F7FEF8013F0146F7E72EB1EB
:1089C0002046F8F7ABF904E04FF07E512046F8F767
:1089D000F1F801462846F8F7EDF8BDE8F08100BF50
:1089E000000080BF0000204120BCBE4C10B5441EDA
:1089F00014F8011F21B1034B1868FCF7BEFAF7E722
:108A000010BD00BF6C1B00200148FFF7EFBF00BF87
:108A100081F2000810B50748FFF7E8FF0024064B75
:108A200006481A19E15852680C34FAF7C3FBC02CF7
:108A3000F5D110BDAFF2000880F10008C5F20008C2
:108A400070B5FCF73BFD274C274B4FF47A71B0FB18
:108A5000F1F11A7825482378FAF7ACFBFFF778F89C
:108A600005462348234902682348B2FBF1F1FAF78F
:108A7000A1FB0024214B53F8241051B1012000FA2E
:108A800004F0284202D01E48FAF794FB0134E4B205
:108A9000F0E70220FFF742F898B11A4C1A49227801
:108AA0001A4851F82210FAF785FB2378022B08D1D7
:108AB0001748047C1748002C0CBF6E216F21FAF771
:108AC00079FB1548FFF792FF144A1488FCF714FA53
:108AD0000246134821464FF46673BDE87040FAF72A
:108AE00069BB00BF0A000020FC160020CDF2000880
:108AF0005001002040420F000BF3000894000108D1
:108B000029F300087408002040F200082DF3000843
:108B10006C1B002037F30008ECF50008E407002088
:108B20003BF3000838B50C680546204605F036F8DA
:108B3000024628682146BDE8384005F05FB80000CD
:108B400008B50948FFF752FF01210020F9F7F4FFAB
:108B50000648FFF74BFF0A20FCF7C1FC0020BDE8E8
:108B60000840FCF739BD00BF6DF3000877F300083B
:108B70007FB5044605F012F8082825D100231F49C7
:108B8000E25C086885186E7806F00301022908BFC8
:108B9000203AE2540133082BF1D10025665D1848D4
:108BA000314604F01FFF28B101356019314604F049
:108BB00019FF18B11348FFF719FF1DE0082DEDD17B
:108BC00020461149FFF7B8F81048FFF70FFF0023C0
:108BD0000F4A04A9981890F808218818084A995C47
:108BE0000133082B00F80C1CF2D100208DF80C008A
:108BF00001A90848FAF7DEFA7FBD00BF6C0100202A
:108C0000D8F0000886F30008D8180020A6F3000862
:108C1000D0170020C8F2000808B5FDF7EFFF0130BB
:108C20000CBF03480348BDE80840FFF7DFBE00BFA4
:108C3000BBF30008E1F300082DE9F041054604F01C
:108C4000ADFF0446FAF780F9064694B92A48FFF7C3
:108C5000CDFE2A4951F8241049B1012202FA04F24A
:108C6000324202D02648FAF7A5FA0134F1E7254846
:108C700021E028462449224604F0C0FF58B9234881
:108C8000FFF7B4FE224C54F8041F0029EFD01C4813
:108C9000FAF790FAF7E72B782D2B04D10135013C38
:108CA0004FF0010801E04FF000080026134850F88B
:108CB000267027B91748BDE8F041FFF797BE284650
:108CC0003946224604F09AFFA0B9012000FA06F0C6
:108CD000B8F1000F03D0FAF72FF90F4802E0F9F7C7
:108CE00099FF0E48FFF782FE0D483946BDE8F04176
:108CF000FAF760BA0136D9E7FFF30008E4F000089C
:108D000029F30008ECF500089EFE000812F40008A4
:108D1000E0F0000827F4000841F400084BF40008D4
:108D2000C8F2000810B504460848FFF75FFE084A7D
:108D3000084809490023036013700B70FDF7ECF835
:108D40002046BDE81040FFF7FBBE00BF54F400080A
:108D5000D510002008110020D410002008B50848C4
:108D6000FFF744FE0120F9F75DFF0648FFF73EFEDE
:108D70000A20FCF7B4FB0020BDE80840FCF72CBC3F
:108D80006CF4000879F30008F8B5074604F006FF14
:108D9000044638B91A491B4B4A791B48511E53F8EF
:108DA000211028E038461949224604F027FF60B90F
:108DB0001748FFF71BFE174C54F8041F19B116484B
:108DC000FAF7F8F9F8E7154805E000250D4B53F8D8
:108DD000256026B91248BDE8F840FFF707BE3846BF
:108DE0003146224604F00AFF01350028EED104483E
:108DF000314645710B48BDE8F840FAF7DBB900BFD2
:108E0000D017002024F1000887F400089EFE000817
:108E10009BF4000820F1000829F30008ECF5000895
:108E2000AEF40008C6F4000810B50446204604F06D
:108E3000B5FE10F0FF0F07D10B490C4891F89413C1
:108E4000BDE81040FAF7B6B9204604F0C5FB022889
:108E500008D8054B064C83F8940300200146F9F727
:108E60006BFEE3E710BD00BFD0170020D8F4000868
:108E7000FCF7000870B5044604F090FE08B92048DD
:108E800030E020461F4905F001FB00242646254618
:108E900078B12CB1012C06D104F09EFB064602E00D
:108EA00004F09AFB054600201649013405F0EEFA5D
:108EB000EEE70B2D05D914480C21BDE87040FAF7F8
:108EC00079B9012C08DC114A114832F915202946DC
:108ED000BDE87040FAF76EB9A6F57A73B3F57A7FFC
:108EE00004D90C48BDE87040FAF764B90A4829462D
:108EF0003246FAF75FF9054820F8156070BD00BFEB
:108F0000EEF40008C6F7000828F50008B81C002099
:108F10004EF5000866F5000888F5000838B50546E6
:108F200004F03CFEC0B268B904461249124801EB95
:108F30004402B2F8422021460134FAF73BF9152CDD
:108F4000F3D138BD284604F047FB142804460BDC57
:108F50002021284604F046FD04F03EFB054B03EBC0
:108F60004404A4F8420038BD04481521BDE8384047
:108F7000FAF720B904170020A1F50008ADF50008A4
:108F8000931E222B88BF0A22031E10B50C4603DA5B
:108F90002D2001F8010B5842FFF77EFC00210170E3
:108FA000204610BD30B587B005460C4603A8002109
:108FB0000C2204F05BFC28460021F7F7B7FF20B134
:108FC00028462949F7F7EEFC03E028462649F7F73B
:108FD000E7FC2649F7F7EEFDF7F7B2FF054685EA0D
:108FE000E570A0EBE5700A226946FFF7C9FF002D86
:108FF00001DB202300E02D2368468DF80C3004F0BF
:10900000CDFD012807D130228DF80D208DF80E20DE
:109010008DF80F200CE0022805D130218DF80D10BD
:109020008DF80E1004E0032802D130208DF80D00D9
:10903000694603A804F0B0FC03A804F0AFFDC51E08
:10904000EDB22A4603A9204604F046FE00236355EC
:109050002046074904F0A0FC03A92046491904F062
:109060009BFC204607B030BD6F12033A00007A44E3
:1090700084F3000837B5037904460D46052B34D830
:10908000DFE803F003060A0D1114816809782DE06A
:10909000806890F9001029E08368198826E08268CA
:1090A000B2F9001022E0816809681FE08068694613
:1090B0000068FFF777FF01461148FAF77BF8F5B132
:1090C000E068F7F723FD6946FFF76CFF01460D489E
:1090D000FAF770F82069F7F719FD6946FFF762FFA4
:1090E00001460848FAF766F809E000210648FAF751
:1090F00061F825B10548E1682269FAF75BF83EBDE1
:1091000034F3000833F30008D7F50008D3F500085E
:109110002DE9F047064604F041FD054620B101283F
:1091200019D133782A2B16D14748FFF75FFC00246A
:1091300014266643454F4648F159FAF73BF8B819EB
:109140002946FFF797FF01344248FFF74FFC6E2C8A
:10915000EED1BDE8F08730463D2104F043FC002805
:1091600057D0441C204604F037FA82462046FFF7C9
:10917000A7FB0027054614247C43DFF8D09054F861
:109180000980404604F00AFD41460246304604F09C
:1091900035FD002835D14C44E068F7F7B7FC0146AF
:1091A0002846F7F7B9FE002829D02069F7F7AEFC6A
:1091B00001462846F7F7A6FE002820D0207922791C
:1091C000052818BF5546052A0FD8DFE802F003032B
:1091D0000606090CA1680D7007E0A268158004E07E
:1091E000A068056001E0A1680D6041461A48F9F7E2
:1091F000E1FF20460021BDE8F047FFF73BBF1748DD
:1092000003E001376E2FB6D11548BDE8F047FFF7F0
:10921000EDBB0446142565430C4F314655F80780D5
:10922000404604F0BDFF50B109484146F9F7C2FF7E
:1092300078190021FFF71EFF0648F9F7BBFF01343C
:109240006E2CE7D1BDE8F087DAF50008B40001081C
:10925000B9F60008ECF50008EFF50008FAF500088B
:109260001FF600082DE9F043584885B0584CF9F72F
:10927000A1FF5848FFF752FE6279574B511E5748DD
:1092800053F82110F9F796FF20690021F7F726FE21
:10929000002858D10025266900213046F7F71EFE28
:1092A00000284CD101354E482946D4F81490D4F802
:1092B0001880E769F9F77EFF30460021F7F718FEBE
:1092C00010B14848F9F776FF69463046FFF76AFE65
:1092D00001464548F9F76EFF48460021F7F708FEBA
:1092E00010B14048F9F766FF69464846FFF75AFE55
:1092F00001463D48F9F75EFF40460021F7F7F8FDCB
:1093000010B13848F9F756FF69464046FFF74AFE64
:1093100001463548F9F74EFF38460021F7F7E8FDDA
:1093200010B13048F9F746FF69463846FFF73AFE74
:1093300001462E48F9F73EFF10340C2DABD12C48D6
:10934000691CF9F737FFF9F7FFFD2A4C064654F878
:10935000041F19B12848F9F72DFFF8E70D462748F3
:1093600050F8251049B1012202FA05F2324202D02A
:109370002348F9F71FFF0135F1E7154B214ACE18B5
:1093800096F808418B5C04A801310519082905F8F5
:10939000103CF2D100241C4869468DF80840F9F7CA
:1093A00009FF14256543194E1948A959F9F702FF19
:1093B00000217019FFF75EFE01341648FFF716FB17
:1093C0006E2CEED105B0BDE8F08300BF3CF600087E
:1093D000D0170020FCF7000824F100086CF6000804
:1093E00077F60008C6F7000834F30008C8F2000852
:1093F0007FF60008E0F0000891F60008E4F00008AD
:109400009FF60008D8F00008ACF60008B400010888
:10941000B5F60008ECF500082DE9F04389B00446E4
:1094200004F0BCFBC6B2002E6AD17948FFF7DEFA21
:10943000784C20690021F7F751FD38BB013676489A
:109440003146F9F7B7FE206904A9FFF7ABFD0146E5
:109450007248F9F7AFFE606904A9FFF7A3FD014662
:109460006E48F9F7A7FEA06904A9FFF79BFD014626
:109470006A48F9F79FFEE06904A9FFF793FD0146EA
:109480006748F9F797FE10340C2ED2D10025654CB1
:109490002F46A8464FF000091034B14514DA404673
:1094A00054F8101CF7F77EFA54F80C1C8046284636
:1094B000F7F778FA54F8081C05463846F7F772FAB9
:1094C00009F101090746E7E75748CDF804800295FE
:1094D0000397FFF78BFA002401A82358534923F080
:1094E0000040F7F723FD5249524A0434002814BFC4
:1094F00010460846FFF77AFA0C2CEDD14E4870E082
:1095000020464E49052204F079FB38B9414B002230
:10951000C1181030C0280A61F8D176E020464849C9
:10952000042204F06BFB0546204605BB202104F015
:1095300059FA002869D0461C304604F02FFB2C460F
:109540000746404850F824500DB93F4849E030469E
:109550002946FAB204F052FB38B92046FCF77EFDEA
:109560003A482946F9F726FE47E00134E9E704F0D6
:1095700033F8461E0B2E074643DC2046202104F01C
:1095800031FA054640B1451C2846FFF799F9214BB1
:109590003F01D851012400E004462846202104F070
:1095A00021FA054640B1451C2846FFF789F91949BB
:1095B000013401EB061250612846202104F012FA12
:1095C000054640B1451C2846FFF77AF9114B013496
:1095D00003EB061188612846202104F003FA18B92C
:1095E0001B48FFF703FA10E00130FFF769F9094A59
:1095F000032C02EB0616F061F2D11648FFF70CFFC0
:1096000003E015480C21F9F7D5FD09B0BDE8F0835A
:10961000C7F60008D0170020F2F60008F8F6000898
:10962000C8F20008E4170020FCF600080AD7233C23
:10963000C3F60008BFF60008ECF500080BF70008B9
:1096400011F7000824F10008AEF4000816F700082E
:1096500029F70008FCF7000863F70008F0B5694B2C
:1096600087B01A783AB9012018706748FFF7BEF939
:109670006648FFF7BBF9664C2068FBF78EFC0028B4
:1096800000F0BD802068FBF78DFC09280146614A87
:1096900001D03F2851D1002517685F4C2E462FB1CD
:1096A0005E4821683A4604F0A9FA10B9254606B981
:1096B00026465B490C348C42F1D3C6B13468D5F8E8
:1096C00000E03B46E05C1EF8031081420DD1534A96
:1096D00041B92D2B06D820244E48D45401330360C1
:1096E000D15404E0D0540133ECE74A490B60494AB5
:1096F00014681CB1AE4201D13C4612E04948FFF764
:1097000075F9AE4209D856F80C0BFFF76FF9404BCC
:1097100009211868FBF731FCF3E73C48FFF766F9CD
:1097200000243C4B18688442A5D239493B4A08685A
:10973000115DFBF722FC0134F3E713682BB9042811
:1097400038D13648FFF7EEFA59E00C2801D13648F7
:109750008CE70A2901D00D2948D12E4D3348FFF757
:1097600045F92E4C2A6832490023A35404930091F2
:1097700003A8294910220C23039403F031FF054666
:1097800038B1006804F00AFA0130AA68201890473E
:1097900002E02848FFF72AF9002130221F4804F090
:1097A00065F818481B4B027800211960002A7FF4E5
:1097B0005FAF24E00C28CAD07F2903D15BE72F2BB1
:1097C0003FF659AF1F297FF656AF7E293FF653AFBC
:1097D00013B920293FF44FAF104C0E480C4AE15406
:1097E000013303601068FBF7C8FB44E77F29E6D12B
:1097F0000A485C1E0021015514600F4839E707B084
:10980000F0BD00BFD41000208BF70008C3F700089C
:109810006C1B00200811002080F10008D5100020EA
:1098200040F20008C8F70008CDF70008ECF5000882
:10983000258B0008D8F70008F9F70008F8B5174E8F
:10984000174C184D0746C1B230682170FBF795FBE5
:1098500022782B78C7F3072182EA0300287030684A
:109860002170FBF78AFB21782A78306881EA0203AD
:10987000C7F307412B702170FBF77FFB2078297815
:1098800080EA0102390E306821702A70FBF775FBFF
:109890002B78207880EA03012970F8BD6C1B00202A
:1098A000121100200C110020F8B50D4E0D4D0E4C7C
:1098B000C1B2074630682970FBF75FFB2A7823782E
:1098C000391282EA0300207029703068C9B2FBF7B0
:1098D00054FB23782A7882EA03002070F8BD00BF89
:1098E0006C1B0020281100200C110020054B10B526
:1098F000044621461868FBF740FB034802785440B1
:10990000047010BD6C1B00200C110020034B044997
:109910001A78885C01321A70704700BF0D11002060
:109920002911002010B5FFF7F1FF0446FFF7EEFF05
:1099300004EB002080B210BD10B5FFF7F3FF044622
:10994000FFF7F0FF04EB004010BD000038B50446FF
:1099500024200D46FFF7CAFF4D20FFF7C7FF002C5C
:109960000CBF3E202120FFF7C1FF064B00222846F6
:109970001A70FFF7BBFF04480078BDE83840FFF7D6
:10998000B5BF00BF0C110020691100200146002066
:10999000FFF7DCBF01460120FFF7D8BF014B187865
:1099A000FFF7A4BF0C11002070B5054608460E460F
:1099B000FFF7ECFF2C467219D0B2E3B2984204D004
:1099C00014F8010BFFF792FFF5E770BD10B5441EC8
:1099D00014F8010F10B1FFF789FFF9E710BD00007F
:1099E0002DE9F843002701240025144B18788542FF
:1099F0001CDA1349134B15F801800C2202FB0830C6
:109A0000406804F0CBF881460CB13F180CE02646C4
:109A10004E4509DA0B4A0C2101FB08235868805D8A
:109A2000FFF764FF0136F3E70135DEE724B1F8B252
:109A3000FFF7ACFF0024D7E7BDE8F8830E11002044
:109A4000131100203400002070B5024600210323CA
:109A50003B48FBF7E3FB3B4D3B4BFF2118601522D6
:109A6000284603F003FF002028700220FEF756F876
:109A7000012418B102216C70A97003240420FEF7A0
:109A80004DF868B12F4E03224FF400503255651C3B
:109A9000F9F7B6F818B104237355023400E02C46E8
:109AA0000220FEF73BF848B1264805210619062298
:109AB000072501557270B570033404E00820FEF7E5
:109AC0002DF80028F0D12020F9F79AF818B11D4B95
:109AD0000820185501344FF48070F9F791F830B12F
:109AE00018490A260D190B220E556A7002341748C0
:109AF000144B4179082901D00E2902D10C261E559C
:109B000001340D2504201D55651CF9F779F818B1AD
:109B10000C4811224255A51C0C4B132193F82C2103
:109B2000084E6C1C101C18BF01207155F9F768F81D
:109B300010B114203055AC1C05490C7070BD00BF2D
:109B400000380140131100206C1B0020D0170020AA
:109B50000E110020F8B5AF4B187880B1BDE8F84081
:109B6000FFF77CBD2068FBF71DFAAB4B1A7802BBF0
:109B7000B0F12404614251EB04021A703AB1A74CCF
:109B80002068FBF70AFA0028ECD100F010BDA44BC6
:109B90005C78002CF3D1232802D1FFF75FFDEEE7BC
:109BA000A04991F895238242E9D10120FBF714FDE9
:109BB000E5E7012A04D14D280CBF0220002005E072
:109BC000022A05D13C280CBF032000201870D6E7DC
:109BD000032A0FD140284FF0000200F2E584924999
:109BE000924C0870924922700A70924A10700422B6
:109BF00000F0DABC042A08D18E4A8F491478087024
:109C000060401070052200F0CFBC052AB7D187490B
:109C1000854C0A7823789342864B07D91C784440B8
:109C20001C70864B9854501C0870A8E71978814224
:109C300040F0B88480480278782A00F0858277D88E
:109C40006D2A00F01D8341D8682A00F0B18224D823
:109C5000652A00F0BD8118D8642A40F09E84072050
:109C6000704CFFF793FEE620FFF740FE6079FFF7A8
:109C70003DFE0020FFF73AFE94F81911704B714831
:109C8000002918BF184600F02FBC662A00F01E827B
:109C9000672A40F082846C488BE26A2A00F0C08216
:109CA000C0F0B2826B2A00F0D9826C2A40F0758431
:109CB000664C0620FFF76AFEB4F90000FFF7F4FDDA
:109CC000B4F90200FFF7F0FD6148E1E2722A00F00A
:109CD000468313D86F2A00F0EF82C0F0DC82702A2E
:109CE00000F00883712A40F058845A490A785400D9
:109CF00004F0FE00FFF74AFE002415E3752A00F089
:109D00000C8309D8732A00F05C83742A40F04584E0
:109D1000FFF766FE00F044BC762A00F05D83772AE8
:109D200040F03B844B4B00241878FFF72FFE0BE3E9
:109D3000CF2A00F0068147D8CA2A00F0C48037D85D
:109D4000A42A00F0098410D8A02A40F02684424CAE
:109D50000C20FFF71BFE2068FFF770FD3F490868E5
:109D6000FFF76CFD3E4A1068BEE3C82A00F0A280EF
:109D7000C92A40F01284FFF7C9FD294B394CD8722B
:109D8000FFF7C4FD2070FFF7D7FD374C2060FFF7C9
:109D9000D3FD6060FFF7C6FD34490880FFF7C2FDC0
:109DA000334A10803348037843F00204047082E39E
:109DB000CC2A00F0A980C0F09680CD2A00F06983FB
:109DC000CE2A40F0EA836CE3D42A00F0D7810FD882
:109DD000D12A00F02983C0F05583D22A00F0E68012
:109DE000D32A40F0DA83FFF79DFD2349088062E320
:109DF000F02A00F06C8343D8D62A00F0CE80EF2AF8
:109E000040F0CB83FFF78EFD1C4CA085FFF78AFD49
:109E1000608550E3D41000200F1100206C1B00203F
:109E2000EF1C0020D017002011110020101100207D
:109E30000D1100200C1100206911002029110020B3
:109E40000C0000800400008020000020180C00207E
:109E5000581C00200E110020E8F7FF1FECF7FF1F31
:109E6000F0F7FF1FFA1B0020DC1B0020921B0020D4
:109E70009C1B0020A70700202C1C0020041700209A
:109E8000FA2A00F01483FE2A40F087830820FFF7A7
:109E90007DFDCA4CCA4BCB4819682368B1FBF0F270
:109EA000B3FBF0F04FF47A7101FB0204C64AD48090
:109EB000002404E30024FFF735FDC44908530234AD
:109EC000102CF8D1F7E2C24C04F10A05FFF71EFD91
:109ED00001346070FFF71AFDE072FFF717FDAC4226
:109EE0006075F3D1E7E20024BA490A78944280F021
:109EF000E282B94D655DFFF715FDB84B013403EB08
:109F00004505A5F84200EFE7FFF700FDB34CE07709
:109F1000FFF7FCFC84F82000FFF7F8FC84F823002E
:109F2000FFF7F4FC84F82400FFF7F0FC84F8250028
:109F3000FFF7ECFC84F82100FFF7E8FC84F822002E
:109F4000B9E2FFF7EFFCFFF7EDFCA54CA34DA4F839
:109F5000D000FFF7E7FCA4F8D200FFF7E3FCA4F879
:109F6000D400FFF7DFFCA5F8B600FFF7DBFCFFF736
:109F7000E3FCFFF7D7FC0A2148432885FFF7C6FC1E
:109F800084F80401FFF7C2FC84F80601FFF7BEFC69
:109F900084F80501FFF7BAFC8DE20024FFF7C2FC4C
:109FA000904A10530234102CF8D184E28E48427843
:109FB000002A40F08082FFF7A9FC894B022883F831
:109FC000940302D9002483F894430020014670E2F0
:109FD000864D0B20FFF7DAFCB5F90000FFF764FCB3
:109FE000FAF78AFF00B2FFF75FFC0220FDF796FD4B
:109FF00005460420FDF792FD04460820FDF78EFD7E
:10A00000800040EA44022A43202094B2FDF786FDF6
:10A0100044EAC00110208CB2FDF780FD44EA001331
:10A0200018B2FFF741FC70480179C2788C00437880
:10A03000817944EA42021A4342EAC1044279437AEE
:10A0400044EA421141EA8314694BDA79197A44EA05
:10A05000C21444EA01225C7AC17942EA442242EA0B
:10A060008124027A807A44EAC2215A7B41EA003490
:10A07000987B44EA42311A7C41EA8034187944EAF8
:10A0800002415A7C41EA0014987C44EA4241DA7C5D
:10A0900041EA80441B7D4F4844EAC24141EA0354EF
:10A0A0000178002003468B420AD24B4D01225D5DB0
:10A0B00002FA05F525421CBF9A4010430133F2E72E
:10A0C000474CFFF7BBFB94F89403AAE11220FFF77B
:10A0D0005DFC484A1488B4F5806F474CB4F9000021
:10A0E00008D8FFF7E1FBB4F90200FFF7DDFBB4F994
:10A0F00004000EE0082590FBF5F0FFF7D5FBB4F95E
:10A10000021091FBF5F0FFF7CFFBB4F9043093FB9D
:10A11000F5F03A4CFFF7C8FBB4F90000FFF7C4FBB9
:10A12000B4F90200FFF7C0FBB4F90400344CFFF7A8
:10A13000BBFBB4F90000FFF7B7FBB4F90200FFF76F
:10A14000B3FBB4F90400CCE13820FFF71FFC234C2B
:10A1500004F14005B4F97400FFF7A6FBB4F97600EA
:10A16000FFF7A2FBB4F97800FFF79EFB94F87A00A2
:10A170000834FFF7BBFBAC42ECD111E20020FFF743
:10A1800005FC164C04F14005FFF7CCFBA4F8740065
:10A19000FFF7C8FBA4F87600FFF7C4FBA4F878002B
:10A1A000FFF7B4FB84F87A000834AC42ECD1F7E155
:10A1B00014481021FFF7F8FBF2E100BF5001002026
:10A1C0004C01002040420F00A81B0020301D002041
:10A1D000031700200E110020131100200417002087
:10A1E000D0170020B81C0020EF1C0020E40700203E
:10A1F000001D002012000020881C0020F40B00200D
:10A20000141C0020A01C00201020FFF7BFFB00241E
:10A21000B748005F0234FFF747FB102CF8D1BFE1CD
:10A220001020FFF7B3FBB349B34CC87AFFF75EFBCE
:10A23000B24A1078FFF75AFB2068FFF7FFFA606810
:10A24000FFF7FCFAAE4BB3F90000FFF72DFBAD486A
:10A25000B0F90000FFF728FBAB4819E00520FFF735
:10A2600095FBAA48B0F90000FFF71EFBA849B1F919
:10A270000000FFF719FBA74A137803F00100D0E0B4
:10A280000620FFF783FBA44B1868FFF7D7FAA34813
:10A29000B0F9000025E10720FFF778FBA049087816
:10A2A000FFF724FB0020FFF7FFFA9E4AB2F90000F7
:10A2B000FFF7FAFA002014E19B4C0720FFF766FB3A
:10A2C000E07FFFF713FB94F82000FFF70FFB94F8F3
:10A2D0002300FFF70BFB94F82400FFF707FB94F82B
:10A2E0002500FFF703FB94F82100FFF7FFFA94F82D
:10A2F000220096E01E20FFF749FB8C4C04F10A0572
:10A3000001346078FFF7F2FAE07AFFF7EFFA607D48
:10A31000FFF7ECFAAC42F3D142E12F20FFF736FB16
:10A320008348FFF753FB3BE1824B1878844280F06F
:10A33000378181497C4B625C013403EB4200B0F908
:10A340004200FFF7B1FAEFE77A4801788C4280F0DB
:10A350002781794A105DFFF7C9FA0134F4E7774C99
:10A360001620FFF713FB0020FFF79EFAB4F9D00088
:10A37000FFF79AFA6C4DB4F9D200FFF795FAB4F9E9
:10A38000D400FFF791FAB5F9B600FFF78DFA002077
:10A39000FFF78AFA0020FFF751FAB5F928100A22D0
:10A3A00091FBF2F0FFF780FA94F80401FFF79EFAB0
:10A3B00094F80601FFF79AFA94F80501FFF796FA68
:10A3C0002EE00820FFF7E2FA0124E0B20134FFF7A3
:10A3D0008DFA092CF9D1E3E0FFF798FA064612202E
:10A3E000FFF7D4FA0EB9564B02E0102E03D1554BAD
:10A3F0001D685C6801E0002425463046FFF776FAC8
:10A400002846FFF71BFA2046FFF718FA4E48006867
:10A41000FFF714FA0020FFF747FA0020FFF744FA8D
:10A420000020FFF763FABBE0FFF770FA0546FFF77D
:10A4300083FA0746FFF780FA0646FFF77DFA0446DF
:10A44000FFF770FAFFF76EFAFFF760FA55B93C4A6A
:10A45000284B012117605660DD7119735CB33A48CF
:10A46000046028E0102D26D1364A176056600CB1E2
:10A47000354B1C603548022101703248011DFCF744
:10A48000E5FB18E01B494878A8B90120F8F7CAFB9A
:10A4900011E0184A547874B92D4B4FF4C8701880E5
:10A4A00009E01448437833B90121817303E00020A7
:10A4B0000121F8F741FB0020FFF768FA70E0254B17
:10A4C000185F0234FFF7F0F9082CF8D168E0164C59
:10A4D0000420FFF75BFAB4F92C00FFF7E5F9B4F9B3
:10A4E0002A00FFF7E1F95BE0FFF7A8F958E000BFA9
:10A4F000301D0020EF1C0020DC1B0020FA1B002078
:10A50000921B00209C1B002000080020BE1B002086
:10A51000C81B0020A7070020801C0020400C002042
:10A52000FC160020F81B0020041700200317002051
:10A530004C0901080E11002013110020D017002033
:10A54000C01B0020A01B0020841C0020B20700209C
:10A5500008080020A81B0020154C22789000431CFE
:10A56000D8B2FFF713FA2078FFF7C0F9002410499A
:10A570000A78944214D20F48005DFFF7B7F90E4BEA
:10A58000185DFFF7B3F90D49085DFFF7AFF90C4A05
:10A59000105DFFF7ABF90134E9E70020FFF7FAF9A6
:10A5A000FFF7FCF9074B00221A70FFF7E8BAF8BD75
:10A5B000FB1B0020801B0020CA1B0020E41B002086
:10A5C000041C00200F1100202DE9F04107468846A9
:10A5D00016460024B4420ED00025BD4205D04046A8
:10A5E0000135FAF77CFFEDB2F7E73C200134FAF7CA
:10A5F00076FFE4B2EEE7BDE8F08100000F4B1A6889
:10A6000042F00100186059680D4A0A405A60186803
:10A6100020F0847121F480321A60186820F48021BF
:10A6200019605A684FF41F0122F4FE0058609960C7
:10A63000044B4FF000629A60704700BF0010024068
:10A640000000FFF800ED00E0164A174B516801F0DA
:10A650000C00042803D0082805D0144801E0144950
:10A660000868186011E051685068C1F383410231F5
:10A67000C00301D40F4A06E052680D4812F4003FAF
:10A68000026818BF520851431960064B0A485A68BD
:10A69000054BC2F30311415C1A6822FA01F21A60F9
:10A6A000704700BF001002405001002000127A00E5
:10A6B0004C01002000093D003C0100201FB5002393
:10A6C0004F494FF4E01000930193029303900A68FE
:10A6D00042F480330B60886940F010028A61484B75
:10A6E000196801F400300190009A511C0091019802
:10A6F0001A4618B9009BB3F5A06FF0D11168404815
:10A7000011F4003201D0022216E0036843F0010187
:10A71000016000923A48026802F002030193009936
:10A720004A1C0092019B1BB90099B1F5A06FF1D1B1
:10A73000006883073CD50122324B0292196841F030
:10A74000100018601A6822F003011960186840F0C0
:10A7500002021A60A3F5805359685960586858601E
:10A760005A6842F48061284A5960106820F07041AC
:10A770001160264826490860586820F47C1058600B
:10A78000106840F000401060906820F40040906035
:10A79000043A9268100449BF1E4A4FF4E0120A605E
:10A7A0004FF48012039202991548012901D10AE061
:10A7B000FEE702290BD14268039B42EA030141F400
:10A7C0008032426003E0596841F460125A600368C5
:10A7D00043F0807101600A4802689201FBD543682A
:10A7E00023F003014160426842F002034360416884
:10A7F00001F00C02082AFAD1FFF726FF05B000BDD0
:10A8000000100240002002400410014000127A00B3
:10A810004C010020001BB70008B5154B98420BD126
:10A8200001214FF4805000F0C1FD4FF48050002111
:10A83000BDE8084000F0BABD0E49884207D14FF488
:10A840008040012100F0BEFD4FF4804009E00A4A3B
:10A8500090420BD14FF40040012100F0B3FD4FF4C2
:10A8600000400021BDE8084000F0ACBD08BD00BFBD
:10A870000030014000380040003C00400B8810B51B
:10A880004C88028823438C8802F441522343CC88AD
:10A8900023430C8923434C8923438C892343CC894C
:10A8A000098A23431A4393B20380828B22F4006304
:10A8B0001A04130C8383018210BD038819B199B265
:10A8C00041F0400303E023F040010A04130C03802D
:10A8D000704781817047808980B27047038919422F
:10A8E0000CBF002001207047426810B522F470238D
:10A8F0000A6823F4807444EA02030C7943EA0422D0
:10A900004260CB688A6884681A43084B234013432B
:10A910004A7943EA42038360097CC26A4B1E22F4EF
:10A920007002D9B242EA0152C26210BDFDF7F1FFD6
:10A93000836811B143F0010101E023F0010181605E
:10A940007047836811B143F4807101E023F4807192
:10A9500081607047836843F00801816070478068B8
:10A96000C0F3C0007047836843F004018160704702
:10A970008068C0F380007047836811B143F4A00180
:10A9800001E023F4A00181607047092970B54FF000
:10A9900003040CD94C4307251E3C05FA04F503FAC1
:10A9A00004F3C66826EA05052B43C3600BE04C435D
:10A9B000072505FA04F503FA04F3066926EA0505F6
:10A9C00045EA03040461062A4FF005030DD8013A55
:10A9D00053431F2202FA03F201FA03F1446B24EA03
:10A9E000020242EA0103436370BD0C2A0DD85343AF
:10A9F0001F22233B02FA03F201FA03F1046B24EA5B
:10AA0000020242EA0103036370BD53431F22413B2C
:10AA100002FA03F201FA03F1C46A24EA02021143C2
:10AA2000C16270BD40F0BF60024B40F40031D9609C
:10AA3000704700BF00ED00E0C37810B503B3164CBB
:10AA4000E168CB43C3F302244178C4F1040201FA64
:10AA500002F10F2222FA04F28478037822400A439A
:10AA6000110103F16043CAB203F5614181F800238B
:10AA70000078012200F01F03410902FA03F007E009
:10AA80000078012200F01F03410902FA03F020318F
:10AA9000024B43F8210010BD00ED00E000E100E0B2
:10AAA00030B5048C24F001052C04250C0584048B9E
:10AAB000A5B225F0F3052A4342EA0313114A048C98
:10AAC0009042A4B29DB215D002F50063984211D015
:10AAD000B0F1804F0ED0A3F5983290420AD002F523
:10AAE0008063984206D003F58062904218BF24F03C
:10AAF0000A0401D124F0020444F001042143058337
:10AB0000018430BD002C014030B5048C24F01005C8
:10AB10002C04250C0584048B058C24F44074240536
:10AB2000240D44EA022242EA0333144AADB29042B1
:10AB30009BB212D002F5006290420ED0B0F1804F6D
:10AB40000BD0A2F59832904207D002F58062904275
:10AB500003D002F58062904207D125F0200242F036
:10AB6000100545EA011189B204E025F0A00545F081
:10AB7000100529430383018430BD00BF002C014030
:10AB8000224A038890429BB212D002F500629042A2
:10AB90000ED0B0F1804F0BD0A2F59832904207D082
:10ABA00002F58062904203D002F58062904203D1A8
:10ABB0004A8823F070031343154A904208D002F5E7
:10ABC0008062904204D023F44073CA889BB213433E
:10ABD00003808B880A8883850C4B028598420FD0AE
:10ABE00003F5006290420BD002F54063984207D013
:10ABF00003F58062904203D002F58063984201D150
:10AC0000097A018601228282704700BF002C014030
:10AC100000100040038C70B523F001021404250CD1
:10AC20000584068C8388028B9CB222F073052B046A
:10AC30000D881A0C26F0020633042A434E880D892B
:10AC40001B0C3543ADB22B43134DA8420FD005F575
:10AC50000065A8420BD005F54065A84207D005F570
:10AC60008065A84203D005F58065A8420ED123F087
:10AC700008064B898D881E4326F004032B43CE899A
:10AC80008D8924F440743543ADB22C43C988848047
:10AC900002838186038470BD002C0140038C30B593
:10ACA00023F010021404250C0584038C8288048B85
:10ACB00023F0200324F4E6452C040D88240C44EAF8
:10ACC00005241D042B0C0D8992B243EA05134D880F
:10ACD000A4B243EA0513124D9BB2A84203D005F576
:10ACE0000065A84215D14D8923F080039BB243EA49
:10ACF00005134FF6BF751D408B8822F4406245EA6C
:10AD00000315ABB28D8942EA8502CD8942EA8502FC
:10AD100092B2C988828004830187038430BD00BF5A
:10AD2000002C0140038C30B523F480721404250CF0
:10AD30000584038C8288848B23F4007324F07305CC
:10AD40002C040D88240C2C431D042B0C0D8992B26D
:10AD500043EA05234D8843EA0523124D9BB2A842DE
:10AD600003D005F50065A84215D14D8923F4006391
:10AD70009BB243EA05234FF6FF351D408B8822F432
:10AD8000405245EA0325ABB28D8942EA0512CD89CE
:10AD900042EA051292B2C988828084838187038443
:10ADA00030BD00BF002C0140038C30B523F480522D
:10ADB0001404250C0584038C8288858B94B225F4B9
:10ADC000E64215042A0C0D8823F4005342EA0522BA
:10ADD0001D042B0C0D8992B243EA05334D8843EADA
:10ADE00005330A4D9BB2A84203D005F50065A84281
:10ADF00005D18D8924F4804444EA8514A4B2C9881D
:10AE000084808283A0F84010038430BD002C014070
:10AE100000214FF6FF7383800180C1804180017261
:10AE200070470023038043808380C3800381438174
:10AE30008381C38170470023012203804380828085
:10AE4000C38003817047038819B199B241F00103AF
:10AE500003E023F001010A04130C03807047B0F8EB
:10AE6000443029B16FEA43436FEA53418AB201E0AB
:10AE700059044A0CA0F84420704783899BB20AB158
:10AE8000194301E023EA010181817047038B23F01C
:10AE9000080213041A0C114301837047038B23F437
:10AEA000006213041A0C42EA01218BB2038370473B
:10AEB000838B23F0080213041A0C1143818370471B
:10AEC000838B23F4006213041A0C42EA01218BB233
:10AED0008383704781847047038B23F00C02130433
:10AEE0001A0C0283038B9AB2114301837047038BC0
:10AEF00023F4406213041A0C0283038B9AB242EAD1
:10AF000001218BB203837047838B23F00C0213045F
:10AF10001A0C8283838B9AB2114381837047838B8F
:10AF200023F4406213041A0C8283838B9AB242EAA0
:10AF300001218BB283837047F8B50B880D46044618
:10AF40004988AA8843B92B89FFF7AAFDE9882046DA
:10AF5000BDE8F840FFF7C0BF042B08D12B89FFF7ED
:10AF6000D3FDE9882046BDE8F840FFF7C0BF082BB5
:10AF70000E462F89008C3BD120F480731804030CFB
:10AF80002384A08B83B223F0F30343EA0717374BE4
:10AF9000208CBFB29C4280B247EA020212D003F575
:10AFA00000639C420ED0B4F1804F0BD0A3F59833D0
:10AFB0009C4207D003F580639C4203D003F5806375
:10AFC0009C4207D120F4007040EA06218BB243F482
:10AFD000807305E020F4206041F4807140EA0103B1
:10AFE000E9882046A2832384BDE8F840FFF78CBFA0
:10AFF00020F480531804030C2384A38B208C23F4A7
:10B0000040731B051B0D43EA022242EA0733174A2D
:10B0100080B294429BB212D002F5006294420ED0EC
:10B02000B4F1804F0BD0A2F59832944207D002F5CC
:10B030008062944203D002F58062944207D120F4EA
:10B04000005040EA063291B241F4805205E047F6E2
:10B05000FF52024041F480510A43E9882046A3830D
:10B060002284BDE8F840FFF75ABF00BF002C014022
:10B07000808E80B27047008F80B27047808F80B220
:10B080007047B0F8400080B27047038A828911EAA5
:10B09000030092B203D011420CBF00200120704780
:10B0A000C9438AB202827047038A30B50D4604460E
:10B0B000EA8898B220F4405111432182A38928895B
:10B0C000A98823F4B05340EA0102688923F00C01F7
:10B0D00002430804030C1A4391B2A181A08AAA89F1
:10B0E00083B223F4407187B01143A18201A800F01C
:10B0F000EBF81848A38984420CBF0498039819B24E
:10B1000000294FF019032A6803FB00F001DA51000F
:10B1100000E09100B0FBF1F16423B1FBF3F2120106
:10B12000100903FB1011A08900B2002806DAC9003B
:10B130003231B1FBF3F303F0070005E009013231CE
:10B14000B1FBF3F303F00F00024390B2208107B08C
:10B1500030BD00BF00380140838919B199B241F474
:10B16000005303E023F400510A04130C8381704759
:10B17000C1F3421310B5012401F01F01A34204FAE8
:10B1800001F101D10C3004E0022B01D1103000E0BC
:10B190001430036812B143EA010201E023EA01021C
:10B1A000026010BD838A9BB20AB1194301E023EA11
:10B1B0000101818270470000034A044B02F188308C
:10B1C0005A605860704700BF230167450020024065
:10B1D000024B1A6942F0800018617047002002405B
:10B1E000014BD860704700BF00200240084BDA686E
:10B1F000D20709D4D868400708D4D96811F0100FD5
:10B200000CBF0420032070470120704702207047C4
:10B210000020024010B50446FFF7E8FF012806D1E0
:10B220001CB1FFF7E3FF013CF8E7052010BD002C3F
:10B2300008BF052010BD000073B5002306464FF47B
:10B2400000500D460193FFF7E5FF04281AD10E4C7C
:10B25000AAB2206940F0010121614FF40050328010
:10B26000FFF7D8FF042808D102360196019B2D0C68
:10B270001D804FF40050FFF7CDFF216941F6FE72AB
:10B280000A4022617CBD00BF0020024038B505465F
:10B290004FF43020FFF7BEFF042812D1094C236978
:10B2A00043F002002061656121694FF4302041F0D4
:10B2B00040022261FFF7AEFF216941F6FD730B40AA
:10B2C000236138BD00200240204B10B55A6802F0BF
:10B2D0000C01042903D0082905D01D4B01E01D4CA9
:10B2E0002368036011E05C685968C4F38342941CCE
:10B2F000C90301D4184A06E016495B680A6813F4CA
:10B30000003F18BF520854430460104B5968C1F302
:10B31000031212498C5C026822FA04F242605C68F3
:10B32000C4F302240C5D22FA04F484605C68C4F364
:10B33000C224095D22FA01F2C2605B680849C3F3C6
:10B340008133CB5CB2FBF3F2026110BD001002400E
:10B3500000127A004C01002000093D005801002035
:10B3600054010020044B5A6909B1104301E022EA5C
:10B3700000005861704700BF00100240044B9A69FA
:10B3800009B1104301E022EA00009861704700BF54
:10B3900000100240044BDA6909B1104301E022EACF
:10B3A0000000D861704700BF00100240044BDA680B
:10B3B00009B1104301E022EA0000D860704700BFE5
:10B3C00000100240044B1A6909B1104301E022EA5F
:10B3D00000001861704700BF00100240024B5A6A1B
:10B3E00042F08070586270470010024008B50B4B65
:10B3F000984207D14FF400100121FFF7E3FF4FF40B
:10B40000001006E04FF480000121FFF7DBFF4FF44E
:10B4100080000021BDE80840FFF7D4BF0054004081
:10B42000F0B58688044687B026F03F000D4601043B
:10B4300001A80E0CFFF748FF2C4A0399B1FBF2F06C
:10B4400087B23E43A680238823F0010213041A0C1E
:10B4500022802B68264A93420AD85B00B1FBF3F0A6
:10B46000013783B2BFB22784032B98BF042320E0A7
:10B47000EE884BF6FF72964204D103225343B1FB90
:10B48000F3F305E019225343B1FBF3F141F4804398
:10B4900099B20A054FF4967208BF41F0010150437A
:10B4A00041F400434FF47A7190FBF1F0421C91B2E9
:10B4B0002184A383228891B241F001032380208854
:10B4C00020F4816222F002010B04AA886989180C19
:10B4D00041EA02032989AA89184380B241EA02039A
:10B4E000208098B2208107B0F0BD00BF40420F001D
:10B4F000A086010041F28833002103604BF6FF7201
:10B500004FF480438180C2800181418183817047F3
:10B51000038819B199B241F0010303E023F001015E
:10B520000A04130C03807047038819B199B241F4DF
:10B53000807303E023F480710A04130C03807047C6
:10B54000038819B199B241F4007303E023F4007148
:10B550000A04130C03807047038819B199B241F4AF
:10B56000806303E023F480610A04130C03807047B6
:10B5700083889BB20AB1194301E023EA010181806B
:10B58000704701827047008AC0B2704712B141F023
:10B59000010101E001F0FE010182704702684FF6EF
:10B5A000FE73134003602D4B0021984201604160FF
:10B5B0008160C16022D02A49884229D0294B984213
:10B5C00030D02949884237D0284B98423ED0284B6A
:10B5D000984206D153F8681C41F4700043F8680C97
:10B5E00070472449884206D151F87C0C40F07062C3
:10B5F00041F87C2C7047204B984206D153F8042C1C
:10B6000042F00F0143F8041C70471C49884206D1E0
:10B6100051F8183C43F0F00041F8180C7047184BF3
:10B62000984206D153F82C2C42F4706143F82C1C3C
:10B6300070471449884206D151F8403C43F47040A9
:10B6400041F8400C7047104B984205D153F8542CE8
:10B6500042F4702143F8541C704700BF08000240B8
:10B660001C000240300002404400024058000240EA
:10B670006C00024080000240080402401C040240AA
:10B6800030040240440402405804024070B5066889
:10B690008C680D6A26F4FF4222F070060A6945EABA
:10B6A00004034C6913438A692343CC6913431C4345
:10B6B0004B6A44EA03028B6A1A4332430260CB6846
:10B6C0000A68496843608260C16070BD00230360FE
:10B6D00043608360C360036143618361C36103624C
:10B6E00043628362704719B1016841F0010303E0CE
:10B6F00002684FF6FE7313400360704703680AB197
:10B70000194301E023EA010101607047416070477D
:10B71000406880B270470000C3004CBF014B024B31
:10B7200058607047000402400000024000B540F637
:10B73000D87320F00042C3F649739A4283B00146A1
:10B7400015DDB2F1FF4F03DBF5F72AF903B000BDB9
:10B75000694600F095FB00F00302012A0098019968
:10B760000ED0022A07D082B900F0A0FDEEE700213A
:10B7700000F09CFDEAE700F099FD00F10040E5E7EC
:10B7800001F040FC00F10040E0E7012201F03AFC4A
:10B79000DCE700BF30B5C0F3C754A4F17F031E2B14
:10B7A00083B0014621DC581C1DDBCD0F162B0CDDB0
:10B7B00021F07F4323F4000040F40000963C00FA9F
:10B7C00004F005B1404203B030BD114850F82540A7
:10B7D0002046F5F7E7F8019021460198F5F7E0F8E3
:10B7E00020F0004121B90020EDE7F5F7A9FBEAE7D9
:10B7F00020F07F4222F40003C0F3C75043F400015D
:10B80000C0F1960221FA02F0002DDCD0DAE700BF89
:10B810002C0A010800B540F6D87320F00042C3F6A8
:10B8200049739A4283B0014616DDB2F1FF4F03DB44
:10B83000F5F7B6F803B000BD694600F021FB00F053
:10B840000300012815D002280BD0B8B9009801993F
:10B85000012201F0D7FBEDE70021002201F0D2FB2D
:10B86000E8E700980199012201F0CCFB00F10040CB
:10B87000E0E70098019900F019FDDBE700980199D5
:10B8800000F014FD00F10040D4E700BF70B58AB0AD
:10B89000064600F09BF8224C054694F9003001332F
:10B8A00003D0304601F0B0FD10B928460AB070BD93
:10B8B000304601F05BFD4FF07E51F5F737FB002875
:10B8C000F3D0184A012100253046019200910895D5
:10B8D000F4F7ACFD02460B461348CDE90423CDE94D
:10B8E000022301F011FC94F90030CDE90601022B8E
:10B8F0000BD0684601F006FC38B1089850B9DDE974
:10B900000601F4F7F9FF0546CFE701F089FE212192
:10B910000160F2E701F084FE089A0260EFE700BFE1
:10B9200068010020340A01083C0A010800F002BA4C
:10B9300070B58AB0054600F04FFC224C064694F9DB
:10B940000030013308D0284601F05EFD20B12846C2
:10B950000021F5F7CDFA10B930460AB070BD1A4A89
:10B96000012128460026009101920896F4F75EFD19
:10B970002478CDE90401CDE902017CB9002200233D
:10B98000CDE90623684601F0BDFB88B10898A0B94F
:10B99000DDE90601F4F7B0FF0646DDE700200021EF
:10B9A00002460B46F4F7C0FE022CCDE90601E9D1B0
:10B9B00001F036FE21230360E8E701F031FE08992B
:10B9C0000160E5E768010020400A0108F8B520F0B1
:10B9D0000043B3F17E5F044613D00BDCB3F17C5F10
:10B9E00014DAB3F10C5F00F3A48040F6DB70C3F609
:10B9F000C970F8BD0146F4F7D3FF0146F5F78EF99B
:10BA0000F8BD002840F30E810020F8BD0028C0F2E8
:10BA10000E8101464FF07E50F4F7C2FF4FF07C518B
:10BA2000F5F7C8F8044600F0D7FB4EF60871064655
:10BA300020F47F65C3F611012046F5F7BBF847F601
:10BA40000471C3F64F21F4F7ADFF2146F5F7B2F8C4
:10BA500041F24611C3F62451F4F7A2FF2146F5F74F
:10BA6000A9F840F6A821C3F64E61F4F79BFF2146E2
:10BA7000F5F7A0F84BF29001C3F6A661F4F790FF3A
:10BA80002146F5F797F84AF6AB21C3F62A61F4F799
:10BA900089FF2146F5F78EF84CF22E610746C3F672
:10BAA0009D512046F5F786F843F26131C3F63071B7
:10BAB000F4F776FF2146F5F77DF845F22D71C4F2D3
:10BAC0000101F4F76FFF2146F5F774F84DF23911D3
:10BAD000C4F21901F4F764FF2146F5F76BF84FF053
:10BAE0007E51F4F75FFF01463846F5F717F9314606
:10BAF000F5F760F825F00F05074629462846F5F7C3
:10BB000059F801462046F4F74BFF294604463046D3
:10BB1000F4F748FF01462046F5F700F9014638469C
:10BB2000F4F740FF2946F4F73DFF0146F4F73AFFEA
:10BB3000F8BD0146F5F73EF84EF60871C3F611015F
:10BB40000546F5F737F847F60471C3F64F21F4F7C9
:10BB500029FF2946F5F72EF841F24611C3F6245184
:10BB6000F4F71EFF2946F5F725F840F6A821C3F69D
:10BB70004E61F4F717FF2946F5F71CF84BF29001D8
:10BB8000C3F6A661F4F70CFF2946F5F713F84AF659
:10BB9000AB21C3F62A61F4F705FF2946F5F70AF849
:10BBA0004CF22E610646C3F69D512846F5F702F881
:10BBB00043F26131C3F63071F4F7F2FE2946F4F72F
:10BBC000F9FF45F22D71C4F20101F4F7EBFE2946AD
:10BBD000F4F7F0FF4DF23911C4F21901F4F7E0FE69
:10BBE0002946F4F7E7FF4FF07E51F4F7DBFE0146FC
:10BBF0003046F5F793F801462046F4F7DBFF01469F
:10BC000042F26810C3F2A230F4F7CAFE01462046A1
:10BC1000F4F7C6FE014640F6DA70C3F6C970F4F7D1
:10BC2000BFFEF8BD40F6DB70C4F24900F8BD4FF02E
:10BC30007E51F4F7B7FE4FF07C51F4F7BBFF4EF6A0
:10BC40000871C3F611010446F4F7B4FF47F6047116
:10BC5000C3F64F21F4F7A6FE2146F4F7ABFF41F2FD
:10BC60004611C3F62451F4F79BFE2146F4F7A2FFD8
:10BC700040F6A821C3F64E61F4F794FE2146F4F78E
:10BC800099FF4BF29001C3F6A661F4F789FE2146B5
:10BC9000F4F790FF4AF6AB21C3F62A61F4F782FE6F
:10BCA0002146F4F787FF0646204600F095FA4CF24D
:10BCB0002E610546C3F69D512046F4F77BFF43F203
:10BCC0006131C3F63071F4F76BFE2146F4F772FF71
:10BCD00045F22D71C4F20101F4F764FE2146F4F738
:10BCE00069FF4DF23911C4F21901F4F759FE2146EA
:10BCF000F4F760FF4FF07E51F4F754FE01463046F2
:10BD0000F5F70CF82946F4F755FF42F26811C3F233
:10BD1000A231F4F745FE01462846F4F743FE0146FA
:10BD2000F4F740FE014640F6DA70C4F24900F4F739
:10BD300037FEF8BDF8B521F00044B4F1FF4F0346DB
:10BD400017DC20F00045B5F1FF4F064611DCB1F1DC
:10BD50007E5F42D08F1707F0020040EAD37775B9B3
:10BD6000022F35D0032F08D140F6DB73CCF2490304
:10BD700003E01846F4F716FE03461846F8BDD4B1A2
:10BD8000B4F1FF4F2DD0B5F1FF4F14D02C1BE415AB
:10BD90003C2C18DC002952DB1846F4F7BFFF01F0F9
:10BDA000E5FA01F0B7F9012F46D0022F35D0002F68
:10BDB00025D10346E1E7002E40F6DB731CDBC3F61A
:10BDC000C9731846F8BD40F6DB70C3F6C970EAE7E0
:10BDD00040F6DB73C4F24903CFE7BDE8F84001F059
:10BDE00099B9B5F1FF4F2FD0022FF1D0032FBBD05F
:10BDF000012F34D00023C0E7CBF6C973BDE74BF663
:10BE00002E51C3F2BB31F4F7CDFD40F6DB71C4F225
:10BE10004901F4F7C5FD0346AFE74BF62E51C3F2D7
:10BE2000BB31F4F7BFFD014640F6DB70C4F24900B8
:10BE3000F4F7B6FD0346A0E700F100439DE714F1D7
:10BE40003C0FA9DA0020AEE7022F13D0032F0CD04D
:10BE5000012F40F6DB7305D0C3F649738DE74FF031
:10BE600000438AE7CBF6497387E74CF6E433CCF21C
:10BE7000160382E74CF6E433C4F216037DE700BFF5
:10BE80002DE9F04F40F6D87320F00044C3F6497313
:10BE90009C4289B006460D4640F38B804CF6E33158
:10BEA000C4F216018C4226DC4FF478610028C3F6F8
:10BEB000C97140F32B81F4F773FD4FF47D6224F0D8
:10BEC0000F04C3F6C9729442064600F0818044F222
:10BED0004341C3F23571F4F763FD014628603046F3
:10BEE000F4F75EFD44F24341C3F23571F4F758FDB7
:10BEF0000127686061E04FF47867C4F24937BC42BB
:10BF000040F38180B4F1FF4F5BDA4FEAE459A9F1C5
:10BF10008609A4EBC9542046F5F712F8F4F7F6FDAC
:10BF20000246014620460592F4F73AFD4FF087415C
:10BF3000F4F740FE0746F5F703F8F4F7E7FD01468E
:10BF4000044638460694F4F72BFD4FF08741F4F78A
:10BF500031FE00210790F4F7C1FF002800F0F680C1
:10BF60000327204600210DF11808013FF4F7B6FF22
:10BF700040B158F8044D00212046013FF4F7AEFFD0
:10BF80000028F6D1924B02200090019305A83B4671
:10BF900029464A4600F066FA002E07460DDA95E873
:10BFA0000C0002F1004103F1004229606A6047423F
:10BFB00003E00023286000274B60384609B0BDE845
:10BFC000F08F0146F4F7ECFC002768602860F4E786
:10BFD0004FF48841C3F23571F4F7E2FC4AF20831BC
:10BFE000C2F685610446F4F7DBFC01462860204672
:10BFF000F4F7D6FC4AF20831C2F68561F4F7D0FCBA
:10C0000001276860D9E701F0B1F94FF68411C3F652
:10C0100022718046F4F7CEFD4FF07C51F4F7C2FC5C
:10C02000F4F78EFF0746F4F771FD4FF47861C3F61D
:10C03000C9718346F4F7BEFD01464046F4F7B0FCF3
:10C0400044F243418146C3F235715846F4F7B2FDDC
:10C050001F2F8246514648461FDC5E4B7A1E53F81E
:10C06000223024F0FF029A4217D0F4F799FC804660
:10C07000C5F8008041464846F4F792FC5146F4F773
:10C080008FFC002E686098DA08F1004800F100414A
:10C09000C5F8008069607F428FE7F4F781FCE31503
:10C0A0008046C0F3C750191A0829E1DD4FF48841D2
:10C0B000C3F2357158460393F4F77CFD824651462E
:10C0C0004846F4F76DFC044621464846F4F768FC00
:10C0D0005146F4F765FC4AF208318146C2F68561A3
:10C0E0005846F4F767FD4946F4F75AFC8246514634
:10C0F0002046F4F755FC039BC0F3C7528046981ABC
:10C10000192841DCC5F80080A146B3E7F4F74AFCE2
:10C110004FF47D6724F00F04C3F6C977BC4206468E
:10C1200016D044F24341C3F23571F4F73BFC0146AB
:10C1300028603046F4F734FC44F24341C3F23571D1
:10C14000F4F730FC4FF0FF37686036E7032719E754
:10C150004FF48841C3F23571F4F724FC4AF20831F8
:10C16000C2F685610446F4F71DFC014628602046AE
:10C17000F4F716FC4AF20831C2F68561F4F712FCB6
:10C180004FF0FF37686018E74FF42341C2F685612E
:10C190005846F4F70FFD804641462046F4F700FC70
:10C1A000814649462046F4F7FBFB4146F4F7F8FB8D
:10C1B00043F232110446C2F28D415846F4F7FAFCBC
:10C1C0002146F4F7EDFB8246514648464DE700BF55
:10C1D000C80A0108480A010820F00042B2F1FF4FE6
:10C1E000F8B50446034646D2002A42D0002852DB66
:10C1F000C415B2F5000F09D210F4000553D15B004D
:10C2000001351902FBD5C5F10100241823F07F4147
:10C210007F3C21F40006E20746F4000048BF4000DE
:10C2200043004FF08072002760109A423C462CDD9C
:10C230005B004FF400021825A61851089E4205F134
:10C24000FF3502DCB4189B1BBF185B0062189A42D2
:10C2500002DC9B1A54187F185B004A08013DEBD1A1
:10C2600013B107F001017F187C1004F17C5303EB3C
:10C27000C0542046F8BD0146F4F79CFC0146204618
:10C28000F4F790FB04462046F8BD4FF0007403F12C
:10C290007F431746CCE70146F4F782FB0146F4F7EB
:10C2A0003DFD0446E5E70120AFE700BF2DE9F84377
:10C2B00020F00046B6F1485F05460F465BDAF4F71A
:10C2C0003FFE002800F0CA8029462846F4F772FC99
:10C2D0004DF24E71CAF647510446F4F76BFC47F233
:10C2E000F641C3F20F11F4F75DFB2146F4F762FC4F
:10C2F0004FF27C21C3F29341F4F752FB2146F4F74D
:10C3000059FC40F60151C3F2D071F4F74BFB2146C2
:10C31000F4F750FC40F66131C3F6B621F4F740FB68
:10C320002146F4F747FC4AF6AB21C3F62A51F4F74D
:10C3300039FB2146F4F73EFC804620464FF07C5105
:10C34000F4F738FC414606462046F4F733FC3946FC
:10C3500004462846F4F72EFC01462046F4F720FB5D
:10C3600001463046F4F71CFB01464FF07E50F4F7CF
:10C3700017FBBDE8F8830146F4F71CFC4DF24E7143
:10C38000CAF647510446F4F715FC47F2F641C3F2EA
:10C390000F11F4F707FB2146F4F70CFC4FF27C2158
:10C3A000C3F29341F4F7FCFA2146F4F703FC40F69C
:10C3B0000151C3F2D071F4F7F5FA2146F4F7FAFB14
:10C3C00040F66131C3F6B621F4F7EAFA2146F4F7F4
:10C3D000F1FB4AF6AB21C3F62A51F4F7E3FA214602
:10C3E000F4F7E8FB49F69913C3F699639E42804639
:10C3F000A3DD0020C3F64870864227DC06F17F46A5
:10C400004FF07E503146F4F7CBFA814620464FF08C
:10C410007C51F4F7CFFB3146F4F7C2FA41460646A9
:10C420002046F4F7C7FB394604462846F4F7C2FB1A
:10C4300001462046F4F7B4FA01463046F4F7B0FA64
:10C4400001464846F4F7ACFABDE8F8834FF000091E
:10C450000026C3F63879C3F69066D7E74FF07E50D2
:10C46000BDE8F8832DE9F04FDFB00C930C9D224B13
:10C47000689C0A91691ED61E48BF161D834653F854
:10C480002400F71027EAE7730890049104980D93AD
:10C49000089DDC43DDF834C002EBC4024119079269
:10C4A000C0EB0C0750D47E18699BC7EB0609013618
:10C4B000002F03EB870522AC09F0010AC0F2FE82CF
:10C4C0002868F4F723FB0137B74220604FF00408D7
:10C4D0003AD0BAF1000F26D0002FC0F2F18255F801
:10C4E0000800F4F713FB0137B74244F8080008F1DD
:10C4F000040818D128E000BFE00D010855F8080035
:10C50000F4F704FB013708F1040944F8080013D4D8
:10C5100055F80900F4F7FAFA0137B74244F8090070
:10C5200009F1040810D0002FE8DA0020013708F1E3
:10C53000040944F80800EBD501370020B74244F85D
:10C54000090009F10408EED1089A002AC0F24585D5
:10C5500008990C9E8D004AAB5C19039549AF029473
:10C560004FEA860A049A002AC0F296820DF18808E2
:10C5700008EB860555F8041CAAF10403DBF800005B
:10C58000C3F38009F4F716FB01460020F4F70AFA1A
:10C590000424043D544580462BD0B9F1000F0DD042
:10C5A00055F8041DDBF80400F4F704FB014640468F
:10C5B000F4F7F8F90824544580461AD055F8041CBD
:10C5C0005BF80400F4F7F6FA01464046F4F7EAF99E
:10C5D0000434804655F8081C5BF80400F4F7EAFAC6
:10C5E00001464046F4F7DEF90434083D54458046E0
:10C5F000E4D1029847F8048F01368742B2D1039FF5
:10C600000EA9CE190996089EB2005EAB9D18002EA9
:10C61000029255F8509C7DDD0DF5947C4FF06E51E3
:10C6200048460DACA7180CEB0205F4F7C3FAF4F773
:10C6300087FCF4F76BFA4FF087410190F4F7BAFAF0
:10C6400001464846F4F7ACF9F4F77AFC0EAC2060EA
:10C650000198014655F8040DF4F7A4F9BC4281464F
:10C66000C7F3800156D0E9B14FF06E51F4F7A2FA4A
:10C67000F4F766FCF4F74AFA4FF087410190F4F7BB
:10C6800099FA01464846F4F78BF9F4F759FC019AF8
:10C690000FAC2060114655F8040DF4F783F9BC4245
:10C6A000814637D04FF06E514846F4F783FAF4F7DD
:10C6B00047FCF4F72BFA4FF087418046F4F77AFAFB
:10C6C00001464846F4F76CF9F4F73AFC41466060DD
:10C6D00055F8040DF4F766F94FF06E518146F4F702
:10C6E00069FAF4F72DFCF4F711FA4FF08741804610
:10C6F000F4F760FA01464846F4F752F9F4F720FCE3
:10C700004146A06055F8040DF4F74CF90834BC42DA
:10C710008146C7D10799484600F0A2FE4FF07851F4
:10C720000546F4F747FA00F025FE4FF08241F4F792
:10C7300041FA01462846F4F733F90746F4F700FCBE
:10C740008146F4F7E3F901463846F4F729F90799E9
:10C750000746002940F33981721E0EAC079D54F83C
:10C760002230C5F1080043FA00F101FA00F0C5F1EA
:10C7700007041B1A43FA04F40DF1380C89444CF8F1
:10C780002230002C55DD002E09F1010940F394817F
:10C79000029D0EABDDF808C053F8042B281F0DF1E5
:10C7A000380E00250EEB0C01C0F3800022B1C2F55B
:10C7B000807243F8042C01258B4226D060B10F9A79
:10C7C0000433002D40F0F38022B1C2F5807543F8A8
:10C7D000045C01258B4218D053F8042B002D40F047
:10C7E000EC80C2F5807012B143F8040C012553F8B7
:10C7F000042B002D40F0DB80C2F58070002AE9D0C8
:10C8000001258B4243F8040CE6D1079900290DDD80
:10C81000012900F0E280022908D1701E0DF1380EC6
:10C820005EF8202002F03F034EF82030022C00F08A
:10C83000E08038460021F4F751FB002800F0F38037
:10C840000898751EA84225DC029B0DF1380E0EEBF0
:10C8500003010B46DDF824C053F8042DCCEB010096
:10C86000011F6345C1F3800011D030B153F8041D9E
:10C87000DDF824E00A43734509D0099F53F8040DFD
:10C8800053F8041D0243BB4242EA0102F6D1002ADA
:10C8900040F01A81089F0EAD781E55F82020002A1E
:10C8A00040F0108105EB8004012354F8041D01338E
:10C8B0000029FAD0F018771C87420B9075DCDDF860
:10C8C00010E00D9D0B9B0C9C0EEB0702DDF808C0E1
:10C8D000699F991B06EB05094AA8A61922AB07EB2D
:10C8E000890900EB0C05571C8A0003EB86010295B1
:10C8F00006920591002659F8040FF4F707F9059CF4
:10C90000A051049800285EDB22AD05EB8702AAF156
:10C910000403C3F3800452F8041CDBF80000039402
:10C92000141FF4F747F901460020F4F73BF84FF0E5
:10C930000408D04505462DD0039971B154F8041D63
:10C94000DBF80400F4F736F901462846F4F72AF834
:10C950004FF00808D04505461CD054F8041C5BF87D
:10C960000800F4F727F901462846F4F71BF808F108
:10C970000408054654F8081C5BF80800F4F71AF997
:10C9800001462846F4F70EF808F10408083CD045A3
:10C990000546E2D1DDF808E0069804364EF8045F5B
:10C9A00001378642CDF808E0A5D10B9E2CE6C2F1F6
:10C9B000FF0243F8042C01250CE7C2F1FF0543F800
:10C9C000045C012513E70025E4E75ED1701E0DF13C
:10C9D000380E5EF820301C12D3E6711E0DF1380CB3
:10C9E0005CF82100022C00F07F024CF821207FF43B
:10C9F00020AF39464FF07E50F3F7D2FF0746002DA7
:10CA00003FF417AF07994FF07E5000F029FD014623
:10CA10003846F3F7C5FF074638460021F4F75EFABB
:10CA200000287FF40DAF0294079C38466142CDF890
:10CA3000109000F015FD4FF087410546F4F76CFAB1
:10CA4000002800F0D2824FF06E512846F4F7B2F879
:10CA5000F4F776FAF4F75AF84FF087410746F4F7FF
:10CA6000A9F801462846F3F79BFFF4F769FA0EA9E7
:10CA700041F826003846F4F763FA079A013608327F
:10CA80000EAC079244F8260034E04FF07C51F4F7E6
:10CA900043FA58B90024CCE64FF00008029847F852
:10CAA000048F013687427FF45DADA8E50224002E95
:10CAB00009F101093FF76CAE0025A6E6002002E56A
:10CAC000002010E50123F5E6079A0EAE56F8253052
:10CAD000083ACDF8109002940792002B40F08E8215
:10CAE00006EB85042E4654F8045D013E083A002DFD
:10CAF000F9D007924FF07E50079900F0B1FC002E5C
:10CB00000446C0F2AC804FEA860AC6EB867B0EAFC5
:10CB10004FEA8B095744C9F100034AA9386801EB71
:10CB20000A08C3F3800BF3F7F1FF2146F4F742F84C
:10CB30004FF06E51C8F800002046F4F73BF8A9F119
:10CB400004096FF0030ACA45054631D0BBF1000F56
:10CB50000BD057F8040CF3F7D9FF2946F4F72AF85D
:10CB60006FF0070A48F8040C1AE057F80A00F3F7C8
:10CB7000CDFF2946F4F71EF84FF06E5148F80A0031
:10CB80002846F4F717F8AAF1040405463859F3F7D4
:10CB9000BDFF2946F4F70EF8AAF1080A48F8040088
:10CBA00028464FF06E51F4F705F8CA450546DCD12A
:10CBB000701CDFF84C94DDF820A003900027059648
:10CBC000BAF1000FC0F20582002FC0F202820026E7
:10CBD00000241AF0010F354620D0D8F80010D9F8FB
:10CBE0000000F3F7E7FF01462046F3F7DBFE0125DF
:10CBF000AA45044626DB0426BD420FDD22E0BB45E4
:10CC000020DC58F8021059F80200F3F7D3FF014670
:10CC10002046F3F7C7FEBD42044613DC58F8061061
:10CC200059F80600F3F7C6FF01462046F3F7BAFEAF
:10CC300005F1010B06F104020235DA45044602F162
:10CC40000406DCDA5EABDDF80CC003EB87010137CC
:10CC5000674541F8A04CA8F10408B1D1059E689C35
:10CC6000032C16D8DFE814F085011F011F011B00FB
:10CC700000230299002900F00B81379C369804F1BB
:10CC800000420A9C00F1004503F100432560626008
:10CC9000A360049D05F007005FB0BDE8F08F002E93
:10CCA000E6DD06F1FF3836AF07EB88094D4655F84B
:10CCB00004290DF1D40AD5F808B01046594601925E
:10CCC000F3F770FE804641460198F3F769FE01468E
:10CCD0005846F3F767FE5545C9F38003A860C5F8C9
:10CCE000048044D0BBB155F80429D5F808B01046EB
:10CCF00059460192F3F756FE01998046084641468F
:10CD0000F3F74EFE01465846F3F74CFE5545C5F87D
:10CD10000480A8602BD02C4654F80439D4F808B00D
:10CD2000184659460193F3F73DFE80464146019867
:10CD3000F3F736FE01465846F3F734FEC4F8048094
:10CD4000A06055F804BC251FD5F808805846414618
:10CD5000F3F728FE044621465846F3F721FE014624
:10CD60004046F3F71FFE55456C60A860D3D1012EF5
:10CD70007FF77EAF4D4655F804B9C7EB090ED5F8DD
:10CD800008A058465146AEF10409F3F70BFE804661
:10CD900041465846F3F704FE01465046F3F702FEBB
:10CDA000BD42C9F38009C5F80480A86043D0B9F139
:10CDB000000F15D055F804A9D5F8089050464946FB
:10CDC000F3F7F0FD804641465046F3F7E9FD014692
:10CDD0004846F3F7E7FDBD42C5F80480A8602AD0B5
:10CDE0002C4654F804A9D4F8089050464946F3F765
:10CDF000D9FD804641465046F3F7D2FD01464846EC
:10CE0000F3F7D0FDC4F80480A06055F8049C251FFA
:10CE1000D5F8088048464146F3F7C4FD044621464C
:10CE20004846F3F7BDFD01464046F3F7BBFDBD4262
:10CE30006C60A860D4D1013607EB860708353E4602
:10CE40007A1B131F56F8041D0020C3F38007F3F765
:10CE5000A9FDAE4203463FF40CAF3FB156F8041DA6
:10CE6000F3F7A0FDAE4203463FF403AF184656F871
:10CE7000041C341FF3F796FD083E54F8041CF3F726
:10CE800091FDAE42F3D10299034600297FF4F5AE3D
:10CE9000DDF828C036993798CCF80010CCF804009B
:10CEA000CCF80830F5E60023002E29DB36AF751CE0
:10CEB00007EB85042546E21B55F8041DA2F1040E7C
:10CEC0000020CEF38008F3F76DFDBD42034617D076
:10CED000B8F1000F06D055F8041DF3F763FDBD420D
:10CEE00003460DD0184655F8041C2C1FF3F75AFDC5
:10CEF000083D54F8041CF3F755FDBD42F3D1034639
:10CF00000299002967D003F10040DDF828C01946D6
:10CF1000CCF800003698F3F743FD002E034621DDE0
:10CF200036AF07EB8606F51B2A1F3799C2F3800739
:10CF3000F3F738FD37ACB442034613D037B161681C
:10CF4000F3F730FD38ACB44203460BD0184654F822
:10CF5000041FF3F727FD54F8041FF3F723FDB44231
:10CF6000F5D10346029909B103F100430A9C6360BD
:10CF70008FE6002E40DB36AF013607EB8600054614
:10CF8000C21B55F8041D0020141FF3F70BFDBD4212
:10CF9000C4F38006034615D036B155F8041DF3F7E7
:10CFA00001FDBD4203460DD0184655F8041C2C1F48
:10CFB000F3F7F8FC083D54F8041CF3F7F3FCBD420A
:10CFC000F3D10346029909B103F100430A9C23609F
:10CFD0005FE6002436E6184697E7DDF830E090007B
:10CFE00003904FEA8E0AFFF70ABB2846F3F7A8FF23
:10CFF0000EAB43F826007DE50023E3E72E4679E5F6
:10D00000EC0D01082DE9F84320F00043B3F1485F2F
:10D0100004460F46904603DAF3F792FF002859D0F2
:10D0200021462046F3F7C6FD21460546F3F7C2FD2B
:10D030004CF6D311C2F62E7106462846F3F7BAFD18
:10D0400042F63471C3F2D721F3F7AAFC2946F3F76D
:10D05000B1FD4EF61B71C3F23861F3F7A3FC29460C
:10D06000F3F7A8FD40F60151C3F65011F3F798FC11
:10D070002946F3F79FFD48F68901C3F60841F3F707
:10D0800091FC8146B8F1000F27D04FF07C51384613
:10D09000F3F790FD494680463046F3F78BFD014695
:10D0A0004046F3F77DFC2946F3F784FD3946F3F754
:10D0B00077FC4AF6AB210546C3F62A613046F3F702
:10D0C00079FD01462846F3F76DFC01462046F3F74B
:10D0D00067FC04462046BDE8F88301462846F3F77E
:10D0E00069FD4AF6AB21C3F62A61F3F759FC3146D4
:10D0F000F3F760FD01462046F3F754FC0446204652
:10D10000BDE8F8830020704700210020C7F6F871C1
:10D11000704700BF2DE9F04120F00045B5F1A14F67
:10D12000044606460DDBB5F1FF4F00F39C80002856
:10D1300040F6DB7440F3D480C3F6C9742046BDE8E2
:10D14000F0814FF6FF73C3F6DF639D4200F3A280C8
:10D15000B5F1445FC0F28E804FF0FF372146204684
:10D16000F3F728FD01468046F3F724FD46F6D71174
:10D17000C3F685410546F3F71DFD4DF65921C3F66B
:10D180004B51F3F70FFC2946F3F714FD46F6353102
:10D19000C3F68851F3F706FC2946F3F70BFD42F678
:10D1A0006E61C3F6BA51F3F7FDFB2946F3F702FDB2
:10D1B00044F62511C3F61261F3F7F4FB2946F3F7A1
:10D1C000F9FC4AF6AB21C3F6AA61F3F7EBFB414643
:10D1D000F3F7F0FC4AF221218046CBF615512846A0
:10D1E000F3F7E8FC4FF26B11C3F66E51F3F7D8FB7F
:10D1F0002946F3F7DFFC48F29571C3F69D51F3F72A
:10D20000CFFB2946F3F7D6FC48F63861C3F6E35165
:10D21000F3F7C6FB2946F3F7CDFC4CF6CD41C3F638
:10D220004C61F3F7BDFB2946F3F7C4FC7B1C0146B8
:10D23000404658D0F3F7B6FB2146F3F7BBFC494B09
:10D2400053F82710F3F7ACFB2146F3F7A9FB01468F
:10D25000454850F82700F3F7A3FB002E3DDB0446BA
:10D260002046BDE8F0810146F3F79CFB04462046CA
:10D27000BDE8F0814FF2CA21C7F24911F3F792FBE2
:10D280004FF07E51F3F752FE00283FF465AF204681
:10D29000BDE8F08100F06AF84FF6FF71C3F69771B0
:10D2A0008D4204464FF6FF7228DCC3F62F7295427A
:10D2B00046DC0146F3F776FB4FF07E51F3F770FB47
:10D2C0004FF0804105462046F3F76CFB01462846A7
:10D2D000F3F724FD0027044640E700F100442DE762
:10D2E000CBF6C9742AE7F3F75DFB2146F3F762FC3E
:10D2F00001462046F3F754FB04461FE7C4F21B0225
:10D30000954214DC4FF07F51F3F74AFB4FF07F5109
:10D3100005462046F3F74EFC4FF07E51F3F742FBF3
:10D3200001462846F3F7FAFC0227044616E70020D8
:10D330002146CBF68070F3F7F1FC032704460DE796
:10D340004FF07E51F3F72CFB4FF07E5107462046FD
:10D35000F3F728FB01463846F3F7E0FC01270446C3
:10D36000FCE600BF180E0108280E010820F000405E
:10D37000704700BFF8B520F00046F50D7F3D162D33
:10D38000014604461BDC002D074620DB4FF6FF73E9
:10D39000C0F27F0343FA05F606420ED04FF2CA21CF
:10D3A000C7F24911F3F7FEFA0021F3F7BFFD18B1F8
:10D3B000002C1BDB27EA060421460846F8BDB6F11F
:10D3C000FF4FFAD3F3F7EEFA01460846F8BD4FF2E5
:10D3D000CA21C7F24911F3F7E5FA0021F3F7A6FDD8
:10D3E0000028E9D0002C07DB0024E5E74FF400001B
:10D3F00040FA05F56719DDE70021CBF68071002EB4
:10D4000018BF0C46D8E700BF08B902207047B0F13A
:10D41000004FFAD0A0F500026FF001439A4201D804
:10D420000420704700F1FF419942F9D94FF6FE738D
:10D43000421EC0F27F039A4201D80320704700F1D8
:10D4400000414A1E9A42F8D9B0F1FF4F05D010F5BD
:10D45000000F14BF0020012070470120704700BF5B
:10D4600038B530F00044034602460D460FD0B4F103
:10D47000FF4F0ED2B4F5000F11D3E40D6419FE2C4A
:10D4800033DC002C1BDD22F0FF4141EAC453184677
:10D4900038BD0146F3F786FA0346184638BD4FF00B
:10D4A0009841F3F787FB43F6B041CFF6FF718D4209
:10D4B000034612DBC0F3C7540246193CDEE714F101
:10D4C000160F21DA4CF25032954219460EDC44F226
:10D4D0006020C0F6A25000F023F844F26021C0F6AC
:10D4E000A251F3F767FB0346D1E719464FF2CA2072
:10D4F000C7F2491000F014F84FF2CA21C7F24911DF
:10D50000F3F758FB0346C2E722F0FF4304F119008A
:10D5100043EAC0504FF04C51F3F74CFB0346B6E7DB
:10D5200001F0004120F00040084370472DE9F04130
:10D53000274C84B025680746D5F84841002C41D0D7
:10D5400066681F2E1CDD234810B94FF0FF301FE026
:10D550004FF4C870039102920193AFF300800399D6
:10D560000446029A019B0028EFD0D5F848610020BC
:10D5700060602660C5F84841C4F88801C4F88C0191
:10D58000656847B9A81C013544F820106560002083
:10D5900004B0BDE8F081012000FA05F0D4F88861FC
:10D5A00004EB85080643022FC8F88820C4F8886178
:10D5B000C8F80831E6D1D4F88C3143EA0002C4F847
:10D5C0008C21DFE705F5A674C5F84841B8E700BF30
:10D5D000400F01080000000000210A2201F028B8D5
:10D5E0002DE9F84FDDF828B081468A4698469AB171
:10D5F00093B11646002503E00FD0651CAE420BD94F
:10D600007419640808FB04A748463946D84700281F
:10D61000F2DA2646AE42F3D800273846BDE8F88F46
:10D6200040F29853C2F2000318687047114B124A37
:10D6300070B5981A831018D0591E02EB83040D465A
:10D6400054F8042D01F00106904775B126B154F845
:10D65000040D8047013D08D054F8043D9847013D32
:10D6600054F8041D8847013DF6D1BDE8704003F031
:10D670006FBC00BF680F0108640F0108F8B5204FA8
:10D68000204C381B871017D07A1E2368012502F022
:10D6900001069847AF420FD02EB154F8041F02255F
:10D6A0008847AF4208D0606880470235A268261DCF
:10D6B00090470834AF42F6D1134F144C03F042FCAC
:10D6C0003B1B9F1018D07D1E216805F00106012527
:10D6D0008847AF4211D02EB154F8040F022580477D
:10D6E000AF420BD0626890470235A368261D984769
:10D6F0000834AF42F6D1F8BDF8BDF8BDF8BD00BFA3
:10D700005C0F01085C0F0108640F01085C0F010841
:10D710000F2A2DE9F00340F2A18041EA00039B07A4
:10D7200040F09E800C68A2F1100504604B68AC4686
:10D7300043608C68BCF10F0F8460CC68C5F30015A2
:10D74000C46000F1100301F110042BD975B12568F4
:10D75000ACF1100C1D6065685D60A5689D60E568B2
:10D760001034DD601033BCF10F0F1BD9276804F1B2
:10D7700010061F60676803F110055F60A768ACF1D1
:10D78000200C9F60E768DF6024691C61776806F100
:10D7900010046F60B7682033AF60F668BCF10F0FFC
:10D7A000EE60E3D8A2F1100828F00F0302F00F0496
:10D7B00003F1100C032C00EB0C0301EB0C0851D906
:10D7C000211F4FEA9109444608EB890C54F8046B79
:10D7D000C8EB0C010CF1040C1D46644545F8046BC4
:10D7E000C1F3800112D029B154F8041B644545F8F7
:10D7F000041B0BD0274657F8041B2E4646F8041B83
:10D8000064686C603C1D351D6445F3D109F1010C61
:10D810004FEA8C0902F0030208EB09014B44D2B134
:10D820000D789A18DC4303F8015B1419934204F055
:10D83000010410D02CB111F8014F03F8014B9342B1
:10D8400009D04D781C4604F8015B8D7802315D707B
:10D85000631C9342F5D1BDE8F00370470346DEE751
:10D860000346DDE741462246D9E700BFF0B484070E
:10D87000034600F08D80541E002A00F08780E507E3
:10D88000CEB211D41A4602F8016B13461546920720
:10D8900010D0621E002C79D003F8016B14469A0751
:10D8A0001D4607D0013CEDE7034603F8016B9A07DC
:10D8B0001D46F7D1032C52D9CEB246EA06270F2CCB
:10D8C00047EA07432DD9A4F1100217460F2FC2F3E0
:10D8D00000162B606B60AB60EB6005F1100216D98F
:10D8E0003EB1103F136053609360D36010320F2F2E
:10D8F0000DD9203F02F11006136053609360D3608E
:10D90000136153619361D36120320F2FF1D8A4F1D9
:10D91000100222F00F0204F00F041032032C154401
:10D920001DD9271F3E462A46032E42F8043BC7F363
:10D9300080070DD927B1043E032E42F8043B07D9D6
:10D94000174647F8043B083E53603A1D032EF7D8AC
:10D95000231F23F00302131D04F00304ED18ACB1E0
:10D96000C9B2EA432C1905F8011BA318A54203F01C
:10D9700001020BD01AB105F8011BA54206D02B46B7
:10D9800003F8011B69705D1CA542F8D1F0BC70471B
:10D99000054614468EE700BF830770B5064614D1CE
:10D9A0000368A3F1013222EA030010F0803F0CD19A
:10D9B000331D1A4653F8044BA4F1013525EA04043B
:10D9C00014F0803FF5D0104600E0304603782BB1CC
:10D9D000421C147810460132002CFAD100F080F875
:10D9E000304670BDC9B2F0B400294BD082070FD0C9
:10D9F0000278002A71D0914242D0431C05E013F80E
:10DA0000012B002A3BD091423AD09A071846F6D112
:10DA1000036841EA0127A3F1013222EA030212F06E
:10DA2000803F47EA07471CD17B40A3F1013222EA3D
:10DA3000030313F0803F14D1021D02E014F0803F75
:10DA40000FD1104652F8043BA3F1013687EA0304D4
:10DA500026EA0303A4F1013513F0803F25EA04040C
:10DA6000ECD00278002A38D0914209D0431C01E062
:10DA7000914205D0184613F8012B002AF8D1104620
:10DA8000F0BC704783070BD00278002AF8D0431C03
:10DA900003E0017801330029F2D099071846F8D144
:10DAA0000168A1F1013323EA010212F0803F0AD19B
:10DAB000031D184653F8041BA1F1013424EA0102A6
:10DAC00012F0803FF5D00378002BD9D0421C11789A
:10DAD000104601320029FAD1D2E71046D0E700BF44
:10DAE00080EA0102844612F0030F4FD111F0030FB8
:10DAF00032D14DF8044D11F0040F51F8043B0BD016
:10DB0000A3F101329A4312F0803F04BF4CF8043B6A
:10DB100051F8043B16D100BF51F8044BA3F1013278
:10DB20009A4312F0803FA4F101320BD14CF8043B30
:10DB3000A24312F0803F04BF51F8043B4CF8044B61
:10DB4000EAD023460CF8013B13F0FF0F4FEA3323D2
:10DB5000F8D15DF8044B704711F0010F06D011F8B1
:10DB6000012B0CF8012B002A08BF704711F0020F9F
:10DB7000BFD031F8022B12F0FF0F16BF2CF8022B8A
:10DB80008CF8002012F47F4FB3D1704711F8012BAD
:10DB90000CF8012B002AF9D1704700BF20F00301D7
:10DBA00010F00300C0F1000051F8043B00F1040C38
:10DBB0004FEACC0C6FF000021CBF22FA0CF21343A8
:10DBC0004FF0010C4CEA0C2C4CEA0C4CA3EB0C0271
:10DBD00022EA030212EACC1204BF51F8043B0430DB
:10DBE000F4D013F0FF0F1FBF013013F47F4F01304B
:10DBF00013F47F0F18BF0130704700BFF0B4002A44
:10DC000063D0344B04461B6814F8010B571E1D18D3
:10DC10006E7807F0010706F00305012D58D011F8C2
:10DC2000015B5E19767806F00306012E08BF2035E9
:10DC3000401B4BD1002D49D0013A47D02FB314F8E7
:10DC4000010B1D186E7806F00305012D11F8015B1C
:10DC500008BF20305E19767806F00306012E08BF53
:10DC60002035401B32D18DB3013A0ED12EE011F890
:10DC7000012B9E18767806F00306012E08BF20328D
:10DC8000801A23D112B36A1E20D014F8010B1D187C
:10DC90006E7806F00305012D11F8015B08BF2030F6
:10DCA0005E19767806F00306012E08BF2035401B6A
:10DCB0000CD15DB114F8010B551E1A18567806F0F8
:10DCC0000302012AD3D12030D1E71046F0BC7047BF
:10DCD0002030A4E76C01002041EA00039B07F0B468
:10DCE00074D1032A72D90C4654F8045B161FA5F1AF
:10DCF000013727EA050717F0803F0346C6F3800C7B
:10DD000031D10346032E324643F8045B2AD9BCF1D5
:10DD1000000F0AD0214654F8045BA5F1013626EA2B
:10DD2000050616F0803F18D01DE0264656F8045B25
:10DD30002146A5F1013727EA050717F0803F12D1E8
:10DD400043F8045B65683146A5F1013626EA05060D
:10DD5000043A0C1D16F0803F05D1043A032A43F81B
:10DD6000045BE2D821467AB30D78013A03F8015BEF
:10DD70009DB112F0010F1C462AD1234622B311F89F
:10DD8000015F013A03F8015B3DB111F8015F013A0F
:10DD900065705C1C2346002DEFD1AAB100219C18B0
:10DDA000DA4303F8011BA218A34202F001020BD0D0
:10DDB0001AB103F8011BA34206D01A4602F8011B50
:10DDC0005970531CA342F8D1F0BC70470346CAE710
:10DDD00011F8015F1C4604F8015B013A2346002D4F
:10DDE000CBD1DAE72DE9F00701273C4600254FF0BB
:10DDF000FF3663198B4200EB060C0DD21CF804A011
:10DE000010F80380D0452ED201241D469F1B6319B4
:10DE10008B4200EB060CF1D34FF0010A1760544619
:10DE200000254FF0FF3C6319994200EB0C080ED916
:10DE300018F8048010F80390C1451AD901241D4632
:10DE4000CCEB030A6319994200EB0C08F0D80CF1F3
:10DE500001000136B0423CBFBA463046C2F800A0CD
:10DE6000BDE8F00770470BD001272E463C46ED1960
:10DE7000BFE709D04FF0010AAC4654465544D2E7FB
:10DE8000BC4205D00134B4E7544505D00134CAE79B
:10DE900027461D460124ACE7A2461D460124C2E7E1
:10DEA0002DE9F04FADF2244D154606468946104641
:10DEB000194607AA1C46FFF795FF07AB82460DF2ED
:10DEC0001C411A1D5C6008338B425460F9D114B3B5
:10DED00001232F78611E08A8A34240F8271001EA09
:10DEE000030218D032B16A7802234F1EA34240F8D1
:10DEF000227010D0B046A4465C1C15F803E0CE1A80
:10DF00002A5D02330F1B634540F82E6040F82270F3
:10DF1000F2D146466446079928466918524600F0F1
:10DF200045FC002840F0B6800AF1FF3E05EB0E0CE0
:10DF3000CDF808E0CAF1010E834604F1FF38CDF8B0
:10DF40000CC0CDF814E00746CDF810A04A46009565
:10DF5000019408E027B1079FBB4201D20199CB1B76
:10DF60009B4400272246019CB0185C440021A21A61
:10DF700000F07CFB002840F08780002C00F08480BB
:10DF8000301910F8013C08A951F82330002BE1D1D9
:10DF9000049B9F4228BF3B46434527D2DDF80090B3
:10DFA00006EB0B0119F80350CA5C09EB030095421C
:10DFB00066D1DD43454415F0010F024613D001330D
:10DFC000434513D24078CD5C013285420BD057E0F7
:10DFD00012F8010FCD5C854252D1013312F8010FC6
:10DFE000CD5C85424CD101334345F1D3DDF810902F
:10DFF000029B4F4528BF4B4639D2DDF808C0DDF8FB
:10E00000009006EB0B0519F80C1015F80C00814276
:10E0100040F0C080DDF80CE009EB070ACAEB0E0106
:10E02000C80772461ED5DDF8089009F1FF31DDF80A
:10E030000C90685C19F801CC09F1FF32844516D1C7
:10E040000B460FE012F8019C15F800E04A1EF1455E
:10E050000DD10346013815F800C011F8011C6145C7
:10E0600005D10346581E524502F1FF31EAD101376E
:10E070009F4200F29180079F019ABB44D71B71E732
:10E08000DDF814E0F3446BE7002009B00DF5806D76
:10E09000BDE8F08FCAEB0400504538BF5046CAF1C6
:10E0A0000102431C0AF1FF3C05EB0A0704F1FF3BA8
:10E0B000019200944A460793B1464FF00008644627
:10E0C0003E46009909EB020008EB0107BA1A00214D
:10E0D00000F0CCFA0028D7D1002FD5D009EB0700EB
:10E0E00010F8013C08AA52F8230000284AD1DA456A
:10E0F00009EB08002AD210F80A303178994218BF8B
:10E10000534642D16FEA0A0303EB0B01C9073246BB
:10E11000534618D50AF101035B4517D2324612F86F
:10E12000011F10F803E08E450DD02EE012F8011FFC
:10E1300010F803C08C4528D1013312F8011F10F8E4
:10E1400003E08E4521D101335B45EFD3621C2346AA
:10E150009BD0295D025D914213D1E10709D5631E71
:10E16000E95CC25C914204D00BE0E95CC25C914284
:10E1700007D15A1E002B88D0A95C825C023B9142D9
:10E18000F3D0079880443A469BE7DDF804C0E044AA
:10E190009844F8E7049B6AE706EB0B0075E700BFBD
:10E1A0002DE9F04F037889B080460D46002B00F032
:10E1B00065810A789AB184460131012602E011F89E
:10E1C000012B5AB1934214BF002606F001061CF839
:10E1D000013F0C46002BF2D1207820B936B14046E1
:10E1E00009B0BDE8F08F4FF00008F8E708F1010032
:10E1F0002978FFF7F7FB641B06460028F3D0012CB3
:10E2000000F0B580A044404594BFC0EB080701274B
:10E210001F2C06D939462A462346FFF741FE804681
:10E22000DDE7214607AA2846FFF7DCFD07990390A2
:10E2300069182846039A00F0B9FA002840F099803E
:10E24000DDF80CC0DDF80C900CF1FF3E05EB0E0183
:10E25000C9F1010C8346CDF808E080460491CDF861
:10E2600014C03A46B146019508EB040609EB0200DA
:10E270000021B21A00F0FAF90028B4D1002EB2D071
:10E28000039B9B4528BF5B469C4227D9019D09EB18
:10E29000030010F80820E95CE81891425FD1DD43E3
:10E2A0002D1915F0010F024609EB080113D00133B7
:10E2B0009C4213D94078CD5C013285420BD04EE0B0
:10E2C00012F8010FCD5C854249D1013312F8010FDC
:10E2D000CD5C854243D101339C42F1D8DDF80CE09E
:10E2E000029ADE4540F2CD80019B09EB0805995C5E
:10E2F000A85C814240F0C580DDF804A0049BDA44AC
:10E30000CAEB0301C8071AD5029FDDF810C0791EB9
:10E31000685C1CF8017C0CF1FF33874214D10A467B
:10E320000DE013F801EC2F5C4B1EBE450CD10246EC
:10E3300001382F5C11F8011CB94205D10246501E6C
:10E34000534503F1FF31ECD10BF1010B934500F282
:10E350009A80079A9044C2EB040B324684E7059DED
:10E3600005EB080B0BEB03084FF0000BF5E78046BD
:10E3700035E7DDF80CA00399CAEB0403534538BF19
:10E380005346CAF1010B581C06EB0A0205EB0A08BA
:10E39000CDF808B03B4607904FF00009019201F11B
:10E3A000FF3B37468A4609EB0406F8180021F21AAB
:10E3B00000F05CF900287FF416AF002E3FF413AF95
:10E3C000544598BF07EB09002CD9DDF804E098F814
:10E3D00000001EF8093098424AD16FEA0A0211196A
:10E3E000C9074246534607EB090018D50AF1010355
:10E3F0009C4217D9424612F8011F10F803C08C4501
:10E400000DD036E012F8011F10F803E08E4530D130
:10E41000013312F8011F10F803C08C4529D10133D4
:10E420009C42EFD8BBF1FF3F5B463FF4F8AE15F8D6
:10E430000B1010F80B20914216D11BF0010F0AD0DF
:10E440000BF1FF33E95CC25C914204D00CE0E95C63
:10E45000C25C914208D15A1E002B3FF4E0AEA95C89
:10E46000825C023B9142F2D00798814433469AE79E
:10E470005346DDF808E0F1449944F7E70C460126DD
:10E48000AAE6039A60E74E46C844A8E640F29853CD
:10E49000C2F200031A6801235C3200F001B800BF29
:10E4A000F0B4002825D0074638463E780D4601379F
:10E4B00015F8014B3CB1A642FAD1002BF4D11760FC
:10E4C00007F8013C11E0C6B13D4600E01BB915F864
:10E4D000016B0C46284614F8013B9E42F6D136B13A
:10E4E000002105F8011C1060781EF0BC7047304612
:10E4F000F9E710680028D6D1F7E716603046F4E750
:10E500002DE9F00F494C82B0D4F800C001900F46BD
:10E510003C4614F8015B0CEB05004678274606F0F4
:10E520000800C6B2002EF3D12D2D61D02B2D04BFD3
:10E53000244614F8015BB346002B41D1302D43D063
:10E540000A239A46BBF1000F0CBF6FF000474FF053
:10E550000047B7FBFAF90AFB1970009000208046CB
:10E560000CE0303DAB421BDD461C05D0C84539D818
:10E5700035D00AFB0858012014F8015B0CEB0506A6
:10E58000767806F00407FFB2002FEAD116F00306F2
:10E5900006D0012E14BF57263726AD1BAB42E3DC55
:10E5A000431C2AD0BBF1000F01D0C8F10008002A9B
:10E5B00031D0D0B94046116002B0BDE8F00F7047CD
:10E5C000102BBED1302DBCD12578782D25D0582DDB
:10E5D00023D043BB4FF0080A30255346B2E70098DA
:10E5E0008542C6DD4FF0FF30C6E74046611EE2E7D8
:10E5F00014F8015B4FF0010B9EE7BBF1000F01998E
:10E600000CBF6FF000404FF0004022230B60002A47
:10E61000D2D0611ECFE74046CEE74FF0100A6578B2
:10E62000534602348EE79A4630258BE76C01002072
:10E6300070B440F29854C2F2000406460D462068B9
:10E64000134631462A4670BCFFF75ABF024B13B13E
:10E65000024800F005B87047000000002DD6000801
:10E660000146002002460346FEF760BF8307F0B470
:10E67000C9B200F09680531E002A00F09480027800
:10E680008A420BD0421CD8071AD512F0030F10464D
:10E690001CD01478013B01328C4211D1F0BC704780
:10E6A000002B7CD01278013B8A42F7D014F0030F84
:10E6B000204604F1010209D02478013B8C42EDD0C0
:10E6C00012F0030F104602F10104E9D1032B3FD9E8
:10E6D000046841EA012545EA054585EA0407A7F1F2
:10E6E000013222EA07021E1F041D12F0803FC6F30A
:10E6F00080072DD1032E334629D967B126682046DD
:10E7000085EA0602A2F1013626EA0202043412F07A
:10E71000803F19D01CE020462468061D85EA0402CB
:10E72000A2F1013424EA020212F0803F10D13468D1
:10E73000043B85EA0402A2F1013424EA0202341DFA
:10E7400012F0803F304603D1043B032BE3D8204630
:10E750005D1E23B303788B42A0D0431C0022E80740
:10E7600014D51C781846012201338C4296D095426C
:10E77000184603F1010402F102020ED01B788B420D
:10E780008CD020462478431C8C4287D09542184672
:10E7900003F1010402F10202F0D100207EE71846E5
:10E7A0007CE7134692E7104678E700BF032AF0B4EF
:10E7B00031D941EA00039C072ED106680F68151F66
:10E7C000031D0C1DBE42C5F3800C24D1032D2A4627
:10E7D0001FD9BCF1000F08D01E68256821461846D5
:10E7E00004340433AE4211D015E0214618461C68AB
:10E7F0000B68051D0E1D9C420DD1314628462E6822
:10E800000D68043A031D0C1DAE4204D1043A032ADC
:10E81000EBD8214618461AB303780C78A3420AD1E4
:10E82000551E0022EB0714D510F8013F11F8014FD7
:10E830000122A3420DD0181B10E010F8013F11F87F
:10E84000014FA342F7D110F8013F11F8014FA34245
:10E85000F1D1AA4202F10202EFD10020F0BC7047D0
:10E860001046FBE71E1E6464646464641048498AB1
:10E870008B8C8D84858687FF1048494A4B4C4D44CC
:10E88000454647FF202122232425262748498A8BF5
:10E890008C8DFF00A4E8000878E8000884E80008F0
:10E8A0006CE80008202122232425262748494A4BCA
:10E8B0004C4DFF00D31D0008811D0008A51D000858
:10E8C0006D1D0008731D00086F1D0008000000404A
:10E8D0000008014001000000001C00000000004092
:10E8E0000008014002000000041C0000000000407D
:10E8F0000008014004000000081C00000000004067
:10E9000000080140080000000C1C0000000400404A
:10E910000008014040000000001D0000000400400D
:10E920000008014080000000041D000000040040B9
:10E93000000C014001000000081D00000004004020
:10E94000000C0140020000000C1D0000002C0140E2
:10E950000008014000010000001B0100002C0140E4
:10E9600000080140000800000C1B010000080040E6
:10E97000000C014040000000001E000000080040A4
:10E98000000C014080000000041E00000008004050
:10E99000000C014000010000081E000000080040BB
:10E9A000000C0140000200000C1E0000002C014081
:10E9B0000000004000040040000800400004080C73
:10E9C000D007320032003200320032003200320012
:10E9D000C800640000004145545231323334000015
:10E9E000A7500008CF4F0008775000082D500008AE
:10E9F000E54F0008CD4F00080000803F00000000F8
:10EA00000000803F0000803F0000803F000080BF8A
:10EA1000000080BF000000000000803F00000000F8
:10EA20000000803F000080BF0000803F0000803F6A
:10EA3000000080BF000000800000803F0000000058
:10EA4000A8AAAA3F0000803F0000803F000080BFCE
:10EA5000B0AA2ABF000080BF0000803F0000803FB6
:10EA6000B0AA2ABF000080BF0000803F0000000065
:10EA7000A8AAAA3F000080BF0000803F000080BF1E
:10EA8000B0AA2ABF0000803F0000803F0000803F06
:10EA9000B0AA2ABF0000803F0000803F00000000B5
:10EAA000A8AAAA3F000000000000803F000080BF2D
:10EAB000B0AA2ABF000000000000803F0000803F95
:10EAC000B0AA2ABF000000000000803F000080BF05
:10EAD0000000803F000080BF0000803F000080BF3A
:10EAE000000080BF0000803F0000803F0000803FAA
:10EAF0000000803F0000803F0000803F0000803F1A
:10EB0000000080BF000080BF0000803F00000000C8
:10EB100000000000000000000000803F0000000036
:10EB200000000000000000000000803F000000BF67
:10EB3000D0B35D3F0000803F0000803F000000BF79
:10EB4000D0B35DBF0000803F0000803F0000003F69
:10EB5000D0B35D3F000080BF0000803F0000003F59
:10EB6000D0B35DBF000080BF0000803F000080BFC9
:10EB700000000000000080BF0000803F0000803FD8
:10EB8000000000000000803F0000803F0000000007
:10EB90000000803F000080BF0000803F000080BF79
:10EBA000000000000000803F0000803F0000803F28
:10EBB000000000000000803F0000803F00000000D7
:10EBC000000080BF000080BF0000000000000000C7
:10EBD0000301000098EA00080400000088EB000828
:10EBE00004000000C0ED00080201000060ED000814
:10EBF00000010000000000000600000038EA0008E4
:10EC00000600000000ED0008010100000000000007
:10EC10000400000080ED00080600000028EB00085A
:10EC20000800000080EE00080800000080EC0008EA
:10EC30000800000000EE00080101000000000000D4
:10EC400000010000000000000001000000000000C2
:10EC500004000000F8E9000806000000C8EA000807
:10EC600000010000000000000201000000EF0008A9
:10EC70000101000000000000000000000000000092
:10EC80000000803FF704353FF70435BF0000803FA8
:10EC90000000803FF70435BFF70435BF0000803F18
:10ECA0000000803FF70435BFF704353F0000803F88
:10ECB0000000803FF704353FF704353F0000803FF8
:10ECC0000000803F00000000000080BF000080BF07
:10ECD0000000803F000080BF00000000000080BFF7
:10ECE0000000803F000000000000803F000080BF67
:10ECF0000000803F0000803F00000000000080BF57
:10ED00000000803FD0B35DBF0000003F0000803FA7
:10ED10000000803FD0B35DBF000000BF000080BF97
:10ED20000000803FD0B35D3F0000003F0000803F07
:10ED30000000803FD0B35D3F000000BF000080BFF7
:10ED40000000803F00000000000080BF0000803F06
:10ED50000000803F000000000000803F000080BFF6
:10ED60000000803F0000803F000000000000000025
:10ED70000000803F000080BF000000000000000095
:10ED80000000803F000000000000803F000080BFC6
:10ED90000000803F000080BF000080BF0000000036
:10EDA0000000803F000000000000803F0000803F26
:10EDB0000000803F0000803F000080BF0000000096
:10EDC0000000803F000080BF0000803F000080BF47
:10EDD0000000803F000080BF000080BF0000803F37
:10EDE0000000803F0000803F0000803F0000803F27
:10EDF0000000803F0000803F000080BF000080BF17
:10EE00000000803F0000803F000000BF0000803F06
:10EE10000000803F000000BF000080BF0000803F76
:10EE20000000803F000080BF0000003F0000803FE6
:10EE30000000803F0000003F0000803F0000803F56
:10EE40000000803F0000003F000080BF000080BF46
:10EE50000000803F000080BF000000BF000080BFB6
:10EE60000000803F000000BF0000803F000080BF26
:10EE70000000803F0000803F0000003F000080BF96
:10EE80000000803F000080BF0000803F000080BF86
:10EE90000000803F000080BF000080BF0000803F76
:10EEA0000000803F0000803F0000803F0000803F66
:10EEB0000000803F0000803F000080BF000080BF56
:10EEC0000000803F000080BF0000803F0000803FC6
:10EED0000000803F000080BF000080BF000080BFB6
:10EEE0000000803F0000803F0000803F000080BFA6
:10EEF0000000803F0000803F000080BF0000803F96
:10EF00000000803F0000000000000000000080BF03
:10EF10000000803F00000000000000000000803F73
:10EF200024505542582C34312C312C303030332C75
:10EF3000303030312C3131353230302C302A3145BF
:10EF40000D0A0024504D544B3235312C31313532BD
:10EF500030302A31460D0A0024505542582C3431A5
:10EF60002C312C303030332C303030312C3537369A
:10EF700030302C302A32440D0A0024504D544B328C
:10EF800035312C35373630302A32430D0A002450C3
:10EF90005542582C34312C312C303030332C303019
:10EFA00030312C33383430302C302A32360D0A00D0
:10EFB00024504D544B3235312C33383430302A32D2
:10EFC000370D0A0024505542582C34312C312C3046
:10EFD0003030332C303030312C31393230302C302D
:10EFE0002A32330D0A0024504D544B3235312C3126
:10EFF000393230302A32320D0A00B5620601030080
:10F00000F00500FF19B56206010300F00300FD15CD
:10F01000B56206010300F00100FB11B562060103B1
:10F0200000F00000FA0FB56206010300F00200FCD8
:10F0300013B56206010300F00400FE17B562060175
:10F0400003000102010E47B562060103000103013E
:10F050000F49B56206010300010601124FB56206B1
:10F060000103000112011E67B562061608000307BE
:10F070000300510800008A41B56206080600C80076
:10F0800001000100DE6A00000000000000C2010073
:10F0900020EF000843EF00080100000000E100003D
:10F0A00058EF00087AEF0008020000000096000008
:10F0B0008EEF0008B0EF000803000000004B0000D6
:10F0C000C4EF0008E6EF00080400000080250000FF
:10F0D000FCF70008FCF70008414552543132333444
:10F0E000000000001F00010823000108280001089B
:10F0F00039000108420001084D00010858000108CC
:10F100006300010841FF00086C0001083BFF000894
:10F11000750001087F0001088A00010890000108BD
:10F120000000000071FF000875FF00087BFF000869
:10F1300081FF000884FF00088BFF00088EFF000895
:10F1400093FF00089FFF0008A2FF0008A8FF000827
:10F15000AFFF0008B9FF0008C3FF0008CCFF00089C
:10F16000DAFF0008E6FF0008EDFF0008F3FF0008E3
:10F17000000001080B000108180001080000000051
:10F1800083FD000887FD00081D8F0008AEFD000804
:10F19000B3FD000819940008C7FD0008D0FD000861
:10F1A0005D8D0008EDFD0008F2FD00086592000885
:10F1B00021FE0008FCF70008258D000826FE000847
:10F1C0002EFE0008398C000842FE000851FE00089F
:10F1D000198C00086BFE0008FCF70008158A00086F
:10F1E00070FE000874FE0008718B0008C1FD000865
:10F1F00090FE0008898D0008A3FE0008A9FE000803
:10F20000758E0008C4FE0008CCFE0008298E000898
:10F21000DBFE0008E0FE0008418B00080DF7000847
:10F22000F0FE0008119100081EFF000812FF000800
:10F23000418A000825FF0008FCF70008098A000839
:10F24000FCF700084DFF000855FF00085DFF0008AF
:10F2500065FF00086CFF0008000000003031323309
:10F260003435363738394142434445464748494AA0
:10F270004B4C4D4E4F505152535455565758595A66
:10F28000004166726F333220434C492076657273B9
:10F29000696F6E20322E3220417072203138203258
:10F2A000303134202F2031373A32393A333100416E
:10F2B0007661696C61626C6520636F6D6D616E640F
:10F2C000733A0D0A0025730925730D0A00537973EB
:10F2D00074656D20557074696D653A2025642073DE
:10F2E00065636F6E64732C20566F6C746167653A4A
:10F2F000202564202A20302E3156202825645320D2
:10F3000062617474657279290D0A00435055202595
:10F31000644D487A2C206465746563746564207359
:10F32000656E736F72733A2000257320004143436A
:10F3300048573A202573002E2563004379636C6596
:10F340002054696D653A2025642C204932432045BC
:10F3500072726F72733A2025642C20636F6E666937
:10F36000672073697A653A2025640D0A0053617637
:10F37000696E672E2E2E000D0A5265626F6F7469DA
:10F380006E672E2E2E004D75737420626520616E9F
:10F3900079206F72646572206F6620414554523146
:10F3A0003233340D0A0043757272656E74206173D6
:10F3B0007369676E6D656E743A20004572726F7284
:10F3C0003A20456E61626C6520616E6420706C75D8
:10F3D0006720696E204750532066697273740D0A66
:10F3E00000456E61626C696E672047505320706102
:10F3F00073737468726F7567682E2E2E0D0A004540
:10F400006E61626C65642066656174757265733ADD
:10F410002000417661696C61626C6520666561748B
:10F42000757265733A2000496E76616C6964206676
:10F43000656174757265206E616D652E2E2E0D0AE4
:10F440000044697361626C65642000456E61626CA2
:10F45000656420000D0A4C656176696E6720434C37
:10F4600049206D6F64652E2E2E0D0A00526573655E
:10F470007474696E6720746F2064656661756C745E
:10F48000732E2E2E0D0A0043757272656E74206DF8
:10F49000697865723A2025730D0A00417661696CBE
:10F4A00061626C65206D69786572733A2000496EFF
:10F4B00076616C6964206D69786572207479706515
:10F4C0002E2E2E0D0A004D6978657220736574200A
:10F4D000746F2025730D0A0043757272656E742077
:10F4E00070726F66696C653A2025640D0A00557369
:10F4F0006167653A0D0A6D6F746F7220696E64659D
:10F5000078205B76616C75655D202D2073686F7760
:10F51000205B6F72207365745D206D6F746F722055
:10F5200076616C75650D0A004E6F207375636820F7
:10F530006D6F746F722C207573652061206E756D10
:10F54000626572205B302C2025645D0D0A004D6FD2
:10F55000746F722025642069732073657420617450
:10F560002025640D0A00496E76616C6964206D6F18
:10F57000746F722076616C75652C20313030302EBE
:10F580002E323030300D0A0053657474696E672076
:10F590006D6F746F7220256420746F2025640D0ACE
:10F5A000006175782025752025750D0A00496E7655
:10F5B000616C6964204665617475726520696E646A
:10F5C00065783A206D757374206265203C2025753E
:10F5D0000D0A002025642025640043757272656E53
:10F5E000742073657474696E67733A200D0A002580
:10F5F000732073657420746F20004552523A205670
:10F60000616C75652061737369676E6D656E7420DA
:10F610006F7574206F662072616E67650D0A004514
:10F6200052523A20556E6B6E6F776E20766172691A
:10F6300061626C65206E616D650D0A0043757272C2
:10F64000656E7420436F6E6669673A20436F707908
:10F650002065766572797468696E672062656C6F83
:10F660007720686572652E2E2E0D0A006D6978650B
:10F67000722025730D0A00636D697820256400638C
:10F680006D697820256420302030203020300D0A2C
:10F690000066656174757265202D25730D0A00661C
:10F6A0006561747572652025730D0A006D617020A7
:10F6B00025730D0A00736574202573203D20004ECC
:10F6C0004709004F4B0900437573746F6D206D69D6
:10F6D0007865723A200D0A4D6F746F720954687222
:10F6E00009526F6C6C095069746368095961770D30
:10F6F0000A002325643A09002573090053616E69E5
:10F70000747920636865636B3A0900726573657488
:10F71000006C6F6164004C6F616465642025732028
:10F720006D69782E2E2E0D0A0057726F6E67206E4F
:10F73000756D626572206F6620617267756D656EAA
:10F7400074732C206E656564732069647820746816
:10F750007220726F6C6C20706974636820796177B5
:10F760000D0A004D6F746F72206E756D62657220A8
:10F770006D757374206265206265747765656E20AF
:10F780003120616E642025640D0A000D0A456E74F7
:10F790006572696E6720434C49204D6F64652C206B
:10F7A000747970652027657869742720746F2072DA
:10F7B000657475726E2C206F72202768656C7027D7
:10F7C0000D0A000D0A2320000D1B5B4B001B5B3252
:10F7D0004A1B5B313B3148004552523A20556E6B13
:10F7E0006E6F776E20636F6D6D616E642C20747226
:10F7F00079202768656C702700082008006C6F6FFF
:10F800007074696D65006D69647263006D696E7412
:10F8100068726F74746C65006D61787468726F746F
:10F82000746C65006D696E636F6D6D616E64006D03
:10F83000696E636865636B006D6178636865636BAF
:10F84000006465616462616E6433645F6C6F77004D
:10F850006465616462616E6433645F6869676800EF
:10F860006E65757472616C336400646561646261B5
:10F870006E6433645F7468726F74746C65006D6F6E
:10F88000746F725F70776D5F72617465007365721B
:10F89000766F5F70776D5F72617465007265746119
:10F8A000726465645F61726D00666C6170735F7332
:10F8B0007065656400666978656477696E675F6125
:10F8C0006C74686F6C645F646972007265626F6FFC
:10F8D000745F63686172616374657200736F6674EC
:10F8E00073657269616C5F626175647261746500F1
:10F8F000736F667473657269616C5F315F696E7690
:10F90000657274656400736F667473657269616CA7
:10F910005F325F696E766572746564006770735FED
:10F9200074797065006770735F6261756472617489
:10F93000650073657269616C72785F7479706500D7
:10F9400074656C656D657472795F70726F766964E9
:10F9500065720074656C656D657472795F706F7245
:10F96000740074656C656D657472795F7377697422
:10F97000636800766261747363616C6500766261CE
:10F98000746D617863656C6C766F6C74616765002B
:10F99000766261746D696E63656C6C766F6C7461B0
:10F9A000676500706F7765725F6164635F6368614C
:10F9B0006E6E656C00616C69676E5F6779726F006F
:10F9C000616C69676E5F61636300616C69676E5F3C
:10F9D0006D616700616C69676E5F626F6172645F21
:10F9E000726F6C6C00616C69676E5F626F617264EC
:10F9F0005F706974636800616C69676E5F626F61F4
:10FA000072645F796177007961775F636F6E74729A
:10FA10006F6C5F646972656374696F6E00616363C4
:10FA20005F6861726477617265006D61785F616EB5
:10FA3000676C655F696E636C696E6174696F6E0097
:10FA40006D6F726F6E5F7468726573686F6C64005F
:10FA50006779726F5F6C7066006779726F5F636D54
:10FA600070665F666163746F72006779726F5F635F
:10FA70006D70666D5F666163746F72007069645F5C
:10FA8000636F6E74726F6C6C657200796177646518
:10FA9000616462616E6400616C745F686F6C645F66
:10FAA0007468726F74746C655F6E65757472616C86
:10FAB00000616C745F686F6C645F666173745F6330
:10FAC00068616E6765007468726F74746C655F63FB
:10FAD0006F7272656374696F6E5F76616C756500D5
:10FAE0007468726F74746C655F636F72726563744F
:10FAF000696F6E5F616E676C650072635F726174DF
:10FB0000650072635F6578706F007468725F6D691D
:10FB100064007468725F6578706F00726F6C6C5F00
:10FB200070697463685F726174650079617772618E
:10FB300074650074706172617465007470615F62F5
:10FB40007265616B706F696E74006661696C736178
:10FB500066655F64656C6179006661696C73616696
:10FB6000655F6F66665F64656C6179006661696C8C
:10FB7000736166655F7468726F74746C650066614A
:10FB8000696C736166655F6465746563745F7468EE
:10FB9000726573686F6C6400727373695F61757806
:10FBA0005F6368616E6E656C007961775F6469722E
:10FBB000656374696F6E007472695F756E61726DF2
:10FBC00065645F736572766F0067696D62616C5F13
:10FBD000666C616773006163635F6C70665F66612A
:10FBE00063746F720061636378795F6465616462F6
:10FBF000616E64006163637A5F6465616462616E13
:10FC000064006163635F756E61726D656463616CEE
:10FC1000006163635F7472696D5F7069746368002B
:10FC20006163635F7472696D5F726F6C6C006261B7
:10FC3000726F5F7461625F73697A65006261726F8F
:10FC40005F6E6F6973655F6C7066006261726F5F93
:10FC500063665F76656C006261726F5F63665F61A9
:10FC60006C74006D61675F6465636C696E61746973
:10FC70006F6E006770735F706F735F700067707393
:10FC80005F706F735F69006770735F706F735F643D
:10FC9000006770735F706F73725F70006770735F7F
:10FCA000706F73725F69006770735F706F73725FFC
:10FCB00064006770735F6E61765F70006770735F7A
:10FCC0006E61765F69006770735F6E61765F640076
:10FCD0006770735F77705F726164697573006E61DE
:10FCE000765F636F6E74726F6C735F686561646971
:10FCF0006E67006E61765F73706565645F6D696ED7
:10FD0000006E61765F73706565645F6D6178006E2B
:10FD100061765F736C65775F7261746500705F70A8
:10FD20006974636800695F706974636800705F720A
:10FD30006F6C6C00695F726F6C6C00705F796177DB
:10FD400000695F79617700705F616C7400695F6161
:10FD50006C7400645F616C7400705F6C6576656CD8
:10FD600000695F6C6576656C00645F6C6576656CD8
:10FD700000705F76656C00695F76656C00645F7625
:10FD8000656C0061757800666561747572655F6E9B
:10FD9000616D6520617578666C6167206F722062A5
:10FDA0006C616E6B20666F72206C69737400636D9A
:10FDB00069780064657369676E20637573746F6D2D
:10FDC000206D697865720064656661756C74730096
:10FDD000726573657420746F2064656661756C74F8
:10FDE0007320616E64207265626F6F740064756D5C
:10FDF00070007072696E7420636F6E6669677572E9
:10FE000061626C652073657474696E677320696ED6
:10FE10002061207061737461626C6520666F726D21
:10FE200000657869740066656174757265006C6957
:10FE30007374206F72202D76616C206F7220766152
:10FE40006C00677073706173737468726F75676844
:10FE500000706173737468726F7567682067707380
:10FE600020746F2073657269616C0068656C700046
:10FE70006D6170006D617070696E67206F662072D1
:10FE800063206368616E6E656C206F7264657200DA
:10FE90006D69786572206E616D65206F72206C6986
:10FEA0007374006D6F746F72006765742F7365747F
:10FEB000206D6F746F72206F757470757420766129
:10FEC0006C75650070726F66696C6500696E64655B
:10FED0007820283020746F20322900736176650005
:10FEE0007361766520616E64207265626F6F740065
:10FEF0006E616D653D76616C7565206F7220626C18
:10FF0000616E6B206F72202A20666F72206C69739D
:10FF1000740073686F772073797374656D207374E0
:10FF2000617475730076657273696F6E004759521C
:10FF30004F00414343004241524F00534F4E415204
:10FF400000475053004750532B4D41470041445800
:10FF50004C333435004D505536303530004D4D4121
:10FF60003834357800424D41323830004E6F6E657E
:10FF70000054524900515541445000515541445894
:10FF80000042490047494D42414C0059360048451E
:10FF9000583600464C59494E475F57494E4700591D
:10FFA00034004845583658004F43544F5838004F96
:10FFB00043544F464C415450004F43544F464C41DC
:10FFC000545800414952504C414E450048454C4917
:10FFD0005F3132305F4343504D0048454C495F39F3
:10FFE000305F44454700565441494C340048455819
:10FFF00036480050504D5F544F5F534552564F00A6
:020000040801F1
:100000004455414C434F505445520053494E474C80
:1000100045434F5054455200435553544F4D0050A3
:10002000504D005642415400494E464C49474854B1
:100030005F4143435F43414C0053455249414C5259
:1000400058004D4F544F525F53544F500053455238
:10005000564F5F54494C5400534F465453455249F0
:10006000414C004C45445F52494E47004641494C83
:10007000534146450054454C454D45545259005056
:100080004F5745524D4554455200564152494F0035
:10009000334400002DFF000832FF000836FF00083F
:1000A00049FF00083BFF000841FF000845FF00082A
:1000B00000000000FDF7000802000000DC1700202F
:1000C000000000002823000006F8000802000000DD
:1000D000E2180020B0040000A40600000CF800089C
:1000E00002000000A018002000000000D00700005F
:1000F00018F8000802000000A2180020000000000C
:10010000D007000024F8000802000000A418002016
:1001100000000000D00700002FF8000802000000D7
:10012000E418002000000000D007000038F80008A4
:1001300002000000E618002000000000D0070000C8
:1001400041F8000802000000A6180020000000008E
:10015000D007000050F8000802000000A818002096
:1001600000000000D007000060F800080200000056
:10017000AA18002000000000D00700006AF800085C
:1001800002000000AC18002000000000D0070000B2
:100190007EF8000802000000AE18002032000000C7
:1001A000007D00008DF8000802000000B01800205B
:1001B00032000000F20100009CF80008000000007E
:1001C000E81800200000000001000000A9F8000865
:1001D00000000000E918002000000000640000009A
:1001E000B5F8000801000000EA180020FFFFFFFF3B
:1001F00001000000CBF8000800000000651B002093
:10020000300000007E000000E0F80008040000005C
:10021000F0180020B004000000C20100DCF8000863
:1002200004000000F4180020B0040000004B00009F
:10023000F0F8000800000000F8180020000000009E
:100240000100000006F9000800000000F918002075
:1002500000000000010000001CF900080000000080
:10026000EC180020000000000400000025F9000840
:1002700001000000ED180020000000000400000054
:1002800032F9000800000000E01800200000000023
:100290000300000040F9000800000000FA180020E8
:1002A000000000000100000053F9000800000000F9
:1002B000FB180020000000000200000062F90008A6
:1002C00000000000FC1800200000000001000000F9
:1002D00073F9000800000000D41800200A00000094
:1002E000C80000007DF9000800000000D5180020BB
:1002F0000A0000003200000090F900080000000031
:10030000D61800200A00000032000000A3F90008FF
:1003100000000000D71800200000000009000000C5
:10032000B5F9000800000000B2180020000000002D
:1003300008000000C0F9000800000000B318002009
:100340000000000008000000CAF9000800000000DA
:10035000B41800200000000008000000D4F90008D4
:1003600003000000B61800204CFFFFFF68010000EA
:10037000E5F9000803000000B81800204CFFFFFF5B
:1003800068010000F7F9000803000000BA18002017
:100390004CFFFFFF6801000007FA000801000000A1
:1003A000BC180020FFFFFFFF010000001DFA00083D
:1003B00000000000BD180020000000000500000043
:1003C0002AFA000802000000C6180020640000009D
:1003D0008403000040FA000800000000C418002058
:1003E000000000008000000050FA00080200000039
:1003F000BE180020000000000001000059FA0008AB
:1004000002000000C018002064000000E8030000A3
:100410006AFA000802000000C21800206400000010
:10042000E80300007CFA0008000000000417002028
:100430000000000001000000EBFB000800000000CD
:100440007017002000000000200000008BFA000858
:100450000000000071170020000000006400000090
:1004600097FA000800000000721700200100000049
:10047000FA000000B1FA0008000000007317002025
:100480000000000001000000C6FA000800000000A3
:10049000761700200000000096000000E0FA000837
:1004A0000200000074170020010000008403000017
:1004B000FAFA0008000000002317002000000000E6
:1004C000FA00000002FB00080000000024170020D2
:1004D00000000000640000000AFB000800000000AB
:1004E00025170020000000006400000012FB000837
:1004F000000000002617002000000000640000003B
:100500001BFB00080000000027170020000000006F
:10051000640000002BFB00080000000028170020EA
:10052000000000006400000033FB00080000000031
:100530002917002000000000640000003BFB0008B9
:10054000020000002A170020E8030000D007000086
:100550004AFB000800000000B8170020000000005F
:10056000C800000059FB000800000000B917002077
:1005700000000000C80000006CFB00080200000042
:10058000BA170020E8030000D00700007EFB000837
:1005900002000000BC17002064000000D00700002B
:1005A00098FB000801000000EB180020000000008C
:1005B00004000000A9FB000801000000BE17002095
:1005C000FFFFFFFF01000000B7FB00080100000073
:1005D000BF1700200000000001000000C9FB000858
:1005E00000000000C017002000000000FF00000015
:1005F000D6FB0008000000003217002000000000B9
:10060000FA000000E5FB000800000000341700209D
:100610000000000064000000F4FB0008000000007F
:1006200033170020000000006400000002FC0008F6
:10063000000000004417002000000000010000003E
:1006400011FC00080300000030170020D4FEFFFF5B
:100650002C01000020FC0008030000002E170020E1
:10066000D4FEFFFF2C0100002EFC0008000000005B
:100670003517002000000000300000003CFC00089E
:1006800005000000381700200000000001000000F5
:100690004BFC0008050000003C1700200000000093
:1006A0000100000057FC0008050000004017002072
:1006B000000000000100000063FC000803000000CF
:1006C0002C170020B0B9FFFF5046000073FC000853
:1006D000000000000917002000000000C800000012
:1006E0007DFC00080000000013170020000000003F
:1006F000C800000087FC0008000000001D17002053
:1007000000000000C800000091FC0008000000008C
:100710000A17002000000000C80000009CFC000830
:10072000000000001417002000000000C8000000B6
:10073000A7FC0008000000001E17002000000000B9
:10074000C8000000B2FC0008000000000B170020E9
:1007500000000000C8000000BCFC00080000000011
:100760001517002000000000C8000000C6FC0008AB
:10077000000000001F17002000000000C80000005B
:10078000D0FC000802000000C2170020000000009A
:10079000D0070000DEFC000800000000C6170020A3
:1007A0000000000001000000F3FC0008020000004F
:1007B000C81700200A000000D007000001FD000853
:1007C00002000000CA1700200A000000D007000045
:1007D0000FFD000800000000C51700200000000009
:1007E000640000001DFD0008000000000617002046
:1007F00000000000C800000025FD00080000000007
:100800001017002000000000C8000000EFF90008E9
:10081000000000001A17002000000000C8000000BF
:100820002DFD00080000000005170020000000005A
:10083000C800000034FD0008000000000F17002071
:1008400000000000C8000000DEF900080000000001
:100850001917002000000000C80000003BFD000840
:10086000000000000717002000000000C800000082
:1008700041FD0008000000001117002000000000EA
:10088000C800000001FA0008000000001B1700204B
:1008900000000000C800000047FD00080000000044
:1008A0000817002000000000C80000004DFD0008EF
:1008B000000000001217002000000000C800000027
:1008C00053FD0008000000001C170020000000007D
:1008D000C800000059FD0008000000000C170020AF
:1008E00000000000C800000061FD000800000000DA
:1008F0001617002000000000C800000069FD000875
:10090000000000002017002000000000C8000000C8
:1009100071FD0008000000000E170020000000001C
:10092000C800000077FD0008000000001817002034
:1009300000000000C80000007DFD0008000000006D
:100940002217002000000000C8000000524F4C4C4D
:100950003B50495443483B5941573B414C543B5011
:100960006F733B506F73523B4E6176523B4C455612
:10097000454C3B4D41473B56454C3B0041524D3B5E
:1009800000414E474C453B00484F52495A4F4E3B61
:10099000004241524F3B00564152494F3B004D41AE
:1009A000473B0048454144465245453B0048454188
:1009B0004441444A3B0043414D535441423B004370
:1009C000414D545249473B0047505320484F4D45F5
:1009D0003B0047505320484F4C443B005041535339
:1009E000544852553B004245455045523B004C450A
:1009F000444D41583B004C45444C4F573B004C4CF8
:100A000049474854533B0043414C49423B00474F00
:100A10005645524E4F523B004F53442053573B00D4
:100A200054454C454D455452593B00000000004B85
:100A3000000000CB61636F736600000000000000DF
:100A40007371727466000000000FC93F000F4940C7
:100A500000CB9640000FC9400053FB4000CB16412D
:100A600000ED2F41000F49410031624100537B41AD
:100A7000003A8A4100CB9641005CA34100EDAF41B2
:100A8000007EBC41000FC94100A0D5410031E241C8
:100A900000C2EE410053FB4100F20342003A0A4219
:100AA0000083104200CB164200141D42005C23421A
:100AB00000A5294200ED2F4200363642007E3C421E
:100AC00000C74242000F4942A2000000F9000000A6
:100AD000830000006E0000004E0000004400000093
:100AE0001500000029000000FC00000027000000A5
:100AF00057000000D1000000F500000034000000A5
:100B0000DD000000C0000000DB000000620000000B
:100B100095000000990000003C0000004300000028
:100B20009000000041000000FE00000051000000A5
:100B300063000000AB000000DE000000BB0000000E
:100B4000C500000061000000B700000024000000A4
:100B50006E0000003A000000420000004D0000005E
:100B6000D2000000E0000000060000004900000084
:100B70002E000000EA00000009000000D100000083
:100B8000920000001C000000FE0000001D0000009C
:100B9000EB0000001C000000B10000002900000074
:100BA000A70000003E000000E800000082000000F6
:100BB00035000000F50000002E000000BB00000022
:100BC0004400000084000000E90000009C000000D8
:100BD0007000000026000000B40000005F0000006C
:100BE0007E0000004100000039000000910000007C
:100BF000D600000039000000830000005300000010
:100C000039000000F40000009C0000008400000097
:100C10005F0000008B000000BD000000F900000034
:100C2000280000003B0000001F000000F80000004A
:100C300097000000FF000000DE000000050000003B
:100C4000980000000F000000EF0000002F000000DF
:100C5000110000008B0000005A0000000A00000094
:100C60006D0000001F0000006D0000003600000055
:100C70007E000000CF00000027000000CB00000035
:100C800009000000B70000004F000000460000000F
:100C90003F000000660000009E0000005F000000B2
:100CA000EA0000002D000000750000002700000091
:100CB000BA000000C7000000EB000000E5000000E3
:100CC000F10000007B0000003D0000000700000074
:100CD00039000000F70000008A0000005200000008
:100CE00092000000EA0000006B000000FB00000022
:100CF0005F000000B10000001F0000008D00000038
:100D00005D00000008000000560000000300000025
:100D10003000000046000000FC0000007B000000E6
:100D20006B000000AB000000F0000000CF000000EE
:100D3000BC000000200000009A000000F400000049
:100D4000360000001D000000A9000000E3000000C4
:100D500091000000610000005E000000E60000005D
:100D60001B00000008000000650000009900000062
:100D7000850000005F00000014000000A0000000DB
:100D800068000000400000008D000000FF0000002F
:100D9000D8000000800000004D000000730000003B
:100DA00027000000310000000600000006000000DF
:100DB0001500000056000000CA000000730000008B
:100DC000A8000000C900000060000000E200000070
:100DD0007B000000C00000008C0000006B000000E1
:100DE0000400000007000000090000000000C93FE7
:100DF0000000F0390000DA370000A2330000842E32
:100E00000000502B0000C2270000D0220000C41FA9
:100E10000000C61B000044176937AC31682122333B
:100E2000B40F14336821A2333863ED3EDA0F493F23
:100E30005E987B3FDA0FC93F002020202020202031
:100E4000202028282828282020202020202020207A
:100E5000202020202020202020881010101010108A
:100E600010101010101010101004040404040404D6
:100E70000404041010101010101041414141414170
:100E80000101010101010101010101010101010152
:100E90000101010110101010101042424242424262
:100EA0000202020202020202020202020202020222
:100EB00002020202101010102000000000000000CA
:100EC0000000000000000000000000000000000022
:100ED0000000000000000000000000000000000012
:100EE0000000000000000000000000000000000002
:100EF00000000000000000000000000000000000F2
:100F000000000000000000000000000000000000E1
:100F100000000000000000000000000000000000D1
:100F200000000000000000000000000000000000C1
:100F3000000000000000000000000000430000006E
:100F400070010020F8B500BFF8BC08BC9E46704791
:0C0F5000F8B500BFF8BC08BC9E46704716
:080F5C004DE600083501000814
:040F6400110100086F
:100F68000403010103010100D90303011D36000830
:100F78000100000100007A440000000000000000A9
:100F8800DC05DC05DC05DC05DC05DC05DC05DC0551
:100F98000000803F000000007C09010800000000FC
:100FA80001000000810901080100000002000000A2
:100FB80088090108020000000300000091090108E7
:100FC8000300000004000000970901080400000065
:100FD800050000009E090108050000000600000049
:100FE800A30901080600000007000000AD09010878
:100FF8000700000008000000B6090108080000000A
:1010080009000000BF090108090000000A000000EB
:10101800C80901080A0000000B000000D2090108F5
:101028000B0000000C000000DC0901080C000000A7
:101038000D000000E60901080D0000000E00000088
:10104800EE0901080E0000000F000000F609010873
:101058000F00000010000000FE0901081000000049
:1010680011000000070A010811000000120000002A
:101078000E0A01081200000013000000180A0108F7
:101088001300000014000000200A010814000000EA
:101098001500000000000000FF0000000000000034
:1010A80000000000010203040607080900127A0084
:1010B80000A24A040204060800000000010203041A
:1010C800010203040607080901000000380E0108A0
:1010D800000000005C040020C40400202C0500204F
:1010E80000000000000000000000000000000000F8
:1010F80000000000000000000000000000000000E8
:10110800000000003C0F0108000000000000000083
:1011180000000000000000000000000000000000C7
:1011280000000000000000000000000000000000B7
:1011380000000000000000000000000000000000A7
:101148000000000000000000000000000000000097
:101158000000000000000000000000000000000087
:101168000000000000000000000000000000000077
:101178000000000000000000010000000000000066
:101188000E33CDAB34126DE6ECDE05000B0000002B
:101198000000000000000000000000000000000047
:1011A8000000000000000000000000000000000037
:1011B8000000000000000000000000000000000027
:1011C8000000000000000000000000000000000017
:0C14F80000000000000000007001002057
:0400000508000000EF
:00000001FF
